:100000000C9436080C9455080C9455080C9455081B
:100010000C9455080C9455080C94A60A0C94DC0A10
:100020000C9455080C9455080C9455080C945508DC
:100030000C9455080C9455080C9455080C94360EE5
:100040000C9455080C9455080C9455080C945508BC
:100050000C94BC560C94C84D0C9455080C9455083F
:100060000C9455080C949E4E0C9455080C94924E8A
:100070000C9455080C9455080C9455080C9455088C
:100080000C947F620C9455080C9455080C945508F8
:100090000C94DC4E0C9455080C94D04E0C945508DE
:1000A0000C9455080C9455080C9455080C9455085C
:1000B0000C9455080C9455080C9455080C9455084C
:1000C0000C9455080C9455080C9455080C9455083C
:1000D0000C9455080C9455080C9455080C9455082C
:1000E0000C9455080C9475560C947F560C946B56D2
:1000F0000C9425560C94B0560C94A1560C9495561D
:100100000C9489560C9455080C9455080C94550879
:100110000C9455080C9455080C9455080C945508EB
:1001200007634236B79BD8A71A39685618AEBAABE0
:10013000558C1D3CB7CC5763BD6DEDFD753EF61774
:100140007231BF000000803F08000000BE922449C9
:10015000123EABAAAA2ABECDCCCC4C3E00000080F9
:10016000BEABAAAAAA3E00000000BF000000803F6C
:100170000000000000084178D3BB4387D1133D192C
:100180000E3CC3BD4282AD2B3E68EC8276BED98F59
:10019000E1A93E4C80EFFFBE01C4FF7F3F0000009D
:1001A0000000503A20256C642050612020252D3716
:1001B0002E3266206D0A0025630025630049324314
:1001C0003A2000256300256C642050612020252DF5
:1001D000372E3266206D00256C6420432000256395
:1001E00000545F52483D252D342E31662000524880
:1001F0003D252D342E3166200025630025630050F7
:100200007772313D25730A0044656275673D307829
:10021000252D780A00496E7075742050313D257384
:100220000A0048554D5F5057525F414C5741595352
:100230003D25730A0025730A006175746F0A004C2E
:100240006F67206D6F64653D00496E74722E205398
:1002500065633A20202050303D252D372E3366200F
:1002600050313D252D372E33660A00496E74722EAB
:1002700020546F74616C3A2050303D252D6C642001
:1002800050313D252D6C640A005553425F50575242
:100290003D25730A00565F4D43553D252D352E32C1
:1002A000660A00565F494E3D252D352E32660A00FE
:1002B0005265706F7274204D61736B3D3078252DDF
:1002C0007820005265706F727420496E7465727682
:1002D000616C3D252D640A0052494D4520616464DE
:1002E000723D252D642E252D640A004E65696768D0
:1002F000626F72207461626C652073697A653D2556
:10030000640A00545820506F7765723D25640A00D6
:100310004932433A200049443D007478743D2573C6
:100320000A0053797374656D2053756D6D61727930
:100330000A0025630025630043757272656E7420A0
:100340007265706F727420696E74657276616C3D4F
:10035000252D64207365630A004E657720726570F1
:100360006F727420696E74657276616C3D252D64C0
:10037000207365630A002563005573696E672072F8
:1003800065706F72743D3078252D6C7820004E6555
:1003900077207265706F72743D3078255820002583
:1003A0006300256300256300256300204F5343430A
:1003B000414C3D2564200020467573653A206565F3
:1003C0003D253032782068663D25303278206C66D5
:1003D0003D25303278206C623D25303278004D4327
:1003E000553D2530366C7800256300252D31306C65
:1003F0007520252D31306C7520252D31306C752000
:10040000252D31306C75200A007478206C656E20C3
:10041000202020207268206D6973732020202072B4
:1004200068207374616C652020207268206D697388
:10043000630A002563004F4B0A0025630025630013
:10044000256300445F434F4D504153533D30782561
:10045000780A00445F414343454C3D307825780A93
:1004600000445F505245533D307825780A00445F80
:100470005057525F313D307825780A00445F41453E
:10048000533D307825780A00445F50315F4C454435
:100490003D307825780A00445F50305F4C45443D3C
:1004A000307825780A00445F4556454E543D3078F3
:1004B00025780A00445F504F5745523D30782578E3
:1004C0000A00445F4C45443D307825780A00445F7B
:1004D0004F573D307825780A00445F504B543D6EAD
:1004E000307825780A00445F54583D307825780AE2
:1004F00000445F52583D307825780A00445F4F50E1
:1005000045523D307825780A0043757272656E74E5
:100510002064656275673D307825580A004E65771E
:100520002064656275673D307825580A0025730A96
:100530000025372E33662025372E33660025352ECD
:10054000326620004572726F72203020566F6C74D4
:10055000004E6F7420737570706F727465640A005A
:100560004572726F72203020566F6C740045727243
:100570006F72203020566F6C740025730A00545837
:1005800020506F7765723D25640A005465737420AE
:10059000342025730A005465737420332025730AB0
:1005A000005465737420322025730A0054657374F7
:1005B00020312025730A0025730A0025730A0025BF
:1005C000730A0025730A005854414C5F5452494D38
:1005D0003D25640025730A0050413D090930782506
:1005E0006C7800503D09093078256C780041323D27
:1005F0000909307825780041313D0909307825789E
:1006000000565F494E3D0909307825780052483D33
:1006100009093078257800555054494D453D090960
:10062000307825780050315F543D090930782578BD
:100630000050313D0909307825780050305F543D35
:100640000909307825780050303D0909307825783F
:1006500000565F4D43553D09093078257800545FB9
:100660004D43553D0909307825780054313D09093D
:100670003078257800543D090930782578004944C0
:100680003D090930782578005458543D09093078DF
:100690002578005041200050200041322000413197
:1006A0002000565F494E20005248200055505449C2
:1006B0004D45200050315F54200050312000503013
:1006C0005F54200050302000565F4D4355200054A9
:1006D0005F4D4355200054312000542000494420F0
:1006E000005458542000253032780025372E3366C8
:1006F0002025372E33660025352E32662000204E09
:10070000657665722D7573656420737461636B2003
:100710003E2025642062797465730A0055707469FF
:100720006D6520256420646179732C202530326446
:100730003A253032643A253032640A0074657374A5
:10074000205B6F66667C317C327C335D202020200C
:1007500020202020202020202D2074657374206DFF
:100760006F6465730A0D00776474205B6F6E7C6F35
:1007700066667C746573745D202020202020202014
:100780002020202D207761746368646F670A0D0054
:10079000757067722020202020202020202020201B
:1007A0002020202020202020202020202D207265A5
:1007B000626F6F742076696120626F6F746C6F6115
:1007C0006465720A0D00626F6F7420202020202063
:1007D0002020202020202020202020202020202019
:1007E00020202D207265626F6F740A0D0070777281
:1007F00073205B646565707C666F7263655F6964B6
:100800006C655D2020202020202D206D63752073D5
:100810006C656570206D6F64650A0D007265737498
:1008200020656570726F6D20202020202020202000
:1008300020202020202020202D20726573746F72CC
:100840006520656570726F6D0A0D007031205B6FF9
:100850006E7C6F66665D20202020202020202020D6
:10086000202020202020202D2064697361626C6587
:100870002070756C736520703120746F2073617601
:100880006520706F7765720A0D0070777231205B9A
:100890006F6E7C6F66665D20202020202020202047
:1008A0002020202020202D2070696E31207077724A
:1008B0000A0D0074787077205B31352D305D202073
:1008C0002020202020202020202020202020202D1B
:1008D000205458205077722E2048696768657374D9
:1008E000203020283364426D290A0D00747874206A
:1008F0005B737472696E675D2020202020202020A9
:1009000020202020202020202D2053657420726577
:10091000706F7274207465787420737472696E6776
:100920000A0D00737320202020202020202020206A
:100930002020202020202020202020202020202DAA
:100940002073797374656D2073756D6D6172790AAA
:100950000D00727320202020202020202020202025
:1009600020202020202020202020202020202D207A
:10097000726164696F2073746174730A0D00726927
:10098000205B696E745D2020202020202020202004
:10099000202020202020202020202D207265706F14
:1009A000727420696E74657276616C0A0D007265EE
:1009B000205B6D61736B5D20202020202020202093
:1009C000202020202020202020202D206D6F7465E5
:1009D000207265706F72742073657474696E670A33
:1009E0000D006F7720202020202020202020202094
:1009F00020202020202020202020202020202D20EA
:100A00006F6E652D776972652073656E736F727393
:100A10000A0D006C6F67205B6175746F7C6F6E7C74
:100A20006F66665D20202020202020202020202DA1
:100A3000206D6F7465732064617461206F6E205542
:100A400053420A0D006E65205B666C7573685D200D
:100A50002020202020202020202020202020202096
:100A6000202D206E65696768626F72207461626C08
:100A7000650A0D0065727220202020202020202091
:100A80002020202020202020202020202020202066
:100A90002D206572726F7220696E666F0A0D006D8F
:100AA00063752020202020202020202020202020AE
:100AB00020202020202020202020202D206D637544
:100AC00020696E666F0A0D006964205B726573654C
:100AD000745D202020202020202020202020202085
:100AE000202020202D2069642068616E646C696E6E
:100AF000670A0D0068756D70205B6F6E7C6F6666AF
:100B00005D202020202020202020202020202020A8
:100B10002D2068756D6964697479207065726D2027
:100B200073656E736F72207077720A0D0068756D51
:100B300020202020202020202020202020202020B5
:100B40002020202020202020202D2068756D696421
:100B50006974792073656E736F720A0D0064652085
:100B60005B6D61736B5D20202020202020202020E1
:100B70002020202020202020202D20646562756701
:100B80000A0D0063616C69205B5B765F696E7C6156
:100B9000317C61325D20766F6C747C726573657434
:100BA0007C6E6F6E655D202D2063616C6962726181
:100BB00074650A0D0061646320202020202020201D
:100BC0002020202020202020202020202020202025
:100BD000202D2073686F7720765F696E2C2061313D
:100BE0002C20613220766F6C74616765730A0D008A
:100BF000616573205B6F6E7C6F66665D20202020D0
:100C00002020202020202020202020202D20696E40
:100C1000746567726574790A0D00752020202020A4
:100C200020202020202020202020202020202020C4
:100C30002020202020202D20757074696D650A0DFC
:100C4000007620202020202020202020202020206E
:100C5000202020202020202020202020202D207631
:100C6000657273696F6E0A0D0068202020202020B5
:100C70002020202020202020202020202020202074
:100C800020202020202D2068656C700A0D0025632F
:100C900000756E6B6E6F776E20636D640A004E4850
:100CA00044433032313620004C3347343230304404
:100CB0002000484D433538383320004144584C33E8
:100CC00034352000424D50303835200048494836F0
:100CD0003133302000415432344D4143200020252F
:100CE00073002025362E3266200025303278002011
:100CF0002573002025362E3266204F6E2D426F61FF
:100D000072640025303278000A00452025642E25C3
:100D10006420636C6F636B20256C75206370752095
:100D2000256C75206C706D20256C752069727120A2
:100D3000256C7520676C656420256C7520796C6561
:100D40006420256C7520726C656420256C75207498
:100D50007820256C75206C697374656E20256C7520
:100D60002073656E736F727320256C7520736572C6
:100D700069616C20256C750A00532025642E25645A
:100D800020636C6F636B20256C7520747820256C54
:100D90007520727820256C752072747820256C750A
:100DA0002072727820256C75207265786D697420C8
:100DB000256C752061636B747820256C75206E6FCF
:100DC00061636B747820256C752061636B72782089
:100DD000256C752074696D65646F757420256C755C
:100DE0002062616461636B727820256C7520746F7A
:100DF0006F6C6F6E6720256C7520746F6F73686FF2
:100E0000727420256C752062616473796E6368204A
:100E1000256C752062616463726320256C752063A4
:100E20006F6E74656E74696F6E64726F7020256C7E
:100E3000752073656E64696E6764726F7020256CCF
:100E400075206C6C747820256C75206C6C72782021
:100E5000256C750A00257325730A004F6E6C696E48
:100E6000650A000A002C20636865636B2072617458
:100E70006520257520487A0025732025732C206372
:100E800068616E6E656C20257520706F77657220C5
:100E90002575000A0025783A004D414320616464BD
:100EA00072657373200052616E646F6D2045554901
:100EB000363420616464726573732067656E657291
:100EC000617465640A000A2A2A2A2A2A2A2A426F99
:100ED0006F74696E672025732A2A2A2A2A2A2A0A09
:100EE00000020000FFFE00000141544D4547413122
:100EF000323872666131006C6F63616C686F737455
:100F000000454550524F4D20697320636F727275D2
:100F100070742C20726577726974696E67207769C6
:100F200074682064656661756C74732E0A006E6166
:100F30006E00696E660000407A10F35A00A0724E8F
:100F400018090010A5D4E80000E87648170000E46E
:100F50000B54020000CA9A3B000000E1F5050000B6
:100F600080969800000040420F000000A08601001B
:100F70000000102700000000E803000000006400EB
:100F8000000000000A000000000001000000000056
:100F90002C76D888DC674F0823DFC1DFAE59E1B17A
:100FA000B796E5E3E453C63AE651997696E8E6C289
:100FB0008426EB898C9B62ED407C6FFCEFBC9C9F90
:100FC00040F2BAA56FA5F490055A2AF75C936B6CB2
:100FD000F9676DC11BFCE0E40D47FEF520E6B500A6
:100FE000D0ED902E0300943577050080841E080014
:100FF00000204E0A000000C80C333333330F986EC4
:1010000012831141EF8D2114893BE65516CFFEE680
:10101000DB18D1844B381BF77C1D901DA4BBE42446
:10102000203284725E228100C9F124ECA1E53D27C3
:10103000494E46494E4954594E414ECDCCCC3D0ABD
:10104000D7233C17B7D13877CC2B329595E6241FA0
:10105000B14F0A000020410000C84200401C462059
:10106000BCBE4CCA1B0E5AAEC59D740011241FBED7
:10107000CFEFD1E4DEBFCDBF16E0A0E0B2E0E8E8FC
:10108000FBEF00E00BBF02C007900D92AE3CB10732
:10109000D9F71DE2AEECB6E001C01D92A238B1074F
:1010A000E1F70E94824C0C94C27D0C94000029E070
:1010B000FC0120935700C895802D0895E091A71753
:1010C000F0E0EF71F070E450F84E80838091A71744
:1010D0008F5F8093A7178091BC2488608093BC2485
:1010E0004FED54E0CA0161E10E94CA3D80E090E00A
:1010F00008954F925F926F927F928F929F92AF92DC
:10110000BF92CF92DF92EF92FF920F931F93DF93E4
:10111000CF93CDB7DEB760970FB6F894DEBF0FBEA2
:10112000CDBF3B018091CE069091CF0681FD749892
:101130000E9492446C01DC018C91982F92959F70D3
:10114000913009F05CC190E08F709070009709F4C5
:1011500056C181EC94E2B3010E94973B009709F0DD
:101160004EC183EF96E00E94C13E1CC0C8010296AA
:10117000B3010E94973B009791F0C8010D9660E083
:1011800074E649E25AE098010E948641F601918195
:10119000D80118968C911897981761F530C1C8013D
:1011A0000E94873F082F192F01151105F9F62FC14D
:1011B000C8010296B3010E948E3BF60181818150E5
:1011C000D80118968C9380E091E0A0E0B0E0F8019F
:1011D00081879287A387B48783EF96E0B8010E9446
:1011E000483FC8010D9660E074E649E25AE0980174
:1011F0000E94864184E00E94C645D80115969C93C2
:101200008E93149783E00E94C6452C01F8019783C2
:101210008683D60111968C908085881A9924AA24F9
:10122000BB2486E0880C991CAA1CBB1C8A95D1F7AC
:10123000618572858385948520EC30E040E050E044
:101240000E94D476672F782F892F9927860E971EB4
:10125000A81EB91EF80181869286A386B486D6019F
:1012600011968C91119780878091CE069091CF0630
:1012700081FD08C08091B90480FD04C081FFBFC01A
:101280001D9BBDC0EDB7FEB774970FB6F894FEBFB7
:101290000FBEEDBFEDB6FEB60894E11CF11C80E078
:1012A00092E092838183C6010296D70113969C93A4
:1012B0008E931297F301808114968C931497159650
:1012C0001C921597818116968C93169717961C92EF
:1012D000D60111968C911197F701808711868C9118
:1012E00090E08F70907093878287D80114968D91CB
:1012F0009C9115979587848757864686BB27AB2D8B
:101300009A2D892D918B808BC501B40124E630E0A4
:1013100040E050E00E94D476672F782F892F9927DC
:101320000E941A77F701738B628B0E949A7A209140
:101330009C048DB79EB744960FB6F8949EBF0FBE1F
:101340008DBF2223A9F000D000D0EDB7FEB73196B3
:101350008AEB91E0ADB7BEB712969C938E9311972E
:10136000228313820E94AC7A0F900F900F900F90FF
:101370008091451C86FF43C00E94784AC6010596AD
:101380000E94374AEDB7FEB73C970FB6F894FEBF00
:101390000FBEEDBF31967E010894E11CF11CADB784
:1013A000BEB71296FC92EE92119780E190E0938383
:1013B000828384E492E095838483D80114968D918E
:1013C0009C9115979783868316968D919C9117977C
:1013D00091878087D60111968C91828713860E940F
:1013E0000A7BEDB7FEB73C960FB6F894FEBF0FBE72
:1013F000EDBF82E00E94544AC7010E94374A8091A3
:10140000CE069091CF0681FF0DC0749A0BC088E480
:1014100095E00E94553E082F192F0115110509F07E
:10142000C7CEEDCF60960FB6F894DEBF0FBECDBF2E
:10143000CF91DF911F910F91FF90EF90DF90CF90B0
:10144000BF90AF909F908F907F906F905F904F90E4
:101450000895EF92FF92CF93DF93E82EE7017E018C
:10146000F92EE7018091CE069091CF0687FF2FC01D
:101470008DB79EB70C970FB6F8949EBF0FBE8DBF69
:10148000EDB7FEB7319687E592E0ADB7BEB71296DD
:101490009C938E9311978A81828313828B8184839C
:1014A00015828885868317828C819D8191878087AC
:1014B0008E819F81938782870E949A7A2DB73EB74B
:1014C000245F3F4F0FB6F8943EBF0FBE2DBF83EF92
:1014D00096E0BE010E940F3F88E495E0BE010E94A5
:1014E0007B3EDF91CF91FF90EF90089587EE93E0E0
:1014F0008115910511F00197F1F70895882369F09E
:101500006D987598ED9A80916A00886080936A0062
:10151000809168008160809368008091B904909107
:10152000BA0491FF10C06E988EB18F6B8EB9EE9A8F
:1015300080916A00806280936A0080916800816077
:10154000809368000895769AEE9808951F920F92FE
:101550000FB60F9211248F939F93AF93BF938091F7
:10156000680080FF20C080919C2490919D24A091D0
:101570009E24B0919F240196A11DB11D80939C24AF
:1015800090939D24A0939E24B0939F248091CE0697
:101590009091CF0690FF07C0749882E090E09093FE
:1015A0008F0480938E04BF91AF919F918F910F9084
:1015B0000FBE0F901F9018951F920F920FB60F92AB
:1015C00011248F939F93AF93BF938091680080FF06
:1015D00020C08091A0249091A124A091A224B09138
:1015E000A3240196A11DB11D8093A0249093A12452
:1015F000A093A224B093A3248091CE069091CF060D
:1016000091FF07C0739882E090E090938F048093DD
:101610008E04BF91AF919F918F910F900FBE0F904D
:101620001F90189580937C0080917B00877F80932A
:101630007B0080917C00806C80937C0085E08093AF
:101640007A0080917A00806880937A0080917B0094
:1016500087FFFCCF80917B0085FFFCCF80917A00D3
:10166000806480937A0080917A0086FDFCCF10928E
:1016700079001092780084E090E060E070E02091C2
:101680007A00206420937A0020917A0026FDFCCF16
:101690002091780030917900620F731F019779F7DC
:1016A00010927C0080917A008F7780937A007695F3
:1016B00067957695679580E090E00E945A7408954A
:1016C00080E00E94120B209190043091910440918F
:1016D0009204509193040E940C7521EE3AE744E97C
:1016E0005EE30E948A73089580E1809351018093A4
:1016F00051019091510195FF03C08F5F8F31B9F770
:101700006BE4869FB0011124882777FD8095982F80
:101710000E945C7420E030E64FE954E40E948A7332
:1017200020E030E04AE754E40E94F273089580918B
:10173000B30484FF4BC080917B00886080937B0062
:1017400089EC80937C0085E080937A0080917A0018
:10175000806880937A0080917B0087FFFCCF809126
:101760007B0085FFFCCF80917A00806480937A00B3
:1017700080917A0086FDFCCF80917A00806480930E
:101780007A0080917A0086FDFCCF6091780070919C
:10179000790080E090E00E945A7427ED33EA40E936
:1017A0005FE30E940C7526E636E648E853E40E94A3
:1017B000897360939C1770939D1780939E179093E5
:1017C0009F1780917A008F7780937A0008956F92A7
:1017D0007F928F929F92AF92BF92CF92DF92EF92C1
:1017E000FF920F931F93DF93CF93CDB7DEB72A9766
:1017F0000FB6F894DEBF0FBECDBF3C011092D606E7
:101800008FEF898358EBC52E57E1D52E00E010E00D
:1018100042E0E42EF12CEC0EFD1E4E010894811CDA
:10182000911C3AE0A32EB12CAC0EBD1E3FC0083077
:10183000110509F441C0C401B7012A870E948447F9
:1018400089812A858F3F11F08E3F19F48093D60647
:1018500034C06114710479F4C7010E949E478093DB
:10186000B924F701A1EBB4E281918D93EA15FB0550
:10187000D9F721E022C0C7010E949E47F60180836C
:10188000D701F80123E0EE0FFF1F2A95E1F7E00FE3
:10189000F11FE055F84E8D918193AA15BB05D9F73C
:1018A0000F5F1F4F89E090E0C80ED91E202F89815D
:1018B000882309F0BCCF01C028E0822F2A960FB6FA
:1018C000F894DEBF0FBECDBFCF91DF911F910F9176
:1018D000FF90EF90DF90CF90BF90AF909F908F9050
:1018E0007F906F90089500D088E09DE0EDB7FEB73F
:1018F000928381830E94AC7A0F900F9008952F926B
:101900003F924F925F926F927F928F929F92AF928F
:10191000BF92CF92DF92EF92FF920F931F93DF93CC
:10192000CF9300D000D0CDB7DEB78C01009741F443
:1019300089E290E06BE270E04AE250E027E00AC002
:101940008130910549F489E290E06BE270E04AE26F
:1019500050E026E00E946046C8010E94E70BF801B3
:10196000EC52F94F808301151105A1F018EBC12E3F
:1019700017E1D12E00E010E04F01BAEE6B2EBCE073
:101980007B2EA2EE4A2EACE05A2EFEED2F2EFCE06E
:101990003F2EFAC081EB94E20E94D0489C01B9012D
:1019A000882777FD8095982F0E945C74C82EE92EB9
:1019B000E1EBAE2EE4E2BE2E03E01DE0D5018D91F9
:1019C0005D0100D000D0EDB7FEB73196ADB7BEB720
:1019D00012961C930E931197828313826B837C83E0
:1019E0000E94AC7A0F900F900F900F906B817C81CA
:1019F000B9EBAB16B4E2BB0609F700D000D000D0BB
:101A00000DB71EB70F5F1F4F23EF3CE0EDB7FEB7DA
:101A1000328321838C2D9E2D20E030E048EC52E46F
:101A20000E94F273D80112966D937D938D939C93CF
:101A300015970E94AC7AEDB7FEB736960FB6F894BC
:101A4000FEBF0FBEEDBF8091B924882319F086E850
:101A500092E002C08FE892E000D000D02FEE3CE090
:101A6000ADB7BEB712963C932E93119714969C93E4
:101A70008E9313970E94AC7A0F900F900F900F9057
:101A80000E94730C88C0780163E0EE0CFF1C6A951D
:101A9000E1F7E00EF11EE0EBF7E1EE0EFF1EC701ED
:101AA0000E94D0489C01B901882777FD8095982F26
:101AB0000E945C745C0120E030E0D7018D917D01D3
:101AC00000D000D0EDB7FEB73196ADB7BEB71296D5
:101AD0007C926E9211978283138229833A836B835F
:101AE0007C830E94AC7A29813A812F5F3F4F0F900F
:101AF0000F900F900F906B817C8128303105E9F6B3
:101B000000D000D000D0EDB6FEB60894E11CF11C68
:101B1000EDB7FEB7528241828A2D9B2D20E030E046
:101B200048EC52E40E94F273D70112966D937D93B4
:101B30008D939C9315970E94AC7AEDB7FEB73696BD
:101B40000FB6F894FEBF0FBEEDBFD6018C9188236F
:101B500019F086E892E002C08FE892E000D000D051
:101B6000EDB7FEB732822182948383830E94AC7AE0
:101B70000F900F900F900F900E94730C0F5F1F4FEC
:101B800029E030E0C20ED31ED4018C9190E00817FA
:101B900019070CF478CF0F900F900F900F90CF9102
:101BA000DF911F910F91FF90EF90DF90CF90BF904A
:101BB000AF909F908F907F906F905F904F903F90ED
:101BC0002F900895DF93CF9300D0CDB7DEB78091EB
:101BD000B22489838091B8248A83CE0101960E9421
:101BE000A93B0F900F90CF91DF910895CF93DF9392
:101BF000EC018091B1248F3FB1F58091B2248F3FE9
:101C000091F58091B3248F3F71F58091B4248F3F7B
:101C100051F58091B5248F3F31F58091B6248F3FE7
:101C200011F58091B7248F3FF1F48091B8248F3F54
:101C3000D1F489E290E06BE270E04AE250E027E004
:101C40000E94604680E090E00E94E70BCC52D94FA2
:101C5000888381EB94E267E170E049E050E00E9404
:101C6000FC7B0E94E20DDF91CF9108951F920F92AD
:101C70000FB60F920BB60F9211242F933F934F93F1
:101C80005F936F937F938F939F93AF93BF93EF93E4
:101C9000FF938091BC2482608093BC248091B9041E
:101CA00086FD2B9A8091B90487FD2B9A80918E0432
:101CB00090918F041816190614F4749A739A8091EF
:101CC000CE069091CF0685FF02C0749873988091DC
:101CD00050059091510501979093510580935005BF
:101CE000009709F068C08091020790910307019660
:101CF000909303078093020720914720309148205A
:101D00004091492050914A202F5F3F4F4F4F5F4FE6
:101D100020934720309348204093492050934A20F5
:101D200020E130E030935105209350052091B90413
:101D300020FD02C01D9B05C01092D2061092D10654
:101D400006C021E030E03093D2062093D1066091A6
:101D5000B7047091B8046115710599F001960E945D
:101D6000F376009771F477988091CE069091CF0624
:101D700093FF07C0749884E090E090938F04809361
:101D80008E046091B7047091B8046115710579F003
:101D900080910207909103070E94F376009739F42F
:101DA0008BEF94E062E140E050E00E94CA3D8091F8
:101DB000B90486FD2B988AE695E060E040E050E0AB
:101DC0000E94CA3DFF91EF91BF91AF919F918F917A
:101DD0007F916F915F914F913F912F910F900BBE2B
:101DE0000F900FBE0F901F9018958091A71790919C
:101DF0005B20891B08950E94F50E882379F0E091FD
:101E00005B20F0E0EF71F070E450F84E208130E09C
:101E100080915B208F5F80935B2002C02FEF3FEFAC
:101E2000C9010895CF93DF93EC011092F60610924A
:101E3000F50688819981009731F022E0853C920770
:101E400009F0B9C009C00E94F50E882341F485EC61
:101E500092E099838883B3C0613109F0B0C0F894EF
:101E600078940E94FB0E90E09093FA068093F90616
:101E70008D3009F47CC08F3F31F38231910569F1D7
:101E80008F37910521F08830910509F053C080917A
:101E9000FD069091FE06181619060CF060C06091C0
:101EA0007C2D70917D2D88E090E00E946E7A60918B
:101EB0007C2D70917D2D80E290E00E946E7A609181
:101EC0007C2D70917D2D88E090E00E946E7A80914B
:101ED000FD069091FE0601973EC060917C2D7091A9
:101EE0007D2D8DE090E00E946E7A1092FC0610929B
:101EF000FB0614C0845A9F4DFC01808160917C2DAB
:101F000070917D2D90E00E946E7A8091FB069091F9
:101F1000FC0601969093FC068093FB068091FB06DD
:101F20009091FC062091FD063091FE0682179307E2
:101F30000CF315C060917C2D70917D2D0E946E7AFE
:101F40008091FD069091FE062091F906FC01E45A6D
:101F5000FF4D208301969093FE068093FD068091AD
:101F6000FD069091FE068F33910509F06CCF10921B
:101F70005B2080915B208093A7178091FD06909154
:101F8000FE06FC01E45AFF4D10829093F606809302
:101F9000F5061092FE061092FD068091BA249091EB
:101FA000BB24009709F44FCF6091F70640E050E062
:101FB0000E94CA3D48CF1982188283E001C081E0A7
:101FC000DF91CF91089578948091D1069091D206B7
:101FD000009731F08091B9049091BA0490FF03C04A
:101FE00083B7817F03C083B7817F866083BFF89406
:101FF00083B7816083BF7894889583B78E7F83BFD2
:1020000078940895CF93DF93EC01888199810097AC
:1020100021F02AE08F33920799F40E94D94F0E9451
:10202000E30F8091880E9091890E65E840E050E0C2
:102030000E94CA3D8FE39AE09983888381E003C0C0
:102040001982188283E0DF91CF910895CF93DF93B7
:102050000E94D94F80EB0E9450498823B1F40E941E
:10206000B6498091451C9091461C81609093461C16
:102070008093451C00D085ED9CE0EDB7FEB79283C0
:1020800081830E94AC7A0F900F908EB1C82FD0E060
:10209000C470D070729A0E94D94F8EE40E94504949
:1020A0008823B1F40E94B6498091451C9091461C4A
:1020B00082609093461C8093451C00D08CEC9CE081
:1020C000EDB7FEB7928381830E94AC7A0F900F9098
:1020D000209709F472980E94D94F8EEE0E945049C1
:1020E0008823B1F40E94B6498091451C9091461C0A
:1020F00084609093461C8093451C00D084EC9CE047
:10210000EDB7FEB7928381830E94AC7A0F900F9057
:1021100086EA0E9450498823B1F40E94B649809112
:10212000451C9091461C88609093461C8093451CEA
:1021300000D08BEB9CE0EDB7FEB7928381830E94C9
:10214000AC7A0F900F900E94D94F8CE30E945049B7
:102150008823B1F40E94B6498091451C9091461C99
:1021600080619093461C8093451C00D082EB9CE0DC
:10217000EDB7FEB7928381830E94AC7A0F900F90E7
:102180000E94D94F82ED0E9450498823B1F40E94E9
:10219000B6498091451C9091461C80629093461CE4
:1021A0008093451C00D088EA9CE0EDB7FEB792838F
:1021B00081830E94AC7A0F900F90C7E0D0E00E941C
:1021C000D94F8CE70E9450498823B9F40E94B64940
:1021D0008091451C9091461C80649093461C80938E
:1021E000451C00D08EE99CE0EDB7FEB79283818359
:1021F0000E94AC7A0F900F9002C0219701F70E94C5
:10220000B6490E94730CDF91CF910895DF93CF936D
:1022100000D0CDB7DEB74A8369830E948C496981BB
:10222000862F0E94BE494A81842F0E94BE490E9487
:10223000B6490F900F90CF91DF910895AF92BF9262
:10224000DF92EF92FF920F931F93DF93CF9300D013
:102250000F92CDB7DEB7082FD22E4A835B836983F6
:102260000E948C496981862F0E94BE49802F81601F
:102270000E94B3494A815B81042F152FAA24BB24F5
:10228000ED2CFF240894E108F1080FC0AE14BF0440
:1022900019F40E94D94902C00E94CF49F8018083F5
:1022A0000894A11CB11C0F5F1F4FAD1478F30E945E
:1022B000B6490F900F900F90CF91DF911F910F9122
:1022C000FF90EF90DF90BF90AF9008958F929F9214
:1022D000AF92BF92CF92DF92EF92FF920F931F9334
:1022E000DF93CF93CDB7DEB760970FB6F894DEBF1C
:1022F0000FBECDBF8E010F5F1F4F80E1D8011D9231
:102300008A95E9F780EB68E9A80128E00E941E1190
:1023100000D080E992E0EDB7FEB7928381830E94FE
:102320009A7A680198E0892E912C8C0E9D1E0F9050
:102330000F90780187E9A82E82E0B82ED7018D9101
:102340007D0100D000D0EDB7FEB73196ADB7BEB776
:102350001296BC92AE921197828313820E949A7A4F
:102360000F900F900F900F90E814F90439F700D0F8
:1023700000D0EDB7FEB731968DE992E0ADB7BEB7AC
:1023800012969C938E9311978885828313820E9464
:102390009A7AAE014F5F5F4F80E1FA0111928A9500
:1023A000E9F70F900F900F900F9080EB60E828E016
:1023B0000E941E1100D083EA92E0ADB7BEB712961C
:1023C0009C938E9311970E949A7A015F1F4F0F90F2
:1023D0000F908A2CEB2CF60181916F0100D000D078
:1023E000EDB7FEB73196ADB7BEB711968C92119787
:1023F0001296EC92828313820E949A7A0F900F9029
:102400000F900F90C016D10631F700D000D0EDB775
:10241000FEB731968DE992E0ADB7BEB712969C93A8
:102420008E9311978885828313820E949A7A0F90E7
:102430000F900F900F9060960FB6F894DEBF0FBE0E
:10244000CDBFCF91DF911F910F91FF90EF90DF9063
:10245000CF90BF90AF909F908F9008950F931F9350
:10246000DF93CF9300D0CDB7DEB71A8219828EEEFC
:102470006AEA8E010F5F1F4FA80122E00E941E1121
:10248000398120E08A8190E0822B932B90931D1854
:1024900080931C188EEE6CEAA80122E00E941E11A7
:1024A000398120E08A8190E0822B932B90931F1832
:1024B00080931E188EEE6EEAA80122E00E941E1183
:1024C000398120E08A8190E0822B932B9093211810
:1024D000809320188EEE60EBA80122E00E941E116E
:1024E000398120E08A8190E0822B932B90932F18E2
:1024F00080932E188EEE62EBA80122E00E941E113E
:10250000398120E08A8190E0822B932B90933118BF
:10251000809330188EEE64EBA80122E00E941E1119
:10252000398120E08A8190E0822B932B909333189D
:10253000809332188EEE66EBA80122E00E941E11F5
:10254000398120E08A8190E0822B932B909323188D
:10255000809322188EEE68EBA80122E00E941E11E3
:10256000398120E08A8190E0822B932B909325186B
:10257000809324188EEE6AEBA80122E00E941E11BF
:10258000398120E08A8190E0822B932B9093291847
:10259000809328188EEE6CEBA80122E00E941E1199
:1025A000398120E08A8190E0822B932B90932B1825
:1025B00080932A188EEE6EEBA80122E00E941E1175
:1025C000398120E08A8190E0822B932B90932D1803
:1025D00080932C180F900F90CF91DF911F910F9146
:1025E00008952F923F924F925F926F927F928F92B7
:1025F0009F92AF92BF92CF92DF92EF92FF920F9392
:102600001F93DF93CF93CDB7DEB76C970FB6F894D7
:10261000DEBF0FBECDBFA82E4A8B2B8FFE01319699
:1026200083E0DF011D928A95E9F7809140188823A5
:1026300039F46C8F0E942E1281E0809340186C8DCB
:10264000662309F475C08EEE64EF4EE20E94061117
:1026500069E07AE180E090E00E943D498EEE66EF0D
:10266000AE014F5F5F4F22E00E941E11698170E052
:1026700080E090E0982F872F762F66272A8130E020
:1026800040E050E0622B732B842B952B2091321865
:102690003091331840E050E0621B730B840B950BB4
:1026A000209130183091311840E050E00E94D476EB
:1026B0007B018C013FE015950795F794E7943A95D7
:1026C000D1F760912A1870912B18882777FD809593
:1026D000982F2BE0660F771F881F991F2A95D1F737
:1026E00020912C1830912D18442737FD4095542FF8
:1026F0002E0D3F1D401F511F0E943C772E0D3F1D88
:102700003093271820932618285F3F4FB4E0359563
:102710002795BA95E1F779010027F7FC0095102F6E
:10272000E0923418F0923518009336181093371849
:10273000BA2DB295BB0FBB0FB07CBC5CB9872A2DFC
:1027400030E03E8B2D8B63E070E00A2C02C0660FF8
:10275000771F0A94E2F7882777FD8095982F25E365
:1027600035E040E050E00E94D476DC01CB010296D7
:10277000A11DB11D8A879B87AC87BD8720E533ECFF
:1027800040E050E004C05595479537952795AA94A9
:10279000D2F72E873F87488B598B18861C821D8263
:1027A0001E821F8248E050E08D899E89481B590B8C
:1027B0005C8B4B8B69C18EEE64EF49850E940611DC
:1027C0006A857B858C859D850E943D498EEE66EFEE
:1027D000AE014F5F5F4F23E00E941E1180912618CB
:1027E00090912718805A9F401C01442437FC409444
:1027F000542CC201B101A20191010E94D4766F8BC9
:10280000788F898F9A8F2091201830912118442732
:1028100037FD4095542FC201B1010E94D4767B014F
:102820008C01ADE015950795F794E794AA95D1F73B
:1028300022E030E040E050E0E20EF31E041F151FDE
:102840006F89788D898D9A8DFCE095958795779520
:102850006795FA95D1F720912218309123184427D3
:1028600037FD4095542F0E94D476BC01992777FDFF
:102870009095892FE60EF71E081F191F72E0159517
:102880000795F794E7947A95D1F780E090E8A0E077
:10289000B0E0E80EF91E0A1F1B1F20912E18309180
:1028A0002F1840E050E0C801B7010E94D4763B01E8
:1028B0004C016FE096948794779467946A95D1F76A
:1028C000A980BB24CC24DD246501BB24AA248A81F1
:1028D00090E0A0E0B0E0BA2FA92F982F8827A82A6F
:1028E000B92ACA2ADB2A8B8190E0A0E0B0E0A82AAE
:1028F000B92ACA2ADB2A0B8804C0D594C794B79496
:10290000A7940A94D2F720911E1830911F184427DB
:1029100037FD4095542FC201B1010E94D4767B014E
:102920008C013BE015950795F794E7943A95D1F71C
:1029300080911C1890911D18AA2797FDA095BA2F79
:1029400022E0880F991FAA1FBB1F2A95D1F7E80E16
:10295000F91E0A1F1B1F20912418309125184427A7
:1029600037FD4095542F6F89788D898D9A8D0E94FF
:10297000D476A7E19595879577956795AA95D1F730
:10298000E60EF71E081F191F0D8804C0EE0CFF1C71
:10299000001F111F0A94D2F722E030E040E050E01F
:1029A000E20EF31E041F151FF2E015950795F7942C
:1029B000E794FA95D1F7AE18BF08C00AD10AC6014C
:1029C000B5012E853F85488959890E94D47697FDA7
:1029D0000BC0660F771F881F991FA40193010E94E7
:1029E0001A7779018A010AC0A40193010E941A771B
:1029F00079018A01EE0CFF1C001F111F552717FDDE
:102A00005A95412F302F2F2DCA01B9010E94D4763B
:102A10002EED3BE040E050E00E94D4765B016C017B
:102A2000C801B70123E433EE4FEF5FEF0E94D47685
:102A3000BC01992777FD9095892F6153714F8F4F76
:102A40009F4F5601DD24B7FCD094CD2C6A0D7B1D21
:102A50008C1D9D1D24E095958795779567952A9502
:102A6000D1F76E0D7F1D801F911F2C813D814E81FE
:102A70005F81260F371F481F591F2C833D834E83CC
:102A80005F8338853F5F388748855A89451708F442
:102A900092CE552391F0252F30E040E050E06C813C
:102AA0007D818E819F810E941A7720933818309300
:102AB000391840933A1850933B188B8D8823C9F1ED
:102AC000609138187091391880913A1890913B189C
:102AD000611571058105910561F10E945C7420E822
:102AE00036EE45EC57E40E94F27321E03EED42E4FD
:102AF0005EE30E946F75562F472F382F292F60E015
:102B000070E080E89FE3DA01F9012B2F3A2F4F2F75
:102B10005E2F0E9489732BE43AE34DEB57E30E944A
:102B2000F27360933C1870933D1880933E18909315
:102B30003F186C960FB6F894DEBF0FBECDBFCF9195
:102B4000DF911F910F91FF90EF90DF90CF90BF909A
:102B5000AF909F908F907F906F905F904F903F903D
:102B60002F900895DF93CF9300D000D000D0CDB741
:102B7000DEB7FE01319686E0DF011D928A95E9F706
:102B80008091A617882399F486EA61E340E00E94C9
:102B9000061186EA6CE24AE00E94061181E0809309
:102BA000A6176CE77EE380E090E00E943D4986EA4C
:102BB0006DE248E00E9406116CE77EE380E090E061
:102BC0000E943D4986EA62E3AE014F5F5F4F26E017
:102BD0000E941E1186EA6DE247E00E9406119A816A
:102BE00080E0498150E0482B592B5093A117409326
:102BF000A0179C8180E02B8130E0282B392B30936B
:102C0000A3172093A2177E8160E08D8190E0862B30
:102C1000972B9093A5178093A4176DB77EB7685034
:102C200070400FB6F8947EBF0FBE6DBFEDB7FEB714
:102C3000319667EA72E0ADB7BEB712967C936E9399
:102C400011975383428335832483978386830E941D
:102C50009A7A6DB77EB7685F7F4F0FB6F8947EBFE4
:102C60000FBE6DBF26960FB6F894DEBF0FBECDBF68
:102C7000CF91DF9108950F931F93DF93CF9300D0EF
:102C800000D000D0CDB7DEB78E010F5F1F4F86E0BA
:102C9000D8011D928A95E9F78CE362E041E00E9439
:102CA00006118CE360E048E50E94061162E174E3DE
:102CB00080E090E00E943D498CE363E0A80126E0BB
:102CC0000E941E118CE362E043E00E94061199818C
:102CD00080E04A8150E0482B592B50937D17409358
:102CE0007C179B8180E02C8130E0282B392B30939E
:102CF0007F1720937E177D8160E08E8190E0862B88
:102D0000972B9093811780938017EDB7FEB7389774
:102D10000FB6F894FEBF0FBEEDBF319665EB72E0C3
:102D2000ADB7BEB712967C936E93119753834283CF
:102D300035832483978386830E949A7AEDB7FEB702
:102D400038960FB6F894FEBF0FBEEDBF26960FB6AD
:102D5000F894DEBF0FBECDBFCF91DF911F910F91D1
:102D60000895CF93DF93EC0188819981009731F02A
:102D70002AE08832920709F071C00BC087ED96E017
:102D800060E870E00E94804088E29AE0998388833E
:102D900069C087ED96E00E94AB40009709F462C0DD
:102DA0008091CE069091CF0694FF3FC08091451C44
:102DB00082FF3BC083E061E048E021E00E94F11225
:102DC0008DB79EB70A970FB6F8949EBF0FBE8DBF02
:102DD000EDB7FEB7319682EA91E0ADB7BEB7129675
:102DE0009C938E9311978091381890913918A091E7
:102DF0003A18B0913B1882839383A483B583809162
:102E00003C1890913D18A0913E18B0913F188683D0
:102E10009783A087B1870E94AC7A8DB79EB70A9638
:102E20000FB6F8949EBF0FBE8DBF8091CE069091D5
:102E3000CF0695FF06C08091451C83FF02C00E940B
:102E4000B2158091CE069091CF0696FF97CF8091D4
:102E5000451C84FF93CF0E943B1690CF19821882A5
:102E600083E001C081E0DF91CF910895EF92FF925E
:102E70000F931F93CF93DF93729A8091B90483FDD0
:102E800006C0C0E5D0E00E94760A2197E1F78EE403
:102E90000E9450498823B1F080914B2090914C20A2
:102EA000A0914D20B0914E200196A11DB11D80939F
:102EB0004B2090934C20A0934D20B0934E2021E0C6
:102EC00030E087C0C0E5D0E00E94760A2197E1F7A4
:102ED0008FE40E9450490E94CF49982F9295969571
:102EE000969593709130A9F420914F203091502005
:102EF00040915120509152202F5F3F4F4F4F5F4FD5
:102F000020934F20309350204093512050935220D3
:102F100016C09230A0F0209153203091542040915F
:102F20005520509156202F5F3F4F4F4F5F4F2093BA
:102F300053203093542040935520509356206FE3F4
:102F4000E62EE8220E94CF49F82E0E94CF49082F92
:102F50000E94D949182F0E94B6498091B90483FF75
:102F600072987E2D60E06F0D711D80E090E00E94F0
:102F70005A7420E134E048EC5BE30E940C756093E6
:102F80004118709342188093431890934418702FFF
:102F900060E0610F711D769567957695679580E085
:102FA00090E00E945A7424EA3CEF44E25CE30E9401
:102FB0000C7520E030E040E252E40E948973609397
:102FC000BD247093BE248093BF249093C02420E03E
:102FD00030E0C901DF91CF911F910F91FF90EF90E9
:102FE00008957298729A8EE40E94504980EA0E9475
:102FF000BE4980E00E94BE4980E00E94BE498FE445
:103000000E9450490E94CF4982958695869583708B
:103010008130A9F420914F203091502040915120CF
:10302000509152202F5F3F4F4F4F5F4F20934F20C3
:1030300030935020409351205093522016C082303C
:10304000A0F0209153203091542040915520509170
:1030500056202F5F3F4F4F4F5F4F209353203093A9
:103060005420409355205093562000D000D0EDB707
:10307000FEB7319623EC32E0ADB7BEB712963C9363
:103080002E931197828313820E949A7A0F900F9049
:103090000F900F908EE40E94504980E80E94BE4934
:1030A00080E00E94BE4980E00E94BE490E94B6496D
:1030B00080E090E0089500D081E99CE0ADB7BEB714
:1030C00012969C938E9311970E94AC7A20919C0447
:1030D0000F900F902223A9F000D000D0EDB7FEB7DB
:1030E00031968EE89CE0ADB7BEB712969C938E9356
:1030F0001197228313820E94AC7A0F900F900F9049
:103100000F90089500D089E69CE0EDB7FEB792835A
:1031100081830E94AC7A81E49CE0EDB7FEB7928394
:1031200081830E94AC7A8AE19CE0EDB7FEB792837E
:1031300081830E94AC7A80EF9BE0EDB7FEB792836B
:1031400081830E94AC7A85EB9BE0EDB7FEB792835A
:1031500081830E94AC7A83E89BE0EDB7FEB792834F
:1031600081830E94AC7A8DE59BE0EDB7FEB7928338
:1031700081830E94AC7A8DE29BE0EDB7FEB792832B
:1031800081830E94AC7A84EF9AE0EDB7FEB7928318
:1031900081830E94AC7A88EC9AE0EDB7FEB7928307
:1031A00081830E94AC7A8FE99AE0EDB7FEB79283F3
:1031B00081830E94AC7A84E79AE0EDB7FEB79283F0
:1031C00081830E94AC7A85E49AE0EDB7FEB79283E2
:1031D00081830E94AC7A83E19AE0EDB7FEB79283D7
:1031E00081830E94AC7A82EE99E0EDB7FEB79283BC
:1031F00081830E94AC7A8EEA99E0EDB7FEB79283A4
:1032000081830E94AC7A8EE799E0EDB7FEB7928396
:1032100081830E94AC7A82E599E0EDB7FEB7928394
:1032200081830E94AC7A83E299E0EDB7FEB7928386
:1032300081830E94AC7A8CEE98E0EDB7FEB7928362
:1032400081830E94AC7A83EB98E0EDB7FEB792835E
:1032500081830E94AC7A8AE898E0EDB7FEB792834A
:1032600081830E94AC7A8BE498E0EDB7FEB792833D
:1032700081830E94AC7A8CE198E0EDB7FEB792832F
:1032800081830E94AC7A8DEE97E0EDB7FEB7928312
:1032900081830E94AC7A86EC97E0EDB7FEB792830B
:1032A00081830E94AC7A80E997E0EDB7FEB7928304
:1032B00081830E94AC7A87E697E0EDB7FEB79283F0
:1032C00081830E94AC7A8CE397E0EDB7FEB79283DE
:1032D00081830E94AC7A0F900F90089583ED92E065
:1032E0000E94D37A08952F923F924F925F926F92ED
:1032F0007F928F929F92AF92BF92CF92DF92EF9286
:10330000FF920F931F93CF93DF93609147207091AB
:1033100048208091492090914A20A0904720B09069
:103320004820C0904920D0904A206090472070905B
:1033300048208090492090904A202090472030904B
:1033400048204090492050904A202DB73EB72A503F
:1033500030400FB6F8943EBF0FBE2DBFCDB7DEB7DD
:1033600021962CE137E0EDB7FEB732832183A0E848
:10337000EA2EA1E5FA2EA1E00A2F112DA80197014E
:103380000E941A773B832A83C601B501A8019701E1
:103390000E941A77F0E1EF2EFEE0FF2E012D112D95
:1033A000A80197010E941A77332727FD30953D83A6
:1033B0002C83C401B301A80197010E941A77ECE3A2
:1033C000EE2EF12C012D112DA80197010E941A77E4
:1033D000332727FD30953F832E83C201B101A80119
:1033E00097010E941A77772767FD7095798768871C
:1033F0000E94AC7A2DB73EB7265F3F4F0FB6F894C8
:103400003EBF0FBE2DBFDF91CF911F910F91FF9057
:10341000EF90DF90CF90BF90AF909F908F907F9074
:103420006F905F904F903F902F900895E2E8FDE2FB
:103430008081918122E482349207B9F000D000D0DB
:103440008EEF96E0ADB7BEB712969C938E93119710
:10345000E258FD421496FC93EE9313970E94AC7AC7
:103460000F900F900F900F9008953A96B1E4E53FBA
:10347000FB07F0F20895EF92FF920F931F93CF9303
:10348000DF930E94600B00D000D000D027EF36E021
:10349000ADB7BEB712963C932E931197EDB7FEB71A
:1034A00063837483858396830E94AC7A8DB79EB7BD
:1034B00006960FB6F8949EBF0FBE8DBF81E00E94A6
:1034C000120B2091940430919504409196045091F0
:1034D00097040E940C757B018C0182E00E94120B04
:1034E0009B01AC01ADB7BEB71A970FB6F894BEBF3B
:1034F0000FBEADBFCDB7DEB72196EBEEF6E012966C
:10350000FC93EE9311978E2D9F2DA02FB12F8A83C0
:103510009B83AC83BD83CA01B9012091980430918B
:10352000990440919A0450919B040E940C756E83FB
:103530007F83888799870E94AC7AEDB7FEB73A9669
:103540000FB6F894FEBF0FBEEDBF0E94730CDF9163
:10355000CF911F910F91FF90EF9008950F931F93BC
:10356000CF93DF93882389F081EB94E26FEF70E0D3
:1035700049E050E00E94157A81EB94E267E170E047
:1035800049E050E00E94FC7B1CC0C1EBD4E206EE97
:1035900016E0899100D000D0EDB7FEB73196ADB7F7
:1035A000BEB712961C930E931197828313820E94CA
:1035B000AC7A0F900F900F900F90B4E2C93BDB07ED
:1035C00041F70E94730CDF91CF911F910F910895E5
:1035D000EF92FF920F931F936091A1047091A20448
:1035E00080E090E00E94077A6EEE72E00E941C7A02
:1035F000009709F098C086E294E1A0E0B0E08093E3
:10360000B3049093B404A093B504B093B60483EBD1
:1036100094E06EE070E042E050E00E94FC7B8CE3BE
:1036200090E09093B8048093B70487EB94E062E154
:1036300070E042E050E00E94FC7B8AE090E09093D2
:10364000BA048093B90489EB94E064E170E042E04D
:1036500050E00E94FC7B1092CF061092CE068EECBA
:1036600096E060E070E042E050E00E94FC7B0F2EAC
:10367000F2E2EF2EFFEFFF2EFCEC0F2FFBE31F2FEC
:10368000F02DE0929404F092950400939604109328
:10369000970484E994E066E070E044E050E00E9422
:1036A000FC7BE0929804F092990400939A041093A2
:1036B0009B0488E994E06AE070E044E050E00E94F6
:1036C000FC7B8DEE97E4AAE8BCE380939004909392
:1036D0009104A0939204B093930480E994E062E093
:1036E00070E044E050E00E94FC7B1092D30683ED32
:1036F00096E066E170E041E050E00E94FC7B82E9E8
:1037000097E12AE0FC0111922A95E9F760E270E066
:103710004AE050E00E94FC7B81E00E94AE1A80E00B
:1037200090E00E94F60D1F910F91FF90EF90089589
:10373000882309F436C18091B30480FF0BC000D008
:1037400081EE96E0EDB7FEB7928381830E94AC7A5A
:103750000F900F908091B30481FF0BC000D08DEDCE
:1037600096E0EDB7FEB7928381830E94AC7A0F900A
:103770000F908091B30482FF0BC000D08AED96E0D9
:10378000EDB7FEB7928381830E94AC7A0F900F90C1
:103790008091B30483FF0BC000D086ED96E0EDB7B7
:1037A000FEB7928381830E94AC7A0F900F90809134
:1037B000B30484FF0BC000D08FEC96E0EDB7FEB7EA
:1037C000928381830E94AC7A0F900F908091B30412
:1037D00085FF0BC000D088EC96E0EDB7FEB7928372
:1037E00081830E94AC7A0F900F908091B30486FF82
:1037F0000BC000D084EC96E0EDB7FEB792838183D6
:103800000E94AC7A0F900F908091B30487FF0BC099
:1038100000D08EEB96E0EDB7FEB7928381830E94D5
:10382000AC7A0F900F908091B3049091B404A09162
:10383000B504B091B60490FF0BC000D08AEB96E0BF
:10384000EDB7FEB7928381830E94AC7A0F900F9000
:103850008091B3049091B404A091B504B091B604E2
:1038600091FF0BC000D084EB96E0EDB7FEB79283DA
:1038700081830E94AC7A0F900F908091B304909155
:10388000B404A091B504B091B60492FF0BC000D06F
:103890008CEA96E0EDB7FEB7928381830E94AC7A02
:1038A0000F900F908091B3049091B404A091B5044F
:1038B000B091B60493FF0BC000D088EA96E0EDB754
:1038C000FEB7928381830E94AC7A0F900F90809113
:1038D000B3049091B404A091B504B091B60494FFE0
:1038E0000BC000D082EA96E0EDB7FEB792838183E9
:1038F0000E94AC7A0F900F908091B3049091B40421
:10390000A091B504B091B60495FF0BC000D08EE92C
:1039100096E0EDB7FEB7928381830E94AC7A0F9058
:103920000F908091B3049091B404A091B504B0912C
:10393000B60496FF0BC000D08AE996E0EDB7FEB75B
:10394000928381830E94AC7A0F900F908091B30490
:103950009091B404A091B504B091B60497FF0BC048
:1039600000D087E996E0EDB7FEB7928381830E948D
:10397000AC7A0F900F908091B3049091B404A09111
:10398000B504B091B604A0FFF7C100D083E996E07A
:10399000EDB7FEB7928381830E94AC7A0F900F90AF
:1039A000EBC100D000D000D088E896E0EDB7FEB7BC
:1039B0009283818381E090E0A0E0B0E083839483F0
:1039C000A583B6830E94AC7A8DB79EB706960FB6D4
:1039D000F8949EBF0FBE8DBF0E94730C00D000D024
:1039E00000D08EE796E0EDB7FEB79283818382E048
:1039F00090E0A0E0B0E083839483A583B6830E9427
:103A0000AC7A8DB79EB706960FB6F8949EBF0FBEE0
:103A10008DBF0E94730C00D000D000D085E796E0E7
:103A2000EDB7FEB79283818384E090E0A0E0B0E040
:103A300083839483A583B6830E94AC7A8DB79EB7A7
:103A400006960FB6F8949EBF0FBE8DBF0E94730CF2
:103A500000D000D000D08BE696E0EDB7FEB79283A1
:103A6000818388E090E0A0E0B0E083839483A58325
:103A7000B6830E94AC7A8DB79EB706960FB6F894BF
:103A80009EBF0FBE8DBF0E94730C00D000D000D02F
:103A90008EE596E0EDB7FEB79283818380E190E0FA
:103AA000A0E0B0E083839483A583B6830E94AC7AC0
:103AB0008DB79EB706960FB6F8949EBF0FBE8DBF0A
:103AC0000E94730C00D000D000D081E596E0EDB7E5
:103AD000FEB79283818380E290E0A0E0B0E0838330
:103AE0009483A583B6830E94AC7A8DB79EB7069661
:103AF0000FB6F8949EBF0FBE8DBF0E94730C00D00E
:103B000000D000D087E496E0EDB7FEB792838183C2
:103B100080E490E0A0E0B0E083839483A583B68343
:103B20000E94AC7A8DB79EB706960FB6F8949EBFEA
:103B30000FBE8DBF0E94730C00D000D000D08BE36D
:103B400096E0EDB7FEB79283818380E890E0A0E035
:103B5000B0E083839483A583B6830E94AC7A8DB74B
:103B60009EB706960FB6F8949EBF0FBE8DBF0E94FB
:103B7000730C00D000D000D081E396E0EDB7FEB723
:103B80009283818380E091E0A0E0B0E0838394831E
:103B9000A583B6830E94AC7A8DB79EB706960FB602
:103BA000F8949EBF0FBE8DBF0E94730C00D000D052
:103BB00000D085E296E0EDB7FEB79283818380E086
:103BC00092E0A0E0B0E083839483A583B6830E9453
:103BD000AC7A8DB79EB706960FB6F8949EBF0FBE0F
:103BE0008DBF0E94730C00D000D000D087E196E01A
:103BF000EDB7FEB79283818380E094E0A0E0B0E06F
:103C000083839483A583B6830E94AC7A8DB79EB7D5
:103C100006960FB6F8949EBF0FBE8DBF0E94730C20
:103C200000D000D000D08DE096E0EDB7FEB79283D3
:103C3000818380E098E0A0E0B0E083839483A58353
:103C4000B6830E94AC7A8DB79EB706960FB6F894ED
:103C50009EBF0FBE8DBF0E94730C00D000D000D05D
:103C600081E096E0EDB7FEB79283818380E090E13A
:103C7000A0E0B0E083839483A583B6830E94AC7AEE
:103C80008DB79EB706960FB6F8949EBF0FBE8DBF38
:103C90000E94730C00D000D000D087EF95E0EDB704
:103CA000FEB79283818380E090E2A0E0B0E083835E
:103CB0009483A583B6830E94AC7A8DB79EB706968F
:103CC0000FB6F8949EBF0FBE8DBF0E94730C00D03C
:103CD00000D000D08DEE95E0EDB7FEB792838183E2
:103CE00080E090E4A0E0B0E083839483A583B68372
:103CF0000E94AC7A8DB79EB706960FB6F8949EBF19
:103D00000FBE8DBF0E94730C00D000D000D083EE98
:103D100095E0EDB7FEB79283818380E090E8A0E064
:103D2000B0E083839483A583B6830E94AC7A8DB779
:103D30009EB706960FB6F8949EBF0FBE8DBF0E9429
:103D4000730C00D000D000D088ED95E0EDB7FEB741
:103D50009283818380E090E0A1E0B0E0838394834C
:103D6000A583B6830E94AC7A8DB79EB706960FB630
:103D7000F8949EBF0FBE8DBF0E94730C08952F92C2
:103D80003F924F925F926F927F928F929F92AF92EB
:103D9000BF92CF92DF92EF92FF920F931F93DF9328
:103DA000CF9300D0CDB7DEB79A838983DC018D91A4
:103DB0009C911197009711F00C94B9316091A10476
:103DC0007091A2048CE590E20E94077A8CE590E263
:103DD00060E470E00E94347A009759F460917C2D81
:103DE00070917D2D8AE090E00E946E7A81E00C94C3
:103DF000BF318130910549F420905C203324442464
:103E00005524662477244301BFC18230910599F47B
:103E100030915C2020915D20932F80E0820F911DD6
:103E20001C01892F880F880B482E582E682E782E5B
:103E3000882E982EA9C18330910509F09CC020914D
:103E40005C20A0905D2080905E2030E040E050E05B
:103E500060E070E080E090E000E10E94266FF22ECA
:103E6000132FE42ED52EC62EB72E282E992E2A2DAE
:103E700030E040E050E060E070E080E090E008E09A
:103E80000E94266F2F0DB1E02F1508F0B0E0310F22
:103E9000E1E0311708F0E0E0B30FF1E0B31708F00C
:103EA000F0E0EF2B4E0D31E04E1508F030E0E40F5E
:103EB000F1E0E41708F0F0E03F2B5D0D41E05D1507
:103EC00008F040E0A32FA50F31E0A51708F030E07F
:103ED000432B6C0D31E06C1508F030E0F42FF60F39
:103EE00041E0F61708F040E0342B7B0D41E07B15F4
:103EF00008F040E0532F570F31E0571708F030E03B
:103F0000432B820D31E0821508F030E0480F61E06C
:103F1000481708F060E0362B990D930F022F080D1B
:103F200011E0021708F010E01B0F81E01B1708F0EA
:103F300080E0B82FBE0F71E0BE1708F070E07A0F76
:103F400061E07A1708F060E06F0F31E06F1708F05A
:103F500030E0350F21E0351708F020E0240F81E034
:103F6000241708F080E018014B2E572E662E732E72
:103F7000822E982EFEC08430910509F0FCC020915D
:103F80005C20A0905D2070905E2080905F2030E0EB
:103F900040E050E060E070E080E090E008E10E94E6
:103FA000266FF22E132FE42ED52EC62EB72E282ED6
:103FB000992E2A2D30E040E050E060E070E080E093
:103FC00090E000E10E94266F2F0DF1E02F1508F020
:103FD000F0E0310FE1E0311708F0E0E0F30FA1E08D
:103FE000F31708F0A0E0EA2B4E0D31E04E1508F073
:103FF00030E0E40FA1E0E41708F0A0E03A2B5D0DFB
:1040000041E05D1508F040E0B32FB50F31E0B51782
:1040100008F030E0432B6C0D31E06C1508F030E017
:10402000A42FA60F41E0A61708F040E0342B7B0D2B
:1040300041E07B1508F040E0532F570F31E0571750
:1040400008F030E0432B820D31E0821508F030E0BB
:10405000480F61E0481708F060E0362B990E930E88
:10406000122F180D81E0121708F080E0282E2F0E75
:1040700081E02F1608F080E0F82EFE0E81E0FE169B
:1040800008F080E0E82EEB0E81E0EB1608F080E00F
:10409000D82EDA0E81E0DA1608F080E0C82EC50EC0
:1040A00081E0C51608F080E0B82EB40E81E0B416A9
:1040B00008F080E0980E272D30E040E050E060E00E
:1040C00070E080E090E008E00E94266F210FE1E0C0
:1040D000211708F0E0E0320DF1E0321508F0F0E0D1
:1040E000E30FA1E0E31708F0A0E0FA2B4F0D31E059
:1040F0004F1508F030E0F40FA1E0F41708F0A0E04D
:104100003A2B5E0D41E05E1508F040E0A32FA50FAD
:1041100031E0A51708F030E0432B6D0D31E06D154F
:1041200008F030E0542F560F41E0561708F040E0F9
:10413000342B7C0D41E07C1508F040E0632F670FC5
:1041400031E0671708F030E0432B8B0D31E08B1521
:1041500008F030E0480F71E0481708F070E0372BA6
:10416000990D222E3E2E4F2E5A2E652E762E842EFF
:10417000932E990E09C01AE0212E3324442455248D
:1041800066247724882499240E94730CB22DB336B8
:1041900089F4E32DE23371F4F42DF93659F4552006
:1041A00049F4662039F4772029F4882019F49920FD
:1041B00009F44EC59101A201B301C401B3E6AB2ECF
:1041C000A2E3BA2EF9E6CF2EDD24EE24FF2400E090
:1041D00010E00E94976F823008F073C2822D8536FE
:1041E00089F4932D923771F4442061F4552051F4F1
:1041F000662041F4772031F4882021F4992011F4CD
:104200000C94402D9101A201B301C401E5E6AE2E4C
:1042100002E7B02ECC24DD24EE24FF2400E010E0E1
:104220000E94976F823008F008C1A22DA53681F454
:10423000B32DB43669F4442059F4552049F466206E
:1042400039F4772029F4882019F4992009F4CDC68F
:104250009101A201B301C40115E6A12EB4E6BB2E63
:10426000CC24DD24EE24FF2400E010E00E94976FB0
:10427000823008F062C0E22DE53779F4332069F42A
:10428000442059F4552049F4662039F4772029F464
:10429000882019F4992009F4EAC79101A201B30119
:1042A000C401A5E7AA2EBB24CC24DD24EE24FF24E0
:1042B00000E010E00E94976F823010F5F22DF83682
:1042C00011F00C94B731332011F00C94B731442025
:1042D00011F00C94B731552011F00C94B7316620D1
:1042E00011F00C94B731772011F00C94B73188207D
:1042F00011F00C94B731992011F00C94B73192C79A
:10430000822D863779F4332069F4442059F45520FE
:1043100049F4662039F4772029F4882019F499208B
:1043200009F4BEC7922D943611F00C94B731A32D29
:10433000A13611F00C94B7317BC0B22DB73789F498
:10434000E32DEF3671F4442061F4552051F46620DA
:1043500041F4772031F4882021F4992011F40C9451
:10436000D62B9101A201B301C401F7E7AF2EEFE60E
:10437000BE2ECC24DD24EE24FF2400E010E00E94B9
:10438000976F8230B8F5F22DF43681F4832D89369B
:1043900069F4442059F4552049F4662039F4772013
:1043A00029F4882019F4992009F440C7922D9536F4
:1043B00011F00C94B731A32DAE3611F00C94B73137
:1043C000442011F00C94B731552011F00C94B73102
:1043D000662011F00C94B731772011F00C94B731AE
:1043E000882011F00C94B731992011F00C94B7315A
:1043F0000C942A2CB22DB13389F4E32DE03771F4FB
:10440000442061F4552051F4662041F4772031F4C2
:10441000882021F4992011F40C94BB2CF22DF33355
:1044200011F00C94B731832D813711F00C94B73112
:10443000442011F00C94B73195C0922D983789F42F
:10444000A32DA43671F4B42DB13659F4552049F496
:10445000662039F4772029F4882019F4992009F48A
:10446000F3C39101A201B301C40108E7A02E14E631
:10447000B12EB1E6CB2EDD24EE24FF2400E010E0C7
:104480000E94976F823008F083C0E22DE33789F4F1
:10449000F32DF23771F4442061F4552051F4662075
:1044A00041F4772031F4882021F4992011F40C9400
:1044B0000C2E9101A201B301C401A3E7AA2EF2E7D9
:1044C000BF2ECC24DD24EE24FF2400E010E00E9467
:1044D000976F823020F5822D893611F00C94B73118
:1044E000932D923711F00C94B731442011F00C94B5
:1044F000B731552011F00C94B731662011F00C94AF
:10450000B731772011F00C94B731882011F00C945A
:10451000B731992011F00C94B7310C94B92DA22D1C
:10452000A33789F4B32DB33771F4442061F45520D7
:1045300051F4662041F4772031F4882021F4992049
:1045400011F40C941B2EE22DE33611F00C94B731CC
:10455000F32DF43611F00C94B731842D813611F01F
:104560000C94B731552011F00C94B731662011F03E
:104570000C94B731772011F00C94B731882011F0EA
:104580000C94B731992011F00C94B7310C942F3062
:10459000922D923791F4A32DA23779F4B42DB5362C
:1045A00061F4552051F4662041F4772031F48820DD
:1045B00021F4992011F40C94F92A9101A201B3017C
:1045C000C401E2E7AE2E02E7B02E15E6C12EDD24CF
:1045D000EE24FF2400E010E00E94976F8230C0F5C7
:1045E000E22DE33789F4F32DF53671F4842D81360D
:1045F00059F4552049F4662039F4772029F48820AD
:1046000019F4992009F45CC6922D923611F00C949D
:10461000B731A32DA53611F00C94B731B42DB436B3
:1046200011F00C94B731552011F00C94B73166207D
:1046300011F00C94B731772011F00C94B731882029
:1046400011F00C94B731992011F00C94B731CDC40E
:10465000E22DE33689F4F32DFD3671F4842D88368E
:1046600059F4552049F4662039F4772029F488203C
:1046700019F4992009F4F0C2922D9D3611F00C9492
:10468000B731A32DA53711F00C94B731B42DB8363E
:1046900011F00C94B731552011F00C94B73166200D
:1046A00011F00C94B731772011F00C94B7318820B9
:1046B00011F00C94B731992011F00C94B7310C948F
:1046C0003E30E22DE03791F4F32DFC3679F4842D61
:1046D000853661F4952D983649F4662039F47720B3
:1046E00029F4882019F4992009F49CC59101A201AC
:1046F000B301C401B0E7AB2EACE6BA2EF5E6CF2E7F
:10470000E8E6DE2EEE24FF2400E010E00E94976F22
:10471000823008F047C1A22DA13389F4B32DB13303
:1047200071F4E42DE13759F4552049F4662039F449
:10473000772029F4882019F4992009F4BDC7910144
:10474000A201B301C40101E3A02E11E3B12EB1E730
:10475000CB2EDD24EE24FF2400E010E00E94976FB2
:10476000823008F083C0F22DF73689F4832D8F361E
:1047700071F4942D9C3659F4552049F4662039F48F
:10478000772029F4882019F4992009F4DFC69101D3
:10479000A201B301C401A7E6AA2EFFE6BF2EECE6F4
:1047A000CE2EDD24EE24FF2400E010E00E94976F5F
:1047B000823020F5A22DA43611F00C94B731B32D20
:1047C000B33611F00C94B731E42DEC3611F00C94A3
:1047D000B731552011F00C94B731662011F00C94CC
:1047E000B731772011F00C94B731882011F00C9478
:1047F000B731992011F00C94B731A5C6F22DF537D9
:1048000089F4832D833671F4942D9D3659F4552007
:1048100049F4662039F4772029F4882019F4992086
:1048200009F44AC7A22DA03311F00C94B731B32D6F
:10483000B13311F00C94B731E42DE13711F00C9441
:10484000B731552011F00C94B731662011F00C945B
:10485000B731772011F00C94B731882011F00C9407
:10486000B731992011F00C94B731C3C6F22DF4374B
:1048700091F4832D843679F4942D973761F4552083
:1048800051F4662041F4772031F4882021F49920F6
:1048900011F40C944A319101A201B301C40104E75F
:1048A000A02E14E6B12EB7E7CB2EDD24EE24FF2494
:1048B00000E010E00E94976F8230D0F5A22DA03763
:1048C00091F4B32DB53679F4E42DE23761F4552037
:1048D00051F4662041F4772031F4882021F49920A6
:1048E00011F40C94402DF22DF43711F00C94B731E3
:1048F000832D883711F00C94B731942D943711F033
:104900000C94B731552011F00C94B731662011F09A
:104910000C94B731772011F00C94B731882011F046
:104920000C94B731992011F00C94B7310C941F31CD
:10493000A22DA43791F4B32DBF3679F4E42DEF36D0
:1049400061F4F52DF23649F4662039F4772029F424
:10495000882019F4992009F40CC5822D893611F0AC
:104960000C94B731932D9C3611F00C94B731A42DD3
:10497000A13611F00C94B731B52DB33611F00C946B
:10498000B731662011F00C94B731772011F00C94F8
:10499000B731882011F00C94B731992011F00C94A4
:1049A000B73186C1E22DE33799F4F32DF23781F464
:1049B000842D873769F4952D903751F4662041F4A2
:1049C000772031F4882021F4992011F40C94082DDB
:1049D0009101A201B301C401A3E7AA2EF2E7BF2E01
:1049E000E7E7CE2E00E7D02EEE24FF2400E010E013
:1049F0000E94976F823008F089C0A22DA03791F4F1
:104A0000B32DBD3679F4E42DE53761F4F52DF83694
:104A100049F4662039F4772029F4882019F4992084
:104A200009F4EAC69101A201B301C40110E7A12E65
:104A3000BDE6BB2EA5E7CA2EF8E6DF2EEE24FF2446
:104A400000E010E00E94976F823028F5822D8136B9
:104A500011F00C94B731932D9D3611F00C94B731B1
:104A6000A42DA53711F00C94B731B52DB83611F03F
:104A70000C94B731662011F00C94B731772011F007
:104A80000C94B731882011F00C94B731992011F0B3
:104A90000C94B731A0C6E22DE33799F4F32DF53627
:104AA00081F4842D823769F4952D903751F4662076
:104AB00041F4772031F4882021F4992011F40C94EA
:104AC0008830A22DA13311F00C94B731B32DB23739
:104AD00011F00C94B731E42DE73711F00C94B73195
:104AE000F52DF03711F00C94B731662011F00C94CD
:104AF000B731772011F00C94B731882011F00C9465
:104B0000B731992011F00C94B731AAC0822D8737A4
:104B100091F4932D903779F4A42DA83761F4B52D35
:104B2000B43749F4662039F4772029F4882019F441
:104B3000992009F4F5C39101A201B301C401E7E78B
:104B4000AE2E00E7B02E18E7C12EB4E7DB2EEE2420
:104B5000FF2400E010E00E94976F8230D0F5E22D34
:104B6000E43791F4F32DF33779F4842D853661F42D
:104B7000952D923749F4662039F4772029F488205E
:104B800019F4992009F4F4C6A22DA43711F00C945D
:104B9000B731B32DB33711F00C94B731E42DE536AE
:104BA00011F00C94B731F52DF43711F00C94B731A6
:104BB000662011F00C94B731772011F00C94B731C6
:104BC000882011F00C94B731992011F00C94B73172
:104BD000D4C3822D823791F4932D973679F4A42D86
:104BE000A03761F4B52DB53749F4662039F4772044
:104BF00029F4882019F4992009F476C4E22DEC36C2
:104C000011F00C94B731F32DF13611F00C94B7314B
:104C1000842D843711F00C94B731952D983711F00D
:104C20000C94B731662011F00C94B731772011F055
:104C30000C94B731882011F00C94B731992011F001
:104C40000C94B7310C94E3300E94B2150C94B93136
:104C50000E9426100C94B9310E943B160C94B93175
:104C60006091A1047091A20480E090E00E94077A14
:104C70008C0165EF72E00E941C7A009719F4779816
:104C80000C94B931C80168EF72E00E941C7A009759
:104C900019F4779A0C94B931779903C085EF92E0B3
:104CA00002C088EF92E000D000D02DE235E011C4C0
:104CB0006091A1047091A20480E090E00E94077AC4
:104CC0008C016FE073E00E941C7A009709F052C0DB
:104CD0006091A1047091A20480E090E00E94077AA4
:104CE0008C01009711F40C94B93162E173E00E94D9
:104CF0001C7A009729F482E29FEFACECBBE30BC077
:104D0000C80168E173E00E941C7A009769F482E2AE
:104D10009FEFACECBAE38093940490939504A09336
:104D20009604B09397041DC0C8010E94FA787B01D5
:104D30008C0120E030E0A9010E94EE738823B1F0DD
:104D400081E00E94120B9B01AC01C801B7010E94D7
:104D5000F2736093940470939504809396049093F7
:104D6000970484E994E066E070E0BEC000D08DE670
:104D700095E08CC0C8016DE173E00E941C7A009739
:104D800009F052C06091A1047091A20480E090E00B
:104D90000E94077A8C01009711F40C94B93162E1FA
:104DA00073E00E941C7A009729F482E29FEFACEC3A
:104DB000BBE30BC0C80168E173E00E941C7A009756
:104DC00069F482E29FEFACECBAE38093980490938D
:104DD0009904A0939A04B0939B041DC0C8010E943B
:104DE000FA787B018C0120E030E0A9010E94EE738B
:104DF0008823B1F082E00E94120B9B01AC01C80134
:104E0000B7010E94F27360939804709399048093A1
:104E10009A0490939B0488E994E06AE070E064C08F
:104E200000D080E695E067C0C80160E273E00E94B0
:104E30001C7A009709F06BC06091A1047091A204E4
:104E400080E090E00E94077A8C01009711F40C94A6
:104E5000B93162E173E00E941C7A009769F48DEE2B
:104E600097E4AAE8BCE38093900490939104A09304
:104E70009204B093930434C0C80168E173E00E94C7
:104E80001C7A009741F400D081E595E0EDB7FEB7BC
:104E90009283818336C0C8010E94FA781B012C01DD
:104EA00020E030E0A9010E94EE73882309F180E040
:104EB0000E94120B7B018C01C201B10121EE3AE785
:104EC00044E95EE30E948973A80197010E94F2738E
:104ED0006093900470939104809392049093930450
:104EE00080E994E062E070E044E050E00C948D31A1
:104EF00000D084E495E0ADB7BEB712969C938E9334
:104F000011970E94AC7A0F900F900C94B9310E94C7
:104F1000600B00D000D000D02DE335E0EDB7FEB738
:104F200032832183ADB7BEB713966D937D938D9376
:104F30009C9316970E94AC7AEDB7FEB736960FB6E3
:104F4000F894FEBF0FBEEDBF81E00E94120B2091CE
:104F500094043091950440919604509197040E94D6
:104F60000C757B018C0182E00E94120B9B01AC014D
:104F70008DB79EB70A970FB6F8949EBF0FBE8DBF30
:104F8000CDB6DEB60894C11CD11C81E395E0ADB767
:104F9000BEB712969C938E9311978E2D9F2DA02FA6
:104FA000B12FF60182839383A483B583CA01B9012B
:104FB000209198043091990440919A0450919B0457
:104FC0000E940C75D60116966D937D938D939C93DC
:104FD00019970E94AC7AEDB7FEB73A960FB6F894DF
:104FE000FEBF0FBEEDBF0C941C316091A104709107
:104FF000A20480E090E00E94077A009761F160E0EF
:1050000070E040E150E00E94EC772091CE063091B4
:10501000CF062617370799F17093CF066093CE0617
:105020008EEC96E060E070E042E050E00E94FC7B95
:105030008091CE069091CF0600D000D02DE135E0D2
:10504000ADB7BEB712963C932E93119714969C93CE
:105050008E9313970EC08091CE069091CF0600D00C
:1050600000D029E035E0EDB7FEB732832183948389
:1050700083830E94AC7A0F900F900F900F900E9444
:10508000730C00D000D08CEF94E0ADB7BEB7129691
:105090009C938E93119781E090E014969C938E934D
:1050A00013970E94AC7A81EF94E0EDB7FEB792833C
:1050B000818382E090E0948383830E94AC7A86EEC1
:1050C00094E0ADB7BEB712969C938E93119784E08F
:1050D00090E014969C938E9313970E94AC7A89ED7E
:1050E00094E0EDB7FEB79283818388E090E09483EB
:1050F00083830E94AC7A8EEC94E0ADB7BEB7129673
:105100009C938E93119780E190E014969C938E93DC
:1051100013970E94AC7A82EC94E0EDB7FEB79283CD
:10512000818380E290E0948383830E94AC7A84EB55
:1051300094E0ADB7BEB712969C938E93119780E41E
:1051400090E014969C938E9313970E94AC7A86EA13
:1051500094E0EDB7FEB79283818380E890E094837A
:1051600083830E94AC7A87E994E0ADB7BEB712960C
:105170009C938E93119780E091E014969C938E936C
:1051800013970E94AC7A88E894E0EDB7FEB792835B
:10519000818380E092E0948383830E94AC7A8CE7E1
:1051A00094E0ADB7BEB712969C938E93119780E0B2
:1051B00094E014969C938E9313970E94AC7A8EE69B
:1051C00094E0EDB7FEB79283818380E098E094830A
:1051D00083830E94AC7A81E694E0ADB7BEB71296A5
:1051E0009C938E93119780E090E114969C938E93FC
:1051F00013970E94AC7A83E594E0EDB7FEB79283F3
:10520000818380E090E2948383830E94AC7A83E47C
:1052100094E0ADB7BEB712969C938E93119780E041
:1052200090E45DC10E9482180C94B9316091A10490
:105230007091A20480E090E00E94077A62E173E03E
:105240000E941C7A009711F481E001C080E00E9466
:10525000AE1A20919C04222311F40C94B93100D091
:1052600000D0EDB7FEB7319680E494E00FC00E9405
:10527000731920919C04222311F40C94B93100D0AD
:1052800000D0EDB7FEB731968DE394E0ADB7BEB771
:1052900012969C938E931197228313820C94B031B3
:1052A0000E946E1920919C04222311F40C94B931B0
:1052B00000D000D0EDB7FEB731968AE394E0E6CF98
:1052C0006091A1047091A20480E090E00E94077AAE
:1052D0008C0165EF72E00E941C7A009739F480918E
:1052E000B9049091BA0484600C948331C80168EFCA
:1052F00072E00E941C7A4091B9045091BA04009760
:1053000011F44B7FA6C342FF03C085EF92E002C0B9
:1053100088EF92E000D000D02AE735E00C94AA3163
:105320006091A1047091A20480E090E00E94077A4D
:105330000E94FE78803160F48093D30690E00E9452
:10534000325483ED96E066E170E041E050E0E5C75D
:1053500000D000D0EDB7FEB731968EE795E0ADB73F
:10536000BEB712969C938E9311978091D306828339
:1053700094CF0C9400000C94B9316091A104709109
:10538000A20480E090E00E94077A8C0165E273E05D
:105390000E941C7A009739F4219A8091B904909167
:1053A000BA048061B0C7C80167E273E00E941C7A4A
:1053B000009739F4229A8091B9049091BA048062DE
:1053C000A2C7C80169E273E00E941C7A009739F411
:1053D000239A8091B9049091BA04806494C7C8015B
:1053E0006BE273E00E941C7A009739F4239A809153
:1053F000B9049091BA04806886C7C80168EF72E06A
:105400000E941C7A4091B9045091BA04009739F473
:105410004F705093BA044093B9042B9A78C744FF55
:1054200003C085EF92E002C088EF92E000D000D088
:105430002CEA35E0EDB7FEB7328321839483838372
:105440000E94AC7A8091B9040F900F900F900F904A
:1054500085FF03C085EF92E002C088EF92E000D0A4
:1054600000D021EA35E0ADB7BEB712963C932E933B
:10547000119714969C938E9313970E94AC7A809107
:10548000B9040F900F900F900F9086FF03C085EF27
:1054900092E002C088EF92E000D000D026E935E02B
:1054A000EDB7FEB732832183948383830E94AC7A65
:1054B0008091B9040F900F900F900F9087FF03C059
:1054C00085EF92E002C088EF92E000D000D02BE898
:1054D00035E0ADB7BEB712963C932E931197149654
:1054E0009C938E9313973CC700D086E394E0EDB76E
:1054F000FEB7928381830E94AC7A20919C040F9026
:105500000F902223A9F000D000D0EDB7FEB731965E
:1055100083E394E0ADB7BEB712969C938E93119738
:10552000228313820E94AC7A0F900F900F900F90FD
:1055300088E10FB6F89480936000109260000FBE6F
:105540000C94007C16C70E94DC4A13C76091A1042A
:105550007091A20480E090E00E94077A1C0165EF40
:1055600072E00E941C7A009749F40E948951809150
:10557000B9049091BA0481608D7FC5C6C10168EFFE
:1055800072E00E941C7A009741F40E94EB508091D7
:10559000B9049091BA048C7FB6C60DE213E0C10144
:1055A000B8010E941C7A009749F40E94EB50809148
:1055B000B9049091BA048E7F8260A5C68091B90427
:1055C00081FF0BC000D000D08BEB95E0EDB7FEB7AC
:1055D0009283818314830383C3C680FF03C085EF56
:1055E00092E002C088EF92E000D000D027EB35E0D7
:1055F00070CF00D089E094E0EDB7FEB7928381834D
:105600000E94AC7A8DB79EB740970FB6F8949EBFB4
:105610000FBE8DBFEDB7FEB731968BEE93E0ADB701
:10562000BEB712969C938E931197809157209091BC
:105630005820A0915920B0915A2082839383A4834B
:10564000B58380914B2090914C20A0914D20B0913A
:105650004E2086839783A087B18780914F209091B9
:105660005020A0915120B091522082879387A48727
:10567000B5878091532090915420A0915520B091EE
:10568000562086879787A08BB18B0E94AC7A209199
:105690009C04EDB7FEB772960FB6F894FEBF0FBE2E
:1056A000EDBF222309F465C600D000D0EDB7FEB7E8
:1056B000319688EE93E0EACDF89481E090E00E9484
:1056C0005708182F80E090E00E945708082F789420
:1056D000F89483E090E00E945708F82E82E090E072
:1056E0000E945708E82E789400D000D000D02EED0C
:1056F00033E0EDB7FEB7328321832091F817309164
:10570000F9174091FA175091FB17ADB7BEB7139632
:105710002D933D934D935C9316970E94AC7A00D0E5
:1057200000D0EDB7FEB7319627EB33E0ADB7BEB78B
:1057300012963C932E931197E2821382F482158283
:1057400006831782108711860E94AC7AEDB7FEB7E8
:105750003A960FB6F894FEBF0FBEEDBF0E94161A20
:105760002091660000D000D0EDB7FEB731968BEAED
:1057700093E0ADB7BEB712969C938E931197228398
:1057800013820E94AC7A0F900F900F900F900E949E
:10579000730C20919C04222309F4EBC500D000D0A7
:1057A000EDB7FEB7319688EA93E070CD80E090E0E7
:1057B0000E947F0C81E090E00E947F0C20919C046D
:1057C000222309F4D6C500D000D0EDB7FEB731963C
:1057D00085EA93E05BCD0E94F1170E94730C209143
:1057E0009C04222309F4C5C500D000D0EDB7FEB754
:1057F000319682EA93E04ACD6091A1047091A204AF
:1058000080E090E00E94077A8C0165EF72E00E94D0
:105810001C7A009731F48091B9049091BA048860A1
:1058200072C5C80168EF72E00E941C7A4091B90409
:105830005091BA04009711F4477F0BC143FF03C096
:1058400085EF92E002C088EF92E000D000D02FEB0D
:1058500035E080C56091A1047091A20480E090E0E1
:105860000E94077A62E373E00E941C7A009741F578
:10587000F89483EF96E00E94C13E0CC0C8010D96DB
:105880000E940D4288E495E0B8010E947B3EC80169
:105890000E94873F082F192F0115110579F704C0C1
:1058A00083EF96E00E94023F83EF96E00E94673FFD
:1058B0000097B1F783EF96E00E94BD3E78944BC00D
:1058C00083EF96E00E94C13E482F592F7A0108E3EA
:1058D00013E03DC08DB79EB70C970FB6F8949EBFEE
:1058E0000FBE8DBFEDB7FEB73196ADB7BEB71296FE
:1058F0001C930E931197D70112968C911297828365
:10590000138213968C9113978483158218968C9129
:1059100018978683178214968D919C91159791877D
:10592000808716968D919C911797938782870E9406
:105930009A7AEDB7FEB73C960FB6F894FEBF0FBE4D
:10594000EDBFC7010E94873F482F592F7A01E1140C
:10595000F10409F0BFCF20919C04222309F409C56A
:1059600000D000D0EDB7FEB731968FE993E08ECC32
:105970000E94E81AFEC46091A1047091A20480E024
:1059800090E00E94077A8C0165EF72E00E941C7A19
:10599000009751F48091B9049091BA049260909369
:1059A000BA048093B90410C0C80168EF72E00E9485
:1059B0001C7A4091B9045091BA04009771F45D7F4C
:1059C0005093BA044093B90489EB94E064E170E029
:1059D00042E050E00E94FC7B17C051FF03C085EFFE
:1059E00092E002C088EF92E000D000D023EC35E0D6
:1059F000EDB7FEB732832183948383830E94AC7A10
:105A00000F900F900F900F9081E00E947E0AB1C41A
:105A10006091A1047091A20480E090E00E94077A56
:105A20008C0167E073E00E941C7A009731F480914A
:105A3000B9049091BA049E7F66C4C8016CEF72E00D
:105A40000E941C7A4091B9045091BA04009731F435
:105A500051605093BA044093B90459C450FF03C035
:105A60008CEF92E002C087E093E000D000D02FE5F9
:105A700033E0ADB7BEB712963C932E93119703C493
:105A80006091A1047091A20480E090E00E94077AE6
:105A90000097A9F160E070E040E150E00E94EC77EF
:105AA0006093B3047093B4048093B5049093B604E8
:105AB00000D000D000D02EE833E0EDB7FEB732833F
:105AC0002183ADB7BEB713966D937D938D939C9351
:105AD00016970E94AC7AEDB7FEB736960FB6F894DB
:105AE000FEBF0FBEEDBF83EB94E06EE070E044E0DC
:105AF00050E00E94FC7B81E00E94981B3AC480E049
:105B00000E94981B0E94730C00D000D000D089E73F
:105B100093E0ADB7BEB712969C938E931197809188
:105B2000B3049091B404A091B504B091B604EDB75C
:105B3000FEB783839483A583B6830E94AC7A8DB726
:105B40009EB706960FB6F8949EBF0FBE8DBF81E03C
:105B50000E94981B0E94730C20919C04222309F43C
:105B600008C400D000D0EDB7FEB7319686E793E0C9
:105B70008DCB6091A1047091A20480E090E00E941E
:105B8000077A009741F160E070E04AE050E00E943F
:105B9000EC777093B8046093B70400D000D0EDB7F1
:105BA000FEB7319629E533E0ADB7BEB712963C9308
:105BB0002E931197738362830E94AC7A0F900F909B
:105BC0000F900F9087EB94E062E170E042E050E0CC
:105BD0000E94FC7B14C000D000D088E393E0EDB7B6
:105BE000FEB7928381838091B7049091B804948327
:105BF00083830E94AC7A0F900F900F900F902091AA
:105C00009C04222309F4B5C300D000D0EDB7FEB741
:105C1000319685E393E03ACB0E944A4220919C045E
:105C2000222309F4A6C300D000D0EDB7FEB7319609
:105C300082E393E02BCB00D082E293E0EDB7FEB796
:105C4000928381830E94AC7A0F900F900E946E190C
:105C500000D000D08AE193E0ADB7BEB712969C9316
:105C60008E93119782E997E114969C938E931397E4
:105C70000E94AC7A0F900F9086E193E0EDB7FEB7EB
:105C8000928381830E94AC7A0F900F9080E00E94F3
:105C9000AE1A00D080E193E0ADB7BEB712969C93E8
:105CA0008E9311970E94AC7A0F900F900E9426104D
:105CB0008091451C80FF02C00E9466110E947319EA
:105CC00000D000D0EDB7FEB7319683E093E0ADB7DA
:105CD000BEB712969C938E9311978091D3068283C0
:105CE00013820E94AC7A8BEE92E0EDB7FEB79283FE
:105CF000818380E490E0948383830E94AC7A00D017
:105D0000EDB7FEB7319688ED92E0ADB7BEB712960B
:105D10009C938E9311978091C124828313828091EA
:105D2000C224848315820E94AC7A0F900F9083EC7A
:105D300092E0EDB7FEB7928381838091B704909192
:105D4000B804948383830E94AC7A00D080EB92E005
:105D5000ADB7BEB712969C938E9311978091B30402
:105D60009091B404A091B504B091B604EDB7FEB71C
:105D700083839483A583B6830E94AC7A8DB79EB744
:105D800006960FB6F8949EBF0FBE8DBF81E00E94AD
:105D9000981B0E94600B00D000D000D023EA32E0B4
:105DA000ADB7BEB712963C932E931197EDB7FEB7E1
:105DB00063837483858396830E94AC7A8DB79EB784
:105DC00006960FB6F8949EBF0FBE8DBF0E94970B2C
:105DD0000E94740B00D000D000D025E932E0ADB7AE
:105DE000BEB712963C932E931197EDB7FEB763831F
:105DF0007483858396830E94AC7A8DB79EB706968E
:105E00000FB6F8949EBF0FBE8DBF1D9B03C08CE0E4
:105E100093E002C088EF92E000D000D029E832E0A1
:105E2000ADB7BEB712963C932E93119714969C93E0
:105E30008E9313970E94AC7A20919C2430919D24DC
:105E400040919E2450919F248091A0249091A12460
:105E5000A091A224B091A32400D000D000D00DB70F
:105E60001EB70F5F1F4F6BE672E0EDB7FEB7728390
:105E70006183F80122833383448355838683978328
:105E8000A087B1870E94AC7AEDB7FEB7319689E45E
:105E900092E0ADB7BEB712969C938E931197809106
:105EA000A9249091AA24A091AB24B091AC24828320
:105EB0009383A483B5838091AD249091AE24A09167
:105EC000AF24B091B02486839783A087B1870E94C6
:105ED000AC7AEDB7FEB738960FB6F894FEBF0FBE9A
:105EE000EDBF8FE392E0928381830E94AC7A809130
:105EF000B9040F900F9081FF0EC000D089E392E0AB
:105F0000ADB7BEB712969C938E9311970E94AC7A50
:105F10000F900F9017C080FF03C085EF92E002C082
:105F200088EF92E000D000D025E332E0EDB7FEB775
:105F300032832183948383830E94AC7A0F900F90E5
:105F40000F900F908091B90483FF03C085EF92E01A
:105F500002C088EF92E000D000D022E232E0ADB77C
:105F6000BEB712963C932E93119714969C938E93E2
:105F700013970E94AC7A8091B9049091BA040F9063
:105F80000F900F900F9091FF03C085EF92E002C039
:105F900088EF92E000D000D025E132E0EDB7FEB707
:105FA00032832183948383830E94AC7A8091CE06CE
:105FB0009091CF0628E032E0ADB7BEB712963C9381
:105FC0002E93119714969C938E9313970E94AC7AFC
:105FD0000F900F900F900F90779903C085EF92E08C
:105FE00002C088EF92E000D000D02FEF31E0EDB793
:105FF000FEB732832183948383830E94AC7A80919D
:10600000B9049091BA040F900F900F900F9090FFE9
:1060100003C08CEF92E002C087E093E000D000D094
:106020002FE533E0ADB7BEB712963C932E93119790
:1060300014969C938E9313970E949A7A20919C04B5
:106040000F900F900F900F90222309F492C100D06F
:1060500000D0EDB7FEB731968CEF91E017C90E94E2
:106060003B1A20919C04222309F483C100D000D064
:10607000EDB7FEB7319689EF91E008C90E94361757
:106080000097B9F500D000D000D08EEE91E0EDB7CA
:10609000FEB7928381838091411890914218A0911C
:1060A0004318B091441883839483A583B6830E94D8
:1060B000AC7A81EE91E0ADB7BEB712969C938E9309
:1060C00011978091BD249091BE24A091BF24B091DE
:1060D000C024EDB7FEB783839483A583B6830E9463
:1060E000AC7A8DB79EB706960FB6F8949EBF0FBEDA
:1060F0008DBF0E94730C20919C04222309F439C1A6
:1061000000D000D0EDB7FEB731968EED91E0BEC85D
:1061100083E061E048E021E00E94F11200D000D06D
:1061200000D087ED91E0EDB7FEB792838183809137
:10613000341890913518A0913618B0913718838390
:106140009483A583B6830E94AC7A00D000D0EDB7CB
:10615000FEB7319686EC91E0ADB7BEB712969C9330
:106160008E9311978091381890913918A0913A1810
:10617000B0913B1882839383A483B58380913C18AC
:1061800090913D18A0913E18B0913F188683978357
:10619000A087B1870E94AC7AEDB7FEB73A960FB6EA
:1061A000F894FEBF0FBEEDBF0E94730C20919C04BB
:1061B000222309F4DEC000D000D0EDB7FEB731963F
:1061C00083EC91E063C86091A1047091A20480E027
:1061D00090E00E94077A68E673E00E941C7A0097BC
:1061E000B1F46091A1047091A20480E090E00E945B
:1061F000077A009709F4BDC00E94FE78803108F04C
:10620000B8C090915201982B90935201B2C08091E6
:10621000520100D000D027EC35E0EDB7FEB7328355
:10622000218390E08F709070948383830E94AC7A76
:106230000F900F900F900F900E94730C9AC0609176
:10624000A1047091A20480E090E00E94077ABC0152
:10625000009769F082E997E14AE050E00E94257AD0
:1062600082E997E160E270E04AE050E056C000D079
:1062700000D08DE693E0ADB7BEB712969C938E9397
:10628000119782E997E114969C938E9313970E943D
:106290009A7A68C06091A1047091A20480E090E0B5
:1062A0000E94077A8C0165EF72E00E941C7A0097C9
:1062B00041F40E94CD4F8091B9049091BA0494604A
:1062C00022C0C80168EF72E00E941C7A009741F575
:1062D000F8940E94DB4F88E10FB6F8948093600039
:1062E000109260000FBE84B7877F84BF80916000EA
:1062F0008861809360001092600078948091B90466
:106300009091BA049B7F9093BA048093B90489EB6F
:1063100094E064E170E042E050E00E94FC7B29C020
:10632000C80165E773E00E941C7A4091B90450915E
:10633000BA04009721F452FF1CC0F894FFCF52FF1B
:1063400003C085EF92E002C088EF92E000D000D059
:1063500024ED35E0EDB7FEB7328321839483838348
:106360000E94AC7A0F900F900F900F9002C00E9485
:106370005B18A981BA8111961C921E9283E00F903E
:106380000F90CF91DF911F910F91FF90EF90DF90D1
:10639000CF90BF90AF909F908F907F906F905F90C5
:1063A0004F903F902F900895F89491E2E0E0F0E054
:1063B000909357008491E2E0F0E09093570024918D
:1063C000E4E0F0E090935700E49190E0A0E0B0E0CA
:1063D000DC019927882730E040E050E0542F432F1C
:1063E000322F2227820F931FA41FB51F8E0F911DDE
:1063F000A11DB11D8093F8179093F917A093FA1778
:10640000B093FB1778940895DF93CF93CDB7DEB7A1
:1064100061970FB6F894DEBF0FBECDBFCE010296D6
:106420006EE070E042E050E00E94DE7B8A819B815A
:106430002FEF8F3F920749F483EB94E06EE070E01A
:1064400042E050E00E94FC7B0AC0A0E0B0E08093F4
:10645000B3049093B404A093B504B093B604CE01F2
:10646000029662E170E042E050E00E94DE7B8A81A9
:106470009B812FEF8F3F920779F48CE390E090930C
:10648000B8048093B70487EB94E062E170E042E0E7
:1064900050E00E94FC7B04C09093B8048093B70442
:1064A000CE01029664E170E042E050E00E94DE7BA3
:1064B0008A819B812FEF8F3F920779F48AE090E0E9
:1064C0009093BA048093B90489EB94E064E170E09E
:1064D00042E050E00E94FC7B04C09093BA04809399
:1064E000B904CE01029660E070E042E050E00E9404
:1064F000DE7B8A819B812FEF8F3F920769F4109298
:10650000CF061092CE068EEC96E060E070E042E09E
:1065100050E00E94FC7B04C09093CF068093CE068F
:1065200081EB94E267E170E049E050E00E94DE7B9D
:106530000E94E20DCE01049666E070E044E050E077
:106540000E94DE7B8C819D81AE81BF818F3F2FEFCA
:1065500092072FEFA2072FEFB20749F484E994E0E6
:1065600066E070E044E050E00E94FC7B08C084E9F3
:1065700094E066E070E044E050E00E94DE7BCE01F3
:1065800004966AE070E044E050E00E94DE7B8C817B
:106590009D81AE81BF818F3F2FEF92072FEFA20722
:1065A0002FEFB20749F488E994E06AE070E044E034
:1065B00050E00E94FC7B08C088E994E06AE070E04B
:1065C00044E050E00E94DE7BCE01049662E070E081
:1065D00044E050E00E94DE7B8C819D81AE81BF81D2
:1065E0008F3F2FEF92072FEFA2072FEFB20749F44B
:1065F00080E994E062E070E044E050E00E94FC7BBF
:1066000008C080E994E062E070E044E050E00E945D
:10661000DE7BCE01019666E170E041E050E00E9431
:10662000DE7B89818F3F49F483ED96E066E170E07F
:1066300041E050E00E94FC7B08C083ED96E066E1FB
:1066400070E041E050E00E94DE7BCE01089660E2FF
:1066500070E04AE050E00E94DE7B88858F3F49F47D
:1066600082E997E160E270E04AE050E00E94FC7B42
:1066700008C082E997E160E270E04AE050E00E94E1
:10668000DE7B61960FB6F894DEBF0FBECDBFCF9113
:10669000DF9108950E94C14F6C9A6B9A6A9A6F9A23
:1066A000729A749A739A779A809880B3897F80BB24
:1066B00087E080937E00549A0E94D4310E94043275
:1066C00081E00E947E0A80E090E00E94F60D0E9428
:1066D0004A498091B90486FD239A0895CF93DF93A8
:1066E000EC0188819981009731F02AE08931920785
:1066F00009F092C088C00E944A338091B90480FD9D
:1067000006C081FF02C01D9902C00E94EB5080911B
:1067100070008C7F809370008091B60080628093BF
:10672000B6001092B20082E08093B1008091B60072
:1067300090E0877090700097C9F780917000816039
:106740008093700080E090E06EE578E00E94A44FB6
:106750000E946E1980E00E94AE1A00D08DEB91E08D
:10676000ADB7BEB712969C938E9311970E94AC7AE8
:106770000F900F900E9426108091451C86FF02C04A
:106780000E94874A8091D30690E00E9432548AE1A9
:10679000809301078AE190E00E94AA5200D000D0C5
:1067A00000D0EDB7FEB731968AE793E0ADB7BEB73C
:1067B00012969C938E931197809101078283138286
:1067C0008091D306848315820E949A7A10920007E2
:1067D0001092FF06EDB7FEB736960FB6F894FEBFDF
:1067E0000FBEEDBF87EC94E09093BB248093BA2456
:1067F00083E290E09093F8068093F70689E19AE0AF
:10680000998388830DC0633259F48FEF96E060E07E
:1068100070E00E94BF1EE6CF1982188283E001C09B
:1068200081E0DF91CF9108958436910534F100D055
:1068300000D02CE833E0EDB7FEB732832183948398
:1068400083830E949A7A8091572090915820A0913A
:106850005920B0915A200196A11DB11D8093572057
:1068600090935820A0935920B0935A200F900F90E6
:106870000F900F9021E030E002C020E030E0C9012D
:1068800008956F927F928F929F92AF92BF92CF9214
:10689000DF92EF92FF920F931F93DF93CF93CDB7C9
:1068A000DEB7CB57D0400FB6F894DEBF0FBECDBFDA
:1068B0003C01633851F48FED96E0EC966FAFEC97A6
:1068C0000E94013CEC966FADEC97D3018D919C91A9
:1068D0001197B8E08B3F9B07E9F0E8E08C3F9E07FB
:1068E00018F4009761F0FDC6F9E08F3D9F0709F4A9
:1068F000D1C629E0863E920709F0F3C6E4C68FEDC3
:1069000096E061E870E044E455E00E94E63B8BEFDE
:1069100098E0D4C6623109F0E9C60E94970B8091D5
:10692000B3049091B404A091B504B091B60493FF60
:1069300002C00E9436178091B3049091B404A091D4
:10694000B504B091B60494FF0AC00E94600B609336
:10695000A4247093A5248093A6249093A7248091C7
:10696000B30480FF32C0EDB7FEB738970FB6F89486
:10697000FEBF0FBEEDBF3196CE010396ADB7BEB7D9
:1069800012969C938E93119787E790E0938382836E
:1069900080EA93E09583848382E997E197838683F5
:1069A0000E940A7BE82E092FEDB7FEB738960FB686
:1069B000F894FEBF0FBEEDBF0E941434009709F09B
:1069C000A6CF802F0E2D182F02C000E010E080917E
:1069D000B30481FF5FC083E0C82ED12CCC0EDD1E36
:1069E00000D000D000D0EDB7FEB73196C601800FC1
:1069F000911FADB7BEB712969C938E93119787E700
:106A000090E09383828388EA93E0958384830E9455
:106A10000A7B080F191FB1EBEB2EB4E2FB2EEDB78A
:106A2000FEB736960FB6F894FEBF0FBEEDBFA7E7D0
:106A3000AA2EB12CFCEA8F2EF3E09F2ED7012D91C8
:106A40007D01EDB7FEB738970FB6F894FEBF0FBEC5
:106A5000EDBF3196C601800F911FADB7BEB712963C
:106A60009C938E931197B382A2829582848226830F
:106A700017820E940A7B080F191FEDB7FEB73896E0
:106A80000FB6F894FEBF0FBEEDBFF9EBEF16F4E2C0
:106A9000FF06A1F68091B3049091B404A091B504CF
:106AA000B091B6040097A105B10581F12DB73EB7AD
:106AB000285030400FB6F8943EBF0FBE2DBFEDB743
:106AC000FEB73196CE010396800F911FADB7BEB7CA
:106AD00012969C938E93119787E790E0938382831D
:106AE00081EB93E0958384838091D1069091D206C7
:106AF000978386830E940A7B080F191FEDB7FEB7A4
:106B000038960FB6F894FEBF0FBEEDBF8091B30468
:106B100082FF50C089E290E06BE270E04AE250E010
:106B200027E00E94604681EB94E20E94D0482DB796
:106B30003EB72A5030400FB6F8943EBF0FBE2DBF6F
:106B4000EDB6FEB60894E11CF11C9E012D5F3F4F8F
:106B5000200F311FADB7BEB712963C932E931197FD
:106B600027E730E0F7013383228328EB33E03583D6
:106B700024839C01B901882777FD8095982F0E9476
:106B80005C7420E030E048EC52E40E94F273D701DC
:106B900016966D937D938D939C9319970E940A7B13
:106BA000080F191FEDB7FEB73A960FB6F894FEBF5F
:106BB0000FBEEDBF8091B30483FF56C089E290E021
:106BC0006BE270E04AE250E026E00E94604681E01D
:106BD00090E00E94E70B8093D50680EB97E10E943E
:106BE000D0482DB73EB72A5030400FB6F8943EBF7C
:106BF0000FBE2DBFEDB6FEB60894E11CF11C9E0140
:106C00002D5F3F4F200F311FADB7BEB712963C939B
:106C10002E93119727E730E0F7013383228322EC8C
:106C200033E0358324839C01B901882777FD809563
:106C3000982F0E945C7420E030E048EC52E40E94FF
:106C4000F273D70116966D937D938D939C9319974C
:106C50000E940A7B080F191FEDB7FEB73A960FB6D0
:106C6000F894FEBF0FBEEDBF8091B30484FF36C021
:106C70002DB73EB72A5030400FB6F8943EBF0FBE36
:106C80002DBFEDB7FEB73196CE010396800F911F51
:106C9000ADB7BEB712969C938E93119787E790E09D
:106CA000938382838DEC93E09583848380919C17FA
:106CB00090919D17A0919E17B0919F1786839783FF
:106CC000A087B1870E940A7B080F191FEDB7FEB796
:106CD0003A960FB6F894FEBF0FBEEDBF8091B30495
:106CE00085FF31C00E94740B2DB73EB72A5030404B
:106CF0000FB6F8943EBF0FBE2DBFEDB7FEB731966D
:106D00009E012D5F3F4F200F311FADB7BEB71296CA
:106D10003C932E93119727E730E0338322832BEDAA
:106D200033E03583248366837783808791870E944D
:106D30000A7B080F191FEDB7FEB73A960FB6F89405
:106D4000FEBF0FBEEDBF8091B30486FF3AC0F8943A
:106D500080919C2490919D24A0919E24B0919F2489
:106D600078942DB73EB72A5030400FB6F8943EBF06
:106D70000FBE2DBF4DB75EB74F5F5F4F9E012D5FBA
:106D80003F4F200F311FEDB7FEB73283218327E736
:106D900030E0FA013383228329EE33E03583248304
:106DA00086839783A087B1870E940A7B080F191FEB
:106DB0002DB73EB7265F3F4F0FB6F8943EBF0FBECC
:106DC0002DBF8091B30487FF8AC08091B704909152
:106DD000B804009709F483C0F894C0909C24D09024
:106DE0009D24E0909E24F0909F2478948091A81791
:106DF0009091A917A091AA17B091AB17A70196017E
:106E0000281B390B4A0B5B0BCA01B9010E945A744B
:106E1000862EA72EB82E992E6091B7047091B804D3
:106E200080E090E00E945A749B01AC01682D7A2D9D
:106E30008B2D992D0E94F2735C014DB75EB74A50BD
:106E400050400FB6F8945EBF0FBE4DBFEDB7FEB712
:106E50003196CE010396800F911FADB7BEB7129643
:106E60009C938E93119787E790E09383828384EFBE
:106E700093E095838483262F372F4A2D5B2D26831D
:106E8000378340875187EC966FAFEC97EB967FAFD7
:106E9000EB970E940A7B080F191FEC966FADEC97D9
:106EA000EB967FADEB97862F972FAA2DBB2D809366
:106EB000A9249093AA24A093AB24B093AC24C092AD
:106EC000A817D092A917E092AA17F092AB17EDB7C6
:106ED000FEB73A960FB6F894FEBF0FBEEDBF809195
:106EE000B3049091B404A091B504B091B60490FF9E
:106EF00040C0F8948091A0249091A124A091A22454
:106F0000B091A32478942DB73EB72A5030400FB6E5
:106F1000F8943EBF0FBE2DBF4DB75EB74F5F5F4FBA
:106F20009E012D5F3F4F200F311FEDB7FEB732831B
:106F3000218327E730E0FA013383228321E034E024
:106F40003583248386839783A087B1870E940A7B39
:106F5000080F191F2DB73EB7265F3F4F0FB6F894A5
:106F60003EBF0FBE2DBFC8010E941434009709F028
:106F7000CECC8091B3049091B404A091B504B091AB
:106F8000B60491FF88C08091B7049091B80400972F
:106F900009F481C0F894C090A024D090A124E0907E
:106FA000A224F090A32478948091AC179091AD170F
:106FB000A091AE17B091AF17A7019601281B390B0E
:106FC0004A0B5B0BCA01B9010E945A745B014C0168
:106FD0006091B7047091B80480E090E00E945A7408
:106FE0009B01AC016A2D7B2D882D992D0E94F27397
:106FF0005C014DB75EB74A5050400FB6F8945EBF83
:107000000FBE4DBFEDB7FEB73196CE010396800F90
:10701000911FADB7BEB712969C938E93119787E7D9
:1070200090E0938382838CE094E095838483262F81
:10703000372F4A2D5B2D2683378340875187EC9667
:107040006FAFEC97EB967FAFEB970E940A7B080F30
:10705000191FEC966FADEC97EB967FADEB97862FF3
:10706000972FAA2DBB2D8093AD249093AE24A0938F
:10707000AF24B093B024C092AC17D092AD17E09279
:10708000AE17F092AF17EDB7FEB73A960FB6F89479
:10709000FEBF0FBEEDBF8091B3049091B404A091E8
:1070A000B504B091B60492FF3EC080914720909104
:1070B0004820A0914920B0914A202DB73EB72A50D0
:1070C00030400FB6F8943EBF0FBE2DBF4DB75EB730
:1070D0004F5F5F4F9E012D5F3F4F200F311FEDB778
:1070E000FEB73283218327E730E0FA01338322831E
:1070F00029E134E03583248386839783A087B18791
:107100000E940A7B080F191F2DB73EB7265F3F4F1D
:107110000FB6F8943EBF0FBE2DBFC8010E941434B5
:10712000009709F0F4CB8091B3049091B404A0913E
:10713000B504B091B60493FF3CC04DB75EB74A505A
:1071400050400FB6F8945EBF0FBE4DBFEDB7FEB70F
:107150003196CE010396800F911FADB7BEB7129640
:107160009C938E93119787E790E09383828384E2C8
:1071700094E0958384838091411890914218A09166
:107180004318B091441886839783A087B1870E94E3
:107190000A7B080F191FEDB7FEB73A960FB6F894A1
:1071A000FEBF0FBEEDBFC8010E941434009709F066
:1071B000AECB8091B3049091B404A091B504B0918A
:1071C000B60494FF3CC02DB73EB72A5030400FB6EE
:1071D000F8943EBF0FBE2DBFEDB7FEB73196CE017E
:1071E0000396800F911FADB7BEB712969C938E93F6
:1071F000119787E790E0938382838FE294E09583F1
:1072000084838091A4249091A524A091A624B09178
:10721000A72486839783A087B1870E940A7B080FE3
:10722000191FEDB7FEB73A960FB6F894FEBF0FBE22
:10723000EDBFC8010E941434009709F068CB80911B
:10724000B3049091B404A091B504B091B60495FF35
:1072500048C081E00E94120B2DB73EB72A50304043
:107260000FB6F8943EBF0FBE2DBFEDB6FEB6089424
:10727000E11CF11C9E012D5F3F4F200F311FADB768
:10728000BEB712963C932E93119727E730E0F70193
:10729000338322832CE334E03583248320919404C8
:1072A0003091950440919604509197040E940C757A
:1072B000D70116966D937D938D939C9319970E9499
:1072C0000A7B080F191FEDB7FEB73A960FB6F89470
:1072D000FEBF0FBEEDBFC8010E941434009709F035
:1072E00016CB8091B3049091B404A091B504B091F1
:1072F000B60496FF48C082E00E94120B2DB73EB73D
:107300002A5030400FB6F8943EBF0FBE2DBFEDB6E9
:10731000FEB60894E11CF11C9E012D5F3F4F200F2B
:10732000311FADB7BEB712963C932E93119727E746
:1073300030E0F7013383228329E434E0358324836A
:10734000209198043091990440919A0450919B04A3
:107350000E940C75D70116966D937D938D939C9327
:1073600019970E940A7B080F191FEDB7FEB73A96CE
:107370000FB6F894FEBF0FBEEDBFC8010E941434D3
:10738000009709F0C4CA8091B3049091B404A0910D
:10739000B504B091B60497FF06C083E061E046E013
:1073A00020E00E94F1128091B3049091B404A09166
:1073B000B504B091B604A0FF06C083E061E046E0EA
:1073C00021E00E94F1128091B3049091B404A09145
:1073D000B504B091B60497FF3CC02DB73EB72A5014
:1073E00030400FB6F8943EBF0FBE2DBFEDB7FEB7CD
:1073F0003196CE010396800F911FADB7BEB712969E
:107400009C938E93119787E790E09383828386E520
:1074100094E0958384838091381890913918A091D5
:107420003A18B0913B1886839783A087B1870E9452
:107430000A7B080F191FEDB7FEB73A960FB6F894FE
:10744000FEBF0FBEEDBFC8010E941434009709F0C3
:107450005ECA8091B3049091B404A091B504B09138
:10746000B604A0FF3CC02DB73EB72A5030400FB63F
:10747000F8943EBF0FBE2DBFEDB7FEB73196CE01DB
:107480000396800F911FADB7BEB712969C938E9353
:10749000119787E790E0938382838EE594E095834C
:1074A000848380913C1890913D18A0913E18B09132
:1074B0003F1886839783A087B1870E940A7B080FB5
:1074C000191FEDB7FEB73A960FB6F894FEBF0FBE80
:1074D000EDBFC8010E941434009709F018CA779ACA
:1074E0008091CE069091CF0693FD749A8091CE063E
:1074F0009091CF0682FD08C08091B90480FD04C040
:1075000081FF31C01D9B2FC000D000D089E694E0E0
:10751000ADB7BEB712969C938E931197CE0103968A
:1075200014969C938E9313970E949A7A20919C04B0
:107530000F900F900F900F902223A9F000D000D051
:10754000EDB7FEB7319687EB91E0ADB7BEB71296B7
:107550009C938E931197228313820E94AC7A0F9092
:107560000F900F900F908FE189838091F2068A83AC
:10757000FE01E00FF11F138278010894E11CF11C59
:107580008091CE069091CF0680FF12C000D000D02F
:1075900080E794E0EDB7FEB7928381830D5F1F4FC4
:1075A000148303830E949A7A0F900F900F900F908C
:1075B00022E030E0E20EF31E8E010F5F1F4FC80184
:1075C000B7010E945E458091B90482FF42C083EA00
:1075D00094E0B801A7012CE930E20E94E3498091D0
:1075E000CE069091CF0692FF34C00CE910E2E1E89C
:1075F000CE2EE4E0DE2ED8018D918D0100D000D09A
:10760000EDB7FEB73196ADB7BEB71296DC92CE920B
:107610001197828313820E949A7A0F900F900F9095
:107620000F90B0E20C3A1B0731F78AE090E00E941D
:10763000CC7A00D000D086E894E0EDB7FEB7928314
:107640008183F482E3820E949A7A0F900F900F90C8
:107650000F908091CE069091CF0682FD73980E9484
:1076600089518FED96E00E94043C8091D106909163
:10767000D206009711F00E94EB508091F2068F5FC6
:107680008093F2068091CE069091CF0682FF3FC98B
:10769000739A3DC98AEE96E00E94AB40009731F1A3
:1076A0000E9489518091B90487FD2B988AEE96E05B
:1076B00060E470E00E94804086EE99E0D30111966C
:1076C0009C938E9313C08AEE96E00E94AB40009785
:1076D00069F00E94EB508091B90487FF18C92B9A7A
:1076E00016C9F3011182108283E001C081E0C55800
:1076F000DF4F0FB6F894DEBF0FBECDBFCF91DF9145
:107700001F910F91FF90EF90DF90CF90BF90AF90BF
:107710009F908F907F906F9008950895FC01DB01FA
:107720008C91808311968C91119781830895FC012F
:10773000DB0190818C91981741F421E030E0918138
:1077400011968C911197981711F020E030E0C90143
:107750000895FC0180818093C12481818093C2249B
:107760000895DC011996ED91FC911A970280F3813E
:10777000E02D309709F009950895EF92FF920F934D
:107780001F93DF93CF9300D0CDB7DEB78C0188E194
:107790000E94D945BC017E010894E11CF11CC7017F
:1077A0000E948E3BD8011996ED91FC911A97019099
:1077B000F081E02DC801B70109950F900F90CF918E
:1077C000DF911F910F91FF90EF900895EF92FF923C
:1077D0000F931F93CF93DF93EC018B017A0144E564
:1077E00055E00E94123CFA86E986C80168E575E01A
:1077F0000E94713CDF91CF911F910F91FF90EF900C
:1078000008950E942B3C0895CF93DF93EC0188E10B
:1078100061EC74E20E94CF45CE010E942E3CDF91C4
:10782000CF910895EF92FF920F931F93CF93DF9321
:10783000EC018B017A010E944A3CF886EF82C80174
:107840006CE575E00E94713CDF91CF911F910F9123
:10785000FF90EF9008950E94533C08950E94605756
:107860000895FC01A781B0852D913C91F9010995FE
:107870000895DC011796ED91FC9118970280F38131
:10788000E02D309709F00995089584E89EE00E9464
:10789000BD3E0895FC017383628384E89EE0BF01CE
:1078A0000E94483F0895BC0184E89EE00E940F3F7B
:1078B0000895CF93DF93EC0184E89EE00E94C13EDF
:1078C00008C0828193818C179D0739F0CF010E94F7
:1078D000873FE82FF92F3097A1F7CF01DF91CF91A4
:1078E00008950F931F93CF93DF938B010E94593C10
:1078F000EC01009731F01D830C83C8010E94B85938
:107900008E83DF91CF911F910F9108951F93CF9395
:10791000DF93EC01162F888580FF1DC0EC81FD816F
:107920003097C9F0D093890EC093880E82E0888783
:10793000CE0106960995992787FD9095029782308A
:10794000910510F0133829F4CE01BE010E94AF3C1E
:1079500002C081E08887DF91CF911F910895CF9277
:10796000DF92EF92FF920F931F93CF93DF93EC017F
:107970007B01C090880ED090890E0091860E1091E8
:10798000870EF80103C00190F081E02DEC17FD0790
:1079900019F03097C1F746C0209709F443C0888595
:1079A000882309F118860BC0C017D10729F0C80138
:1079B00067E8AE010E94863CF80100811181011543
:1079C000110591F7EC81FD81309769F0CE15DF0547
:1079D00051F0D093890EC093880ECE01069663E8CD
:1079E00040E050E00995E091860EF091870ECE17A9
:1079F000DF0791F4888199819093870E8093860E9A
:107A00000DC0808191818C179D0729F4888199810F
:107A10009183808303C0FC01309799F7D092890E3F
:107A2000C092880EDF91CF911F910F91FF90EF9040
:107A3000DF90CF9008951F93CF93DF9310928A0E1B
:107A4000C091860ED091870E11E00EC089858823E3
:107A500041F018871986CE0162E840E050E00E94AC
:107A6000863C0990D881C02D209781F7DF91CF9176
:107A70001F9108958091350F982F9F5F9093350F38
:107A800008956091880E7091890E0E94AF3C089510
:107A90008AE88093350F10928C0E10928B0E109204
:107AA000870E1092860E1092890E1092880E0895FD
:107AB00080918A0E882311F00E941B3D70918B0EDD
:107AC000772309F455C020918C0E30E0F901EE0FB8
:107AD000FF1FEE0FFF1FE20FF31FE357F14F60810F
:107AE0006093340F418152815093330F4093320F92
:107AF000838194819093310F8093300F2F5F3F4F9C
:107B00002F71307020938C0E715070938B0E0097F4
:107B100041F58091860E9091870E18C080918A0E53
:107B2000882311F00E941B3D4091320F5091330F7A
:107B300080912E0F90912F0F6091340F0E94863C00
:107B4000E0912E0FF0912F0F8081918190932F0F54
:107B500080932E0F80912E0F90912F0F0097F1F6AA
:107B600007C0613819F421E0FC0120870E94863C9F
:107B700080918A0E20918B0E30E0280F311DC901B3
:107B8000089580918A0E20918B0E30E0280F311DD0
:107B9000C901089570918B0E7032D9F020918C0E2E
:107BA000270F2F7120932D0F30E0F901EE0FFF1FEB
:107BB000EE0FFF1FE20FF31FE357F14F6083528375
:107BC0004183948383837F5F70938B0E20E030E04A
:107BD00002C021E030E0C9010895CF93DF93C09146
:107BE000880ED091890E0E94863CD093890EC09356
:107BF000880EDF91CF910895FC01AB019091860E24
:107C00008091870E9C01A32FB22F03C00D90BC91D1
:107C1000A02DAE17BF0791F01097C1F7309771F004
:107C200090838183F093870EE093860E81E08087B6
:107C300017821682CF0161E80E94ED3D0895FC0194
:107C4000009741F080858150823020F481E0818767
:107C500080938A0E089521E030E0FC01808588231E
:107C600011F420E030E0C9010895CF93DF93EC01D7
:107C70004A815B818C819D8160E070E00E94157A71
:107C80004A815B8188819981489F9001499F300D8D
:107C9000589F300D11248E819F8160E070E0A90112
:107CA0000E94157ADF91CF910895FC018281938122
:107CB00020E030E019C0A481B581A20FB31F4C9120
:107CC000442381F481E08C9340815181249FC00141
:107CD000259F900D349F900D112426813781280F08
:107CE000391F07C02F5F3F4F2817390720F320E0C7
:107CF00030E0C9010895FC0126813781428153811A
:107D000080E090E018C02617370781F4A481B58180
:107D1000A80FB91F2C91121614F421502C93048033
:107D2000F581E02DE80FF91F80810895A081B181D0
:107D30002A0F3B1F01968417950728F38FEF0895AC
:107D4000FC01CB01268137816217730790F0A08177
:107D5000B18162817381A69FA001A79F500DB69F3C
:107D6000500D1124420F531F21E030E08417950776
:107D700010F020E030E0C9010895FC01118210826A
:107D80000895FC01808191810895FB01208131815A
:107D9000FC01318320830895FC012081318121156C
:107DA000310511F407C09C01F90180819181009790
:107DB000D1F702C020E030E0C9010895CF93DF93EE
:107DC000DC012D913C91119721153105A9F0F901A4
:107DD00080819181009729F411961C921E920EC009
:107DE000F90120813181D9018D919C9111970097E2
:107DF000B9F71182108202C020E030E0C901DF91A2
:107E0000CF910895DC01ED91FC911197309729F005
:107E10008081918111969C938E93CF010895CF9389
:107E2000DF93FC01A081B1811097D9F0C0E0D0E0D0
:107E300016C0A617B70771F48D919C9111972097E2
:107E400019F49183808302C09983888311961C92D0
:107E50001E9207C0ED0198818981A92FB82F109734
:107E600041F7DF91CF9108950F931F93CF93DF9345
:107E70008C01EB010E940F3FF80180819181998371
:107E80008883D183C083DF91CF911F910F91089593
:107E9000EF92FF920F931F93CF93DF93EC017B013F
:107EA0000E940F3FF70111821082CE010E94CC3E4A
:107EB000FC01009719F4E882F98202C0F182E082A5
:107EC000DF91CF911F910F91FF90EF900895DC010A
:107ED000ED91FC91119720E030E005C02F5F3F4FFE
:107EE0000190F081E02D3097C9F7C9010895FB0199
:107EF000309721F4BA010E94343F0895DA0180815D
:107F0000918111969C938E9351834083089500979D
:107F100021F0FC012081318102C020E030E0C90164
:107F200008958091360F9091370F009729F41092A1
:107F3000390F1092380F08950E944D4EE091360F80
:107F4000F091370F2281338140815181240F351FF9
:107F5000281B390B0CC04281538160817181460F0F
:107F6000571F481B590B4217530708F49A01048006
:107F7000F581E02D309779F7280F391F3093390FAD
:107F80002093380F08958AE695E00E941F3E0895D9
:107F9000CF92DF92EF92FF920F931F93CF93DF93D5
:107FA0007C01FC0180819181009729F08A3591053F
:107FB00009F06EC00BC01092370F1092360F8AE591
:107FC00090E0F7019183808381E066C0673849F5CE
:107FD000CA01E091360FF091370F03C00480F5819C
:107FE000E02D309741F32681378128173907B1F307
:107FF000E093360FF093370F0FC016962D913C91FA
:1080000017972817390739F414962D913C91159735
:1080100035832483DF01FD01A481B581109769F7C1
:10802000CECF623861F6C091360FD091370F00E0A5
:1080300010E02BC0CE010E94B05D0097F1F08E8160
:108040009F8168E8AE010E94CA3D0097A1F41F829B
:108050001E828C819D810115110521F0F801958307
:10806000848304C09093370F8093360F1D821C8247
:108070000E94913FD8CF0E94C33F8E019C818D8189
:10808000C92EE6016E01D82EE601209799F697CF0A
:10809000F7011182108283E0DF91CF911F910F9140
:1080A000FF90EF90DF90CF900895CF93DF93EC0196
:1080B0000E94C33F8E819F81009769F0E091360F47
:1080C000F091370F06C0EC17FD07A9F00480F58189
:1080D000E02D3097C1F78091880E9091890E9F8393
:1080E0008E838091360F9091370F9D838C83D09330
:1080F000370FC093360F0E94913FDF91CF910895C3
:10810000CF93DF93EC010E94905DCE010E94554019
:10811000DF91CF910895CF93DF93EC010E949C5D96
:10812000CE010E945540DF91CF910895CF93DF9308
:10813000EC010E94A65DCE010E945540DF91CF91D7
:108140000895FC0180819181860F971F9183808320
:108150000E94913F089521E030E0FC0186819781E3
:10816000009711F020E030E0C9010895FC01228160
:10817000338180819181280F391FC9010895FC0145
:1081800080819181089521E030E08091360F9091B7
:10819000370F009711F420E030E0C9010895809175
:1081A000360F9091370F009729F02091380F3091BA
:1081B000390F02C020E030E0C9010895CF93DF936A
:1081C000EC01E091360FF091370F8E179F0741F4C5
:1081D0008C819D819093370F8093360F14C0FC01E2
:1081E000309731F0848195818C179D07C1F707C0C6
:1081F0001D821C821F821E82DF91CF9108958C8187
:108200009D81958384830E94913FF2CFCF92DF922C
:10821000EF92FF920F931F93CF93DF938C017A011C
:10822000FC0180819181009729F08B34910509F040
:1082300051C01EC08BE39FE00E94C13EC82EE601E4
:108240007E01F92EE70109C06C817D81CE01029685
:108250000E9480400990D881C02D2097A9F781E025
:1082600080933A0F8BE490E0F8019183808337C0CC
:108270006838A9F58BE39FE00E94C13EC82EE60155
:108280006E01D92EE60123C0CE010296E816F9064A
:10829000D9F48BE39FE0BE010E940F3FE090880E6F
:1082A000F090890E8A859B859093890E8093880E25
:1082B000EC85FD85309719F08E859F850995F092A4
:1082C000890EE092880ECECF0990D881C02D2097DC
:1082D000D9F6C8CFF8011182108283E001C081E095
:1082E000DF91CF911F910F91FF90EF90DF90CF9092
:1082F000089510923A0F8BE39FE00E94BD3E83E801
:1083000095E060E070E00E94FC3D08950F931F939C
:10831000CF93DF93EC010091880E1091890E1B879B
:108320000A875D874C873F872E8780913A0F882385
:1083300079F083E895E09093890E8093880ECE01C2
:1083400002960E9480401093890E0093880E02C00E
:108350007D836C838BE39FE0BE010E940F3F8BE324
:108360009FE0BE010E94483FDF91CF911F910F9186
:1083700008950F931F93CF93DF93EC0180913A0FF1
:10838000882391F00091880E1091890E83E895E082
:108390009093890E8093880ECE0102960E948B40A6
:1083A0001093890E0093880E8BE39FE0BE010E941C
:1083B0000F3F8BE39FE0BE010E94483FDF91CF91CA
:1083C0001F910F9108950F931F93CF93DF93EC01AB
:1083D00080913A0F882391F00091880E1091890EB8
:1083E00083E895E09093890E8093880ECE010296E3
:1083F0000E9496401093890E0093880E8BE39FE0B5
:10840000BE010E940F3F8BE39FE0BE010E94483FE8
:10841000DF91CF911F910F910895CF93DF93EC01DE
:1084200080913A0F882329F0CE0102960E94DE4007
:1084300004C01F821E82198618868BE39FE0BE014E
:108440000E940F3FDF91CF910895CF93DF93EC010E
:1084500080913A0F882331F0CE0102960E94AB4002
:108460009C0114C08BE39FE00E94C13EE82FF92FCE
:1084700006C0EC17FD0741F00190F081E02D309728
:10848000C1F721E030E002C020E030E0C901DF9117
:10849000CF9108950F931F930091C1241091C2248E
:1084A0000E947A4E2DB73EB7225530400FB6F89451
:1084B0003EBF0FBE2DBFEDB7FEB7319629E73DE0B9
:1084C000ADB7BEB712963C932E93119702831382D9
:1084D0001483158266837783808791878091B42681
:1084E0009091B526A091B626B091B7268287938742
:1084F000A487B5878091B8269091B926A091BA2615
:10850000B091BB2686879787A08BB18B8091BC26C4
:108510009091BD26A091BE26B091BF26828B938BF1
:10852000A48BB58B8091C0269091C126A091C226C4
:10853000B091C326868B978BA08FB18F8091C42674
:108540009091C526A091C626B091C726828F938FA1
:10855000A48FB58F8091C8269091C926A091CA2674
:10856000B091CB26868F978FA0A3B1A38091CC2604
:108570009091CD26A091CE26B091CF2682A393A331
:10858000A4A3B5A38091D0269091D126A091D22604
:10859000B091D32686A397A3A0A7B1A78091D42694
:1085A0009091D526A091D626B091D72682A793A7E1
:1085B000A4A7B5A78091D8269091D926A091DA26B4
:1085C000B091DB2686A797A7A0ABB1AB8091DC2644
:1085D0009091DD26A091DE26B091DF2682AB93AB91
:1085E000A4ABB5AB8091E0269091E126A091E22664
:1085F000B091E32686AB97ABA0AFB1AF8091E426F4
:108600009091E526A091E626B091E72682AF93AF40
:10861000A4AFB5AFEDB7FEB7FF968091E826909175
:10862000E926A091EA26B091EB2680839183A2836C
:10863000B383EDB7FEB7ED5BFF4F8091EC269091D1
:10864000ED26A091EE26B091EF2680839183A28340
:10865000B383EDB7FEB7E95BFF4F8091F0269091B1
:10866000F126A091F226B091F32680839183A28314
:10867000B383EDB7FEB7E55BFF4F8091F426909191
:10868000F526A091F626B091F72680839183A283E8
:10869000B383EDB7FEB7E15BFF4F8091F826909171
:1086A000F926A091FA26B091FB2680839183A283BC
:1086B000B3830E94AC7A0091C1241091C2242DB7DB
:1086C0003EB72E5A3F4F0FB6F8943EBF0FBE2DBF98
:1086D0000E947A4EADB7BEB7D2970FB6F894BEBF20
:1086E0000FBEADBFEDB7FEB731962AE03DE0129662
:1086F0003C932E9311970283138214831582668311
:108700007783808791878091FC269091FD26A091A8
:10871000FE26B091FF2682879387A487B587809134
:10872000002790910127A0910227B0910327868707
:108730009787A08BB18B8091042790910527A091FA
:108740000627B0910727828B938BA48BB58B8091E2
:10875000082790910927A0910A27B0910B27868BB3
:10876000978BA08FB18F80910C2790910D27A091AE
:108770000E27B0910F27828F938FA48FB58F809192
:10878000102790911127A0911227B0911327868F5F
:10879000978FA0A3B1A38091142790911527A09142
:1087A0001627B091172782A393A3A4A3B5A3809102
:1087B000182790911927A0911A27B0911B2786A3FB
:1087C00097A3A0A7B1A78091242790912527A091D6
:1087D0002627B091272782A793A7A4A7B5A78091A2
:1087E000282790912927A0912A27B0912B2786A787
:1087F00097A7A0ABB1AB0E94AC7A2DB73EB72E5C69
:108800003F4F0FB6F8943EBF0FBE2DBF1F910F9183
:10881000089580E380933D0F0895EF92FF92CF93E8
:10882000DF9320913D0F30E0C0E3D0E0C21BD30BBB
:108830002E5B304FB901AE010E940C7ACE01DF9160
:10884000CF91FF90EF900895AF92BF92CF92DF92B9
:10885000EF92FF920F931F93CF93DF937C01C09011
:108860003E0FD0903F0F20913D0F30E08601005D1C
:108870001F4F021B130B01381105E0F4C0E3D0E0D9
:10888000C21BD30B2E5B304FB901AE010E940C7A94
:10889000CE0DDF1D2091400F3091410F8091F40FDC
:1088A0009091F50F280F391FCE01B901A6010E9442
:1088B0000C7A02C000E010E0C801DF91CF911F9157
:1088C0000F91FF90EF90DF90CF90BF90AF90089501
:1088D00090913D0F980F90933D0F089540913E0F5A
:1088E00050913F0F9C014817590798F08091F40F61
:1088F0009091F50F820F931F9093F50F8093F40FD3
:10890000421B530B50933F0F40933E0F21E030E04A
:1089100002C020E030E0C901089590933F0F80939A
:108920003E0F08952091F40F3091F50F2E58304FDF
:10893000C901089520913D0F30E02E5B304FC901F1
:10894000089521E030E08091400F9091410F4FE079
:108950008237940711F420E030E0C90108950E94A5
:10896000A144009771F022E73FE06091400F7091C1
:10897000410F40913E0F50913F0FC9010E940C7A68
:108980000895A091F40FB091F50F1097B9F02091D0
:108990003E0F30913F0F205D3F4FAE58B04FE2E7A2
:1089A000FFE080E390E003C04D9141930196821770
:1089B0009307D4F31092F50F1092F40F089580915D
:1089C000400F9091410F089580913E0F90913F0F7D
:1089D000089590913D0F80E3891B089580E3909165
:1089E0003D0F891B20913E0F30913F0F280F311D05
:1089F000C90108951F93CF93DF93EC0110913D0FB0
:108A0000812F90E08C179D076CF00E94EE448C0F34
:108A10009D1F8138910530F41C1B10933D0F21E000
:108A200030E002C020E030E0C901DF91CF911F911A
:108A30000895CF93DF93EBECF4E21192119284E26C
:108A4000EB3FF807D1F7C0E0D0E0CE01880F991FC7
:108A50008D539B4D62E575E00E948E3B2196C4309C
:108A6000D10599F7DF91CF9108951092F50F1092EB
:108A7000F40F10923F0F10923E0F80E380933D0F52
:108A800082E79FE09093410F8093400F0E94194529
:108A900008950F931F93CF93DF93EC018B010E94F6
:108AA0003545D093410FC093400F10933F0F009373
:108AB0003E0FDF91CF911F910F910895CF92DF92DA
:108AC000EF92FF920F931F93DF93CF9300D0CDB718
:108AD000DEB78C0169837A830E94354569817A818A
:108AE000C62ED72E21E8C216D10418F030E8C32EC6
:108AF000D12C8091400F9091410FB801A6010E94A6
:108B00000C7AD0923F0FC0923E0FC6010F900F908B
:108B1000CF91DF911F910F91FF90EF90DF90CF9059
:108B20000895282F392FD901EBECF4E280E301906E
:108B30000D928150E1F7862F972FDC01E3ECF4E2F0
:108B400088E001900D928150E1F70895EBECF4E29A
:108B5000282F392FD90180E30D9001928150E1F740
:108B6000A3ECB4E2862F972FFC0188E001900D92D0
:108B70008150E1F70895E82FF0E0EE0FFF1FE55375
:108B8000FB4D7183608381E090E00895E82FF0E071
:108B9000EE0FFF1FE553FB4D80819181089590E01A
:108BA000880F991F8D569B4D0E948E3B81E090E06F
:108BB0000895282F30E0220F331F2D563B4DC90159
:108BC00008958115910511F00197F1F70895E0914D
:108BD000FE24F091FF2490818091FD248923089543
:108BE000E091FB24F091FC2480819091FD24892B5D
:108BF0008083E0910025F091012580819091FD24F2
:108C0000892B80830895E091FB24F091FC249081CE
:108C10008091FD24809589238083E0910025F09147
:108C2000012590818091FD2480958923808308957A
:108C3000FF920F931F93E091FB24F091FC2490810D
:108C40008091FD24809589238083E0910025F09117
:108C5000012580819091FD24892B80838FEB93E007
:108C60000E94E145FFB6F894E0910025F0910125BE
:108C700090818091FD2480958923808383E890E012
:108C80000E94E145E091FE24F091FF2400811091C3
:108C9000FD24FFBE78948BE393E00E94E145E091D0
:108CA000FE24F091FF2480819091FD24892319F006
:108CB000802F812301C081E01F910F91FF900895C3
:108CC00050930125409300257093FC246093FB246E
:108CD0009093FF248093FE2481E090E002C0880FEF
:108CE000991F2A95E2F78093FD240E941846089563
:108CF0000F931F93182F0FB7F894E0910025F09170
:108D0000012580819091FD24892B808383E090E070
:108D10000E94E145112351F0E0910025F0910125D9
:108D200090818091FD2480958923808387E190E064
:108D30000E94E145E091FE24F091FF248081909112
:108D4000FD24892309F410E089E590E00E94E145C3
:108D5000E0910025F091012590818091FD2480957E
:108D6000892380830FBF8BE390E00E94E145812F30
:108D70001F910F9108950F931F93182F08E0812FD3
:108D800081700E9478461695811110680150B9F7DC
:108D9000812F1F910F9108958FEF0E94BB46089578
:108DA000DF92EF92FF920F931F93CF93DF93182FD1
:108DB000EB010E941846882389F580EF0E94BB468C
:108DC000EE2400E498EFD92ED00E81E00E94784680
:108DD000F82E81E00E947846882319F0FF2069F080
:108DE00020C0FF2051F4011728F0888180FF05C0C2
:108DF000101719F0E02EFF24F3948F2D0E9478466F
:108E0000888186958883FF2011F0806888830150CF
:108E10000D15D9F6002339F02196D4CFEE24EA942B
:108E200002C08EEFE82E8E2DDF91CF911F910F9112
:108E3000FF90EF90DF9008950F931F93CF93DF93F0
:108E4000182FEB010E941846209751F085E50E94EB
:108E5000BB4608E089910E94BB460150D9F703C088
:108E60008CEC0E94BB46812F0E94BB46DF91CF91C4
:108E70001F910F9108950F931F93CF93DF93FB01E1
:108E8000DA01E801408150E0718160E0462B572B08
:108E9000803171F4BA016E7F13E0660F771F1A9567
:108EA000E1F796814CE050E0491B5109460F571FEE
:108EB00057FF06C091E09C93509541955F4F01C0CC
:108EC0001C92883289F4848190E0BC0160767070D5
:108ED0006036710549F086FF02C04E7F05C085FFF0
:108EE00002C04C7F01C0487FCA0154E09695879527
:108EF0005A95E1F7F90180834F70488380E0DF9154
:108F0000CF911F910F9108950F931F93CF93DF93EC
:108F10008C01EB01F8018081BE010E94D046F8016E
:108F2000808381508D3F28F48881883211F0803110
:108F300089F7DF91CF911F910F9108951F93CF93E0
:108F4000DF93EC010E94184684EBBE010E941C478F
:108F500081E00E947846182F0E94184681E0112374
:108F600009F480E0DF91CF911F9108951F93CF9373
:108F7000DF93182FEB010E9418460E94E7458823D3
:108F800049F084E4BE010E941C47113029F00E9480
:108F9000F04502C082E001C080E0DF91CF911F91D7
:108FA00008956F927F928F929F92AF92BF92CF92CD
:108FB000DF92EF92FF920F931F93DF93CF93CDB782
:108FC000DEB729970FB6F894DEBF0FBECDBF7C0188
:108FD0004B013A0159010E9418468EEBB7010E94DD
:108FE0001C478E010F5F1F4F8AE0C82ED12CCC0E7C
:108FF000DD1E0E94CC46F80181938F01EC15FD0522
:10900000C1F78E010F5F1F4FC80169E070E00E9439
:109010006162882351F4F7018081B801A4019301B2
:1090200085010E943B4780E001C083E029960FB68E
:10903000F894DEBF0FBECDBFCF91DF911F910F918E
:10904000FF90EF90DF90CF90BF90AF909F908F9068
:109050007F906F9008957F928F929F92AF92BF9270
:10906000CF92DF92EF92FF920F931F93DF93CF93F4
:10907000CDB7DEB729970FB6F894DEBF0FBECDBFD0
:10908000782E5B014A0179018EEB60E070E00E946E
:109090001C478E010F5F1F4F9AE0C92ED12CCC0EBA
:1090A000DD1E0E94CC46F80181938F01EC15FD0571
:1090B000C1F78E010F5F1F4FC80169E070E00E9489
:1090C0006162882349F4872DB801A50194018701C5
:1090D0000E943B4780E001C083E029960FB6F894D8
:1090E000DEBF0FBECDBFCF91DF911F910F91FF90DB
:1090F000EF90DF90CF90BF90AF909F908F907F9038
:1091000008950F931F93DF93CF93CDB7DEB72897C2
:109110000FB6F894DEBF0FBECDBF182F062FDE01AD
:109120001196E5E9F5E088E001900D928150E1F7B4
:10913000242F332727FD309541E752E0249FC001BB
:10914000259F900D349F900D112464E670E00E94DD
:109150000777AB0164E6069FB0011124460F571F45
:10916000FE013196CE010996619170E0261737070E
:1091700019F44F5F5F4F03C0E817F907A9F71123F0
:1091800019F0509541955F4FCA0128960FB6F89493
:10919000DEBF0FBECDBFCF91DF911F910F9108951C
:1091A0000F931F93DF93CF93CDB7DEB72B970FB6F7
:1091B000F894DEBF0FBECDBF182F092F885F612F37
:1091C000792F0E94B647882309F049C066E471E40C
:1091D0008FE090E00E943D49812F902FBE016F5F8C
:1091E0007F4FAE014E5F5F4F9E012D5F3F4F0E944C
:1091F000D1478823A1F5DE011496EDE8F5E088E07B
:1092000001900D928150E1F74B81642F70E021E7CE
:1092100032E0629FC001639F900D729F900D1124F8
:1092200064E670E00E9407779A8184E6989FC00107
:109230001124680F791FFE013496CE010C962191FE
:10924000421719F46F5F7F4F03C0E817F907B9F7AA
:109250008981882331F0709561957F4F02C064E366
:1092600071E2CB012B960FB6F894DEBF0FBECDBFD7
:10927000CF91DF911F910F910895DC01CB018115F2
:109280009105A105B10529F081509040A040B04062
:10929000D9F708951092B90080E28093B80008953C
:1092A00094EA9093BC0020EA36E841E050E005C023
:1092B0002150304040405040F1F09091BC0097FF69
:1092C000F7CF1DC09031B9F48093BB0084E8809340
:1092D000BC0080EA96E8A1E0B0E004C00197A109D3
:1092E000B10959F02091BC0027FFF8CF0EC081E0F2
:1092F000903421F40FC081E0089581E008959091A9
:10930000B900987F9830F1F6DFCF9091B900987F3F
:10931000983169F780E0089544EA34E824E94093FD
:10932000BC009091BC0097FFFCCF9091B900987F52
:10933000983011F0903199F78093BB003093BC00C6
:109340009091BC0097FFFCCF9091B900987F90322C
:1093500011F0983539F42093BC009091BC0094FD35
:10936000FCCFDDCF08950E945049089584E9809391
:10937000BC008091BC0084FDFCCF08958093BB00AD
:1093800084E88093BC008091BC0087FFFCCF909163
:10939000B900987F81E0983209F480E0089584EC68
:1093A0008093BC008091BC0087FFFCCF8091BB0004
:1093B000089584E88093BC008091BC0087FFFCCFB7
:1093C0008091BB000895E82FF92F80E1919190934F
:1093D0003F018150D9F780913C018F7D80933C0102
:1093E00080913C01877F80933C01862F972FFC0161
:1093F00080E1919190933E018150D9F780913C0199
:10940000806880933C0180913D0180FFFCCF4051FA
:10941000504080913C01806280933C0180913C01EE
:10942000877F80933C0114C0862F972FFC0180E139
:10943000919190933E018150D9F780913C018068D1
:1094400080933C0180913D0180FFFCCF4051504012
:10945000141615064CF3822F932FFC0180E1909196
:109460003E0191938150D9F781E090E008950F93E8
:109470001F93CF93DF938C018CE70E948C498CE77C
:109480000E94BE49C0E0D0E0F80181918F010E94A6
:10949000BE492196C031D105B9F70E94B649DF9186
:1094A000CF911F910F910895813039F48CE790E0AE
:1094B00060E070E040E050E006C08CE790E060E0E3
:1094C00070E040EC50E00E9406110895813039F4BC
:1094D0008CE790E060E070E04EE050E006C08CE782
:1094E00090E060E070E048E050E00E9406110895CE
:1094F0008CE790E060E070E041E050E00E940611EF
:109500006AE67AE080E090E00E943D4908958CE7A9
:1095100090E060E070E048E350E00E9406118CE7C4
:1095200090E060E070E049E350E00E9406118CE7B3
:1095300090E060E070E044E150E00E9406118CE7AA
:1095400090E060E070E048E750E00E9406118CE790
:1095500090E060E070E04EE550E00E9406118CE77C
:1095600090E060E070E04DE650E00E9406116CE192
:109570007AE186E090E00E943D498CE790E060E06F
:1095800070E04CE050E00E9406118CE790E060E053
:1095900070E041E050E00E9406118CE790E060E04E
:1095A00070E046E050E00E9406116AE67AE080E052
:1095B00090E00E943D490895DF93CF93CDB7DEB789
:1095C000A2970FB6F894DEBF0FBECDBFDE01119695
:1095D000EDE9F5E081E101900D928150E1F7DE01C6
:1095E0005296EEEAF5E081E101900D928150E1F7AB
:1095F0000E94874ACE0101960E94374A82E00E946B
:10960000544A6AE67AE080E090E00E943D49CE014B
:1096100042960E94374A60E17EEA88E290E00E942A
:109620003D4980E00E94664A60E17EEA88E290E07F
:109630000E943D4981E00E94664AA2960FB6F894C6
:10964000DEBF0FBECDBFCF91DF910895E6E4F1E01C
:109650008081208190813081829586958695837066
:1096600022952F70822B832B92959F70892B0895C2
:10967000DF92EF92FF920F931F93DF93CF9300D06F
:10968000CDB7DEB780E06CE046E00E940E4F89E186
:109690008093C4001092C50082E08093C00080E0F7
:1096A0000E94B84F0E943D4E84B784B784B784B7F8
:1096B00084B7E2E8FDE222E432E4318320833A9683
:1096C0008DB79EB70A97E817F907B8F300D000D016
:1096D00086EC9EE0ADB7BEB712969C938E93119721
:1096E0008FEB95E014969C938E9313970E94AC7A1F
:1096F0000F900F900F900F900E947A5E0E94483D4D
:109700008AE695E060E070E00E94FC3D0E947941AD
:10971000E0910A06F0910B0609950E94264B90E015
:109720000E94B85ECE0101960E946B4D882359F0CD
:1097300000D086EA9EE0EDB7FEB7928381830E9457
:10974000AC7A0F900F908E010F5F1F4FC8010E94DF
:10975000A93B0E94754D7C010E947A4DBC01C70156
:10976000A8010E94C5520E94D34C0E94AA520E9496
:109770007F4D0E94325400D089E99EE0ADB7BEB75C
:1097800012969C938E9311970E94AC7A00D0EDB7FD
:10979000FEB7319605E91EE0ADB7BEB712961C9331
:1097A0000E9311978A81828313820E94AC7AEDB75F
:1097B000FEB73196ADB7BEB712961C930E931197B4
:1097C0008981828313820E94AC7A0F900F9083E983
:1097D0009EE0EDB7FEB7928381830E94AC7A0F9032
:1097E0000F900E94BE5EE0918D06F0918E06099565
:1097F000E0917406F09175060995E0913606F091B6
:1098000037060995E0907206F090730600918B067A
:1098100010918C060E94A752D82E0E943A542DB760
:109820003EB72A5030400FB6F8943EBF0FBE2DBF52
:10983000EDB7FEB7319628E73EE0ADB7BEB712965A
:109840003C932E931197F382E28215830483D68290
:109850001782808711860E94AC7AE0919706F0917A
:1098600098062DB73EB7265F3F4F0FB6F8943EBF20
:109870000FBE2DBF3097D1F00995BC0100D000D0AC
:1098800085E69EE0ADB7BEB712969C938E93119776
:1098900080E890E00E94F376EDB7FEB774836383AF
:1098A0000E94AC7A0F900F900F900F9000D083E63B
:1098B0009EE0ADB7BEB712969C938E9311970E940F
:1098C000AC7A0F900F9086EB96E060E070E00E941B
:1098D000FC3D88E395E00E94645D00D08BE59EE04E
:1098E000EDB7FEB7928381830E94AC7A0F900F9000
:1098F0000F900F90CF91DF911F910F91FF90EF90FC
:10990000DF900895EF92FF920F931F9380E880936A
:109910006100109261000E94384B0E94583D0E94E5
:10992000D94F8091022590910325009729F0019746
:109930009093032580930225E0900425F09005255F
:1099400000910625109107250E947A4EE616F7062B
:109950000807190711F30E947A4E6093042570934B
:1099600005258093062590930725D7CF00D000D0FA
:1099700000D0EDB7FEB7319625E53EE0ADB7BEB7F6
:1099800012963C932E9311979383828375836483FD
:109990000E94AC7A8DB79EB706960FB6F8949EBF1C
:1099A0000FBE8DBF08950F931F93DF93CF93CDB755
:1099B000DEB7A2970FB6F894DEBF0FBECDBF8CE422
:1099C00090E00E94F67B89839A83982F9B50903178
:1099D00008F08A839A819095891709F470C000D0A5
:1099E00081E09FE0ADB7BEB712969C938E9311971E
:1099F0000E94AC7A8E010D5F1F4F0F900F90D8011F
:109A000080E090E0FC01EF51F14FE491ED9301967D
:109A100088309105B9F7F894CE0103966AE270E0B8
:109A200048E050E00E94FC7BD80180E090E0FC011F
:109A3000E751F14FE491ED9301968E309105B9F71E
:109A4000CE01039662E370E04EE050E00E94FC7BA2
:109A500080E090E0FC01E950F14FE491D801ED93F2
:109A60008D0101968A309105A9F7CE01039660E435
:109A700070E04AE050E00E94FC7B8EE490E06DECE8
:109A80007BEA0E94147C80E590E060E070E00E9438
:109A9000147C82E590E060E00E94067C8AE490E01D
:109AA00060E070E00E94147C8AE1898385EE8A83FD
:109AB00069817A818CE490E00E94147C7894898199
:109AC000A2960FB6F894DEBF0FBECDBFCF91DF9147
:109AD0001F910F910895F8946AE270E042E050E01F
:109AE0000E94DE7B789480E008958EE490E00E94EE
:109AF000F67B089580E590E00E94F67B089582E56C
:109B000090E00E94EE7B0895209110253091112560
:109B1000409112255091132590E0A0E0B0E0280F6D
:109B2000391F4A1F5B1F2093102530931125409346
:109B300012255093132520910C2530910D2540912D
:109B40000E2550910F25280F391F4A1F5B1F2093A8
:109B50000C2530930D2540930E2550930F25209111
:109B6000B0262223A1F020910825309109254091AB
:109B70000A2550910B25280F391F4A1F5B1F209380
:109B800008253093092540930A2550930B25089505
:109B90001F920F920FB60F920BB60F9211242F93B4
:109BA0003F934F935F936F937F938F939F93AF9365
:109BB000BF93EF93FF938091F60F9091F70F01966B
:109BC0009093F70F8093F60F8091F80F8F5F80933B
:109BD000F80F8091F80F8038A9F41092F80F809157
:109BE000102590911125A0911225B0911325019671
:109BF000A11DB11D8093102590931125A0931225CE
:109C0000B09313258091B0268823F1F08091F90F4D
:109C10008F5F8093F90F8091F90F8038A9F410922B
:109C2000F90F8091082590910925A0910A25B091FE
:109C30000B250196A11DB11D809308259093092540
:109C4000A0930A25B0930B250E94C340009711F002
:109C50000E94C33FFF91EF91BF91AF919F918F9170
:109C60007F916F915F914F913F912F910F900BBE1C
:109C70000F900FBE0F901F901895F8941092B60099
:109C800016BC83EF87BD82E084BD94E095BD95B39B
:109C900095BB80936E00789408952091F60F3091D3
:109CA000F70F8091F60F9091F70F28173907A9F752
:109CB000C901089507C022E330E000002150304080
:109CC000E1F701970097B9F708950F931F93CF938A
:109CD000DF938C010E944D4EEC010E944D4E8C1B77
:109CE0009D0B80179107C8F3DF91CF911F910F91C2
:109CF0000895089520911025309111254091122545
:109D0000509113258091102590911125A091122535
:109D1000B0911325281739074A075B0759F7B9018E
:109D2000CA0108951F920F920FB60F92112410923C
:109D3000E3050F900FBE0F901F9018951F920F9282
:109D40000FB60F920BB60F9211242F933F934F93A0
:109D50005F936F937F938F939F93AF93BF93EF9393
:109D6000FF93E091D905F091DA058081E091E40557
:109D7000F091E505309709F00995FF91EF91BF91BA
:109D8000AF919F918F917F916F915F914F913F9193
:109D90002F910F900BBE0F900FBE0F901F90189534
:109DA0001F920F920FB60F9211241092F0050F9090
:109DB0000FBE0F901F9018951F920F920FB60F9223
:109DC0000BB60F9211242F933F934F935F936F9392
:109DD0007F938F939F93AF93BF93EF93FF93E09104
:109DE000E605F091E7058081E091F105F091F2053B
:109DF000309709F00995FF91EF91BF91AF919F9135
:109E00008F917F916F915F914F913F912F910F9023
:109E10000BBE0F900FBE0F901F90189590E02DE095
:109E200030E0829FF001839FF00D929FF00D11248E
:109E3000E752FA4FA281B3811C92A481B5816C9341
:109E4000A681B78188ED8C93A085B1854C9312864D
:109E500014861386089590E02DE030E0829FF00193
:109E6000839FF00D929FF00D1124E752FA4F81E08D
:109E70008287A081B1816C933A9680818823E9F72B
:109E800008951F93182F8A3031F48091FA0F6DE0F6
:109E90000E942B4F02C08D3029F08091FA0F612F64
:109EA0000E942B4F80E090E01F910895EF92FF9267
:109EB0001F93CF93DF93182FE62EE7017E01F72E35
:109EC000E7010CC08A3021F4812F6DE00E942B4FF6
:109ED00069916D3019F0812F0E942B4F8881882362
:109EE00089F7DF91CF911F91FF90EF9008950F9325
:109EF0001F93DF93CF93CDB7DEB7FE013A960BEFFA
:109F00001FE0C80160E470E0488559859F010E9408
:109F1000487B8F81B8010E94564FCF91DF911F91EE
:109F20000F9108951F93CF93DF93182FEB0104C077
:109F3000812F0E942B4F2196FE0164916623C1F769
:109F4000DF91CF911F91089590E02DE030E0829F46
:109F5000F001839FF00D929FF00D1124E752FA4F0C
:109F6000748763870895682F80E00E942B4F0895BF
:109F70008093FA0F8BEC95E090937D2D80937C2D50
:109F8000089584B7877F84BF88E10FB6F8948093E3
:109F90006000109260000FBE08952FE088E190E00D
:109FA0000FB6F894A895809360000FBE20936000D0
:109FB0000895A895089588E10FB6F89480936000FD
:109FC000109260000FBE0895F89428E088E190E0B8
:109FD0000FB6F894A895809360000FBE20936000A0
:109FE000FFCF8091232590E0FC01EE0FFF1F969597
:109FF000982F882797958795E80FF91FEC5DFA4D04
:10A000001082089580911B2580911B2590E0089572
:10A010008091390181FD0CC081E491E06FE140E065
:10A020000E94DB55813039F021E030E0813129F0A8
:10A0300020E030E002C021E030E0C90108958091C5
:10A04000390181FD12C081E491E06FE140E00E949E
:10A05000DB55982F8151823050F09F3141F0913083
:10A0600041F081E0923031F402C081E0089580E057
:10A07000089580E008950E941F508823E1F3089519
:10A0800081E491E06FE140E00E94DB550895E9E34F
:10A09000F1E0808180818D7F80838DE090E0019769
:10A0A000F1F782E491E06FE140E023E00E94E555A2
:10A0B00083E090E00197F1F708950E943B501092E1
:10A0C000B0260E9447508091390182608093390107
:10A0D000809133278823E9F1809194009091950035
:10A0E000209144273091452782179307A0F480914F
:10A0F000102790911127A0911227B09113278C5708
:10A10000914EAF4FBF4F8093102790931127A0938C
:10A110001227B09313278091940090919500821B91
:10A12000930BA0E0B0E020911027309111274091CF
:10A13000122750911327820F931FA41FB51F8093DE
:10A14000102790931127A0931227B09313271092F2
:10A150003327809135278823E9F1809194009091ED
:10A160009500209148273091492782179307A0F442
:10A170008091182790911927A0911A27B0911B2739
:10A180008C57914EAF4FBF4F80931827909319274C
:10A19000A0931A27B0931B2780919400909195006B
:10A1A000821B930BA0E0B0E0209118273091192773
:10A1B00040911A2750911B27820F931FA41FB51F90
:10A1C0008093182790931927A0931A27B0931B27E1
:10A1D0001092352708958091B026882381F08091D0
:10A1E0003B10882321F40E941F50882331F481E022
:10A1F0008093BE1021E030E004C00E945D5020E05A
:10A2000030E0C90108950F931F93182F883049F04B
:10A21000863039F0893029F0863119F0893109F01A
:10A2200041C08091390181FD40C00E943B500E9495
:10A230004050082F181709F43BC0183019F40E9439
:10A24000475029C0193141F48631A9F482E491E0E4
:10A250006FE140E029E009C0163169F4893159F411
:10A2600082E491E06FE140E026E00E94E555E3E002
:10A27000F0E03197F1F782E491E06FE140E0212FC7
:10A280000E94E555083019F4E9E6F1E002C0E3E088
:10A29000F0E03197F1F70E944050811749F023E434
:10A2A00030E008C022E430E005C024E430E002C021
:10A2B00020E430E0C9011F910F910895809194002E
:10A2C00090919500909349278093482721E020930F
:10A2D00035278091390181FF15C02093AF268091E9
:10A2E0009400909195009093452780934427209364
:10A2F0003327809139018D7F809339018091AF267A
:10A300008823E1F786E10E94035181E08093B02623
:10A3100008958091B026882351F480913B108823C2
:10A3200021F081E08093BD1002C00E945E5181E067
:10A3300090E008951F93DF93CF930F92CDB7DEB7D0
:10A340008FB7898380913B10882331F5F8948091F1
:10A35000B026882351F08091390181FD1BC00E94F5
:10A360001F508823B9F080E003C00E94895181E02A
:10A37000909147019E3010F010E001C01FEF88233C
:10A3800011F00E94EB5016FF05C089818FBF21E0BC
:10A3900030E004C089818FBF20E030E0C9010F9018
:10A3A000CF91DF911F9108958091BD10882321F0F6
:10A3B0000E945E511092BD108091BE10882321F042
:10A3C0000E945D501092BE1010923B100895EF92C3
:10A3D000FF92CF93DF93B82FA92FF62FE72F81E0BD
:10A3E00080933B102091F4263091F5264091F6267B
:10A3F0005091F7262F5F3F4F4F4F5F4F2093F4262A
:10A400003093F5264093F6265093F726862F8E5FDD
:10A4100087FF0CC08091AD269091AE260196909357
:10A42000AE268093AD26CFEFDFEF0BC02CE330E1FB
:10A43000C9016B2F7A2F4F2F5E2F0E940C7AC0E03C
:10A44000D0E00E94D451CE01DF91CF91FF90EF90E8
:10A4500008959091390191FD0AC0282F803108F0AC
:10A460002FE085E491E06FE040E00E94E55508951B
:10A470008093C01008950E9440508250813130F482
:10A48000E82FF0E0E25EF94F8081089581E00895C1
:10A4900008958FEF80934E018CE691E060EF44E0E9
:10A4A00022E00E94E5558CE290E06EE041E025E07C
:10A4B0000E94E55580E880936F018091460180936A
:10A4C0006D0184E491E060E245E021E00E94E55501
:10A4D0000895CF93DF93CDEFD3E0CE010197F1F74D
:10A4E0000E94D155109224251092A625109228265C
:10A4F0001092232510922225E9E3F1E080818E7FDE
:10A50000808380818D7F80838DE090E00197F1F7DB
:10A5100080818160808382E491E06FE140E023E00C
:10A520000E94E5552197F1F780915D0180915E01D0
:10A530000E94495280E096E060E070E00E94FC3D9D
:10A540000E945E5181E090E0DF91CF91089580916B
:10A55000BF100895DF93CF930F92CDB7DEB78983F5
:10A560000E943B5029812093BF1088E491E06FE165
:10A5700040E00E94E5550F90CF91DF9108950E9431
:10A58000AA5286E00E94035108958093620190933D
:10A59000630160936001709361014115510531F1D0
:10A5A000FA01819180936B01DA0111968C9180936D
:10A5B0006A01DF011196818180936901FD01319665
:10A5C00011968C9180936801DF01119681818093AF
:10A5D0006701FD01319611968C9111978093660168
:10A5E000818180936501828180936401089580E078
:10A5F00096E00E941F3E81E080931B2580911C25E0
:10A6000090911D25019690931D2580931C2581E036
:10A6100090E00895EF92FF92CF93DF93509123251E
:10A62000252F30E0F901EE0FFF1F3695322F22273C
:10A6300037952795E20FF31FEC5DFA4D40814423D7
:10A6400009F4CEC02091390121FDCAC02091B02665
:10A65000222309F4C5C047FF16C00E94F14F809124
:10A66000E4269091E526A091E626B091E726019692
:10A67000A11DB11D8093E4269093E526A093E626C4
:10A68000B093E726ADC04330B0F40E94F14F809103
:10A69000E0269091E126A091E226B091E326019672
:10A6A000A11DB11D8093E0269093E126A093E226A0
:10A6B000B093E32695C0C42FD0E022976C177D0796
:10A6C000B0F40E94F14F8091DC269091DD26A0919C
:10A6D000DE26B091DF260196A11DB11D8093DC26F8
:10A6E0009093DD26A093DE26B093DF2679C0652FF8
:10A6F00070E09B01220F331F7695762F66277795A2
:10A700006795260F371F2B5D3A4DB90150E00E9427
:10A710000C7A20912325822F90E0FC01EE0FFF1F81
:10A720009695982F882797958795E80FF91FEC55F0
:10A73000FA4D808180931425822F90E0FC01EE0F6A
:10A74000FF1F9695982F882797958795E80FF91FF3
:10A75000EC5DFA4D10822F5F20932325233010F0FB
:10A76000109223258091232590E0FC01EE0FFF1F1E
:10A770009695982F882797958795E80FF91FEC5D98
:10A78000FA4D8081882311F00E94F75260914701B1
:10A790006093152580911A25882311F0681710F40D
:10A7A00060931A2584E070E00E94BB4560911425F7
:10A7B00083E070E00E94BB458091F8269091F926D5
:10A7C000A091FA26B091FB260196A11DB11D8093A0
:10A7D000F8269093F926A093FA26B093FB2602C0A0
:10A7E000C0E0D0E0CE01DF91CF91FF90EF900895CF
:10A7F000CF93DF93EC0188819981009729F024E0C1
:10A800008B3F920739F505C08BEF94E099838883DD
:10A8100025C0623819F510921B250E9435450E940B
:10A82000924460E870E00E940A531816190644F436
:10A830000E948D44E0919106F09192060995E4CF33
:10A840008091182590911925019690931925809350
:10A850001825DACF1982188283E001C081E0DF91E8
:10A86000CF91089591E090933B100E9429520E944D
:10A87000D45108958091390181FD07C085E491E0AC
:10A880006FE040E00E94DB55089580E10895CF928B
:10A89000DF92EF92FF920F931F93CF93DF93182FC6
:10A8A00021E020933B100091B0268091390181FF77
:10A8B00016C08091940090919500909345278093C5
:10A8C0004427209333272093AF26809139018D7F31
:10A8D000809339018091AF268823E1F700E00E9440
:10A8E0003B508091B026882309F441C080913527E0
:10A8F0008823E9F1209194003091950080914827B8
:10A900009091492728173907A0F4209118273091F2
:10A91000192740911A2750911B272C57314E4F4F22
:10A920005F4F209318273093192740931A2750938D
:10A930001B272091940030919500281B390B40E093
:10A9400050E0C0901827D0901927E0901A27F09077
:10A950001B272C0D3D1D4E1D5F1D20931827309386
:10A96000192740931A2750931B271092352789E106
:10A970000E94035186E00E94C645009751F00E9454
:10A980003A54C82F86E00E94C64581500E94295241
:10A9900002C0C0E0D0E08091940090919500909327
:10A9A00047278093462781E080933427F89480914D
:10A9B0003901826080933901809139018D7F8093C4
:10A9C0003901612F6E5F8CE390E10E9416567894F6
:10A9D0008091AA269091AB2601969093AB26809306
:10A9E000AA260E943B5082E491E060EE45E00E947E
:10A9F000DB55182F86E00E94C645009719F08C2F72
:10AA00000E942952002319F00E945E5102C00E9448
:10AA10005D50809134278823E9F1809194009091D2
:10AA20009500409146275091472784179507A0F439
:10AA30008091142790911527A0911627B091172780
:10AA40008C57914EAF4FBF4F80931427909315278B
:10AA5000A0931627B093172720919400309195006A
:10AA6000241B350B40E050E080911427909115276E
:10AA7000A0911627B0911727280F391F4A1F5B1F77
:10AA800020931427309315274093162750931727A8
:10AA9000109234278091B026882361F08091940031
:10AAA00090919500909349278093482781E0809367
:10AAB000352707C082E491E06FE140E023E00E9487
:10AAC000E5550E94D4511130E1F01330A9F4809182
:10AAD000EC269091ED26A091EE26B091EF260196FE
:10AAE000A11DB11D8093EC269093ED26A093EE2638
:10AAF000B093EF2612E00AC0153029F0173031F478
:10AB000004C010E003C013E001C011E0812F90E009
:10AB1000DF91CF911F910F91FF90EF90DF90CF9039
:10AB20000895CF93DF93EB010E94E7519C010097BA
:10AB300031F4CE010E9447549C01009749F0809166
:10AB4000AD269091AE2601969093AE268093AD26C9
:10AB5000C901DF91CF9108950F931F938091B02683
:10AB6000882321F40E94895111E001C010E00E9465
:10AB70004050863111F0813119F40091470109C02C
:10AB800086E491E06FE140E00E94DB55082F000F62
:10AB9000080F112311F00E94EB50802F1F910F918D
:10ABA00008951092C2101092C110EFE6F0E080817B
:10ABB000806280830895FC018081862390E002C03A
:10ABC000959587954A95E2F70895F894FC01908150
:10ABD000862F8095892330E002C0220F331F4A95CB
:10ABE000E2F72623282B208378940895DC01119620
:10ABF00020917B01FC012083215030E0A9014F57B7
:10AC00005E4FE0E8F1E061916D93E417F507D9F745
:10AC1000FC01E058FF4F2F573E4FD9012C91208364
:10AC20008F579F4F21E0FC0120830895FC01609322
:10AC3000800101966350860F911DA1E8B1E021913A
:10AC40002D93E817F907D9F708951F920F920FB6C1
:10AC50000F920BB60F9211242F933F934F935F9354
:10AC60006F937F938F939F93AF93BF93EF93FF93D4
:10AC700080914701809315252091222530E0C9015C
:10AC8000880F991F3695322F222737952795820FE7
:10AC9000931F8C5D9A4D0E94F655809122258F5FFF
:10ACA00080932225833010F0109222250E94F752C3
:10ACB000FF91EF91BF91AF919F918F917F916F9194
:10ACC0005F914F913F912F910F900BBE0F900FBE50
:10ACD0000F901F9018951F920F920FB60F9211248C
:10ACE0000F900FBE0F901F9018951F920F920FB6E6
:10ACF0000F9211240F900FBE0F901F9018951F9266
:10AD00000F920FB60F9211240F900FBE0F901F904D
:10AD100018951F920F920FB60F9211241092AF2622
:10AD20000F900FBE0F901F9018951F920F920FB6A5
:10AD30000F9211241092AF260F900FBE0F901F900C
:10AD400018951F920F920FB60F9211248F9381E0E6
:10AD500080931B258F910F900FBE0F901F90189519
:10AD60001F920F920FB60F9211241092AF260F90E0
:10AD70000FBE0F901F9018951F920F920FB60F9253
:10AD800011248F939F938091C1109091C2100196CE
:10AD90009093C2108093C1109F918F910F900FBE1E
:10ADA0000F901F9018950F931F93CF93DF9380916F
:10ADB000B8269091B926A091BA26B091BB260196EB
:10ADC000A11DB11D8093B8269093B926A093BA26F1
:10ADD000B093BB260E948459EC0183EC90E10E9461
:10ADE000C13E0BC0D8011296ED91FC91139730979C
:10ADF00009F00995C8010E94873F082F192F0115F6
:10AE0000110581F7209719F0CE010E94313CDF91A6
:10AE1000CF911F910F9108950E94BE5E0E9435450B
:10AE20000E948E5782E796E09093B3268093B226D5
:10AE30000E94815982E090E060E074E040E05EE1D1
:10AE40002FEF31E00E9442590895CF92DF92EF92A6
:10AE5000FF920F931F93CF93DF936C01EB018A0155
:10AE600083EC90E10E94C13E0CC0D7011496ED9195
:10AE7000FC911597309711F0CE010995C7010E94FA
:10AE8000873FE82EF92EE114F10479F7C601BE01DF
:10AE9000A8010E94393CDF91CF911F910F91FF9043
:10AEA000EF90DF90CF900895BC0183EC90E10E9479
:10AEB000483F0895BC0183EC90E10E940F3F089544
:10AEC000CF93DF93EC018091B4269091B526A091A9
:10AED000B626B091B7260196A11DB11D8093B42668
:10AEE0009093B526A093B626B093B726CE010E94C4
:10AEF0009B59009769F00E94AF44E0917606F0916B
:10AF0000770685E297E5BE01099521E030E002C0B1
:10AF100020E030E0C901DF91CF91089585EC90E108
:10AF20000E94BD3E08950F93CF93DF93EC017B8386
:10AF30006A8318865F834E8385EC90E1BE010E9490
:10AF4000483FE091C710F091C810309749F04C810C
:10AF50005D818A819B81688520E030E001E0099570
:10AF6000DF91CF910F910895BC0185EC90E10E9493
:10AF70000F3F08950F93DC0118961C921897E091EB
:10AF8000C710F091C810309759F012968D919C918E
:10AF9000139760E040E050E020E030E000E00995E9
:10AFA0000F9108950F93DC01AB0114962D913C9104
:10AFB000159781E018968C93189715967C936E934D
:10AFC0001497E091C710F091C810309739F012969D
:10AFD0008D919C91139761E000E009950F91089580
:10AFE0000F93DC01E091C710F091C810309769F021
:10AFF00014962D913C91159712968D919C911397D3
:10B0000018966C91A90101E009950F910895E091BE
:10B01000C910F091CA10309709F0099508959093DE
:10B02000CA108093C91008959093C8108093C710D8
:10B03000089585EC90E10E94C13E0895EF92FF9241
:10B040000F931F93CF93DF938C01EB017A0185EC73
:10B0500090E10E94C13E15C0DC0112962D913C91F9
:10B0600013972C173D0759F41696ED91FC911797FD
:10B07000309761F0B801AE019701099507C00E94B1
:10B08000873F282F392FC901009731F7DF91CF91E2
:10B090001F910F91FF90EF9008950895AF92BF9286
:10B0A000CF92DF92EF92FF920F931F93DF93CF9394
:10B0B00000D0CDB7DEB75B010E949244FC01008155
:10B0C00011811A8309830C30110518F4EE24FF2432
:10B0D0002EC000D000D08AE396E0EDB7FEB7928391
:10B0E0008183148303830E949A7A0F900F900F90AC
:10B0F0000F9020C00E949244F701EE0FFF1FEE0F49
:10B10000FF1FE80FF91FC280D3800E949244089469
:10B11000E11CF11CF701EE0FFF1FEE0FFF1FE80F00
:10B12000F91F40815181C501B6010E941E58E016E9
:10B13000F10600F30F900F90CF91DF911F910F91C7
:10B14000FF90EF90DF90CF90BF90AF900895CF9396
:10B15000DF93C6EED0E16091FC107091FD10CE013E
:10B1600049ED58E520E030E00E9486410E94BB5E38
:10B170006091FC107091FD100E94F376BC01CE012D
:10B1800040974EEE58E520E030E00E948641DF9186
:10B19000CF9108950F93013051F48091F610909162
:10B1A000F7109093FD108093FC100E94A7580F9108
:10B1B00008958091FC109091FD102091FA1030912B
:10B1C000FB10880F991F2817390708F4C9019093BD
:10B1D000FD108093FC100E94A7580895EF92FF92F3
:10B1E000CF93DF930E9435450E949244E82EE701F9
:10B1F0007E01F92EE701198218820E94195826C093
:10B2000028813981F901EE0FFF1FEE0FFF1FEC0FB0
:10B21000FD1FDC0112964D915C911397538342837D
:10B220002F5F3F4FF901EE0FFF1FEE0FFF1FEC0FD7
:10B23000FD1F14964D915C9115975183408339837E
:10B2400028830E94873F282F392FC901009721F0BA
:10B25000FC0120852223A1F688819981880F991FFE
:10B26000880F991F02960E948D44888199810097CA
:10B2700021F08BEC90E10E94043CDF91CF91FF9094
:10B28000EF900895EF92FF920F931F93CF93DF9368
:10B29000FC018B017A01E9018BEC90E1BF0147E5EC
:10B2A00056E00E94E63B1093F7100093F610F092E0
:10B2B000F910E092F810D093FB10C093FA108AECCA
:10B2C00098E50E941458DF91CF911F910F91FF9044
:10B2D000EF900895CF93DF93C6EED0E1CE010E94A8
:10B2E0000D42CE0140970E940D42CE014B970E9425
:10B2F000013CDF91CF9108958091FC109091FD1059
:10B3000008950E94453C0895EF92FF92CF93DF93FA
:10B31000E0915B06F0915C060995EC01009729F03D
:10B320006A817B8181E00E94BB45CE01DF91CF9194
:10B33000FF90EF9008950F931F93CF93DF938C01AD
:10B34000E0915D06F0915E060995EC01F8016281DD
:10B35000738181E00E94BB4521E030E0209711F429
:10B3600020E030E0C901DF91CF911F910F91089546
:10B37000E0915F06F091600609950895FC0120E0D8
:10B3800030E004C08181280F311D329680818823EE
:10B39000C9F7C9010895FC01818190E0308120E066
:10B3A000822B932B02C0880F991F6A95E2F7892F91
:10B3B0009927FA01EF59F94F208130E08223932336
:10B3C00028E030E0241B350B02C0969587952A951E
:10B3D000E2F708956F927F928F929F92AF92BF9201
:10B3E000CF92DF92EF92FF920F931F93CF93DF9351
:10B3F0006C017B015A0189012830310544F4CB01ED
:10B40000BA01A9010E94CB59F601808341C03901DC
:10B4100033E0759467943A95E1F74115510521F0B1
:10B420004C01C0E0D0E016C0DB01FC01C0E0D0E080
:10B430008D9181932196C615D705D4F3A801477045
:10B4400050704115510521F1C7018C0F9D1F60E01F
:10B4500070E019C0C7018C0F9D1FB50148E050E096
:10B460000E94CB59F40181934F012196C615D7054F
:10B470008CF3A801477050704115510549F0C70180
:10B480008C0F9D1FB5010E94CB59CC0DDD1D88830B
:10B49000DF91CF911F910F91FF90EF90DF90CF90B0
:10B4A000BF90AF909F908F907F906F9008954F9234
:10B4B0005F926F927F928F929F92AF92BF92CF9244
:10B4C000DF92EF92FF920F931F93DF93CF9300D001
:10B4D00000D0CDB7DEB70E949244E82E092F82E05B
:10B4E00090E00E946E44009709F464C0EE2DF02FA6
:10B4F000918180E02081820F911D0E94593C7C0146
:10B50000009709F459C00E9492443C01F70146811A
:10B51000242F30E02770307081E090E02115310554
:10B5200011F480E090E0469546954695840F911D74
:10B530000E946E440097F1F1F70104811581CC243B
:10B54000DD2453E0452E512C4C0E5D1E4E01089417
:10B55000811C911C2AC0F801A180BB24B60143E0E4
:10B56000759567954A95E1F7660D771DA6014770B9
:10B570005070883150F0C40195010E94EA59F801D9
:10B580008081B4010E94CF450CC01C821B82C20185
:10B5900095010E94EA596B817C81F80180810E94AB
:10B5A000BB45CA0CDB1C0E5F1F4FF801808188234E
:10B5B00091F602C0EE24FF24C7010F900F900F9068
:10B5C0000F90CF91DF911F910F91FF90EF90DF903F
:10B5D000CF90BF90AF909F908F907F906F905F9033
:10B5E0004F900895FC0150E080E190E0861B970B9E
:10B5F000821B930B02C0440F551F8A95E2F780818E
:10B60000852B80838181842B818308956F927F9223
:10B610008F929F92AF92BF92CF92DF92EF92FF9262
:10B620000F931F93CF93DF938C015B016A01790124
:10B630002830310524F4C801FA01408156C039018F
:10B6400063E0759467946A95E1F7A114B10421F061
:10B650004A01C0E0D0E021C0DA01F80180E090E0CA
:10B660002D912193019686159705D4F397012770A4
:10B67000307021153105D9F1F601E80FF91F40812D
:10B6800050E068E070E0621B730B02C0559547956F
:10B690006A95E2F7800F911F26C0F40141914F0196
:10B6A000C8018C0F9D1FB50128E030E00E94F25ABE
:10B6B0002196C615D7058CF3970127703070211598
:10B6C0003105A9F0F601EC0FFD1F408150E0C501E6
:10B6D0000896821B930B02C0559547958A95E2F711
:10B6E000C8018C0F9D1F60E070E00E94F25ADF914C
:10B6F000CF911F910F91FF90EF90DF90CF90BF906F
:10B70000AF909F908F907F906F9008954F925F922F
:10B710006F927F928F929F92AF92BF92CF92DF9261
:10B72000EF92FF920F931F93DF93CF9300D0CDB78B
:10B73000DEB78C01DC0116964C911697842F90E0B1
:10B740008770907021E030E0009711F420E030E045
:10B750004695469546957901E40EF11CC70102967F
:10B760000E94FA44009709F453C00E949A44FC01D5
:10B77000D80112968C911297808313968C918183B5
:10B780000E949A44F2E06F2E712C680E791EC3015C
:10B7900060E070E0A7010E94157AF801C480D580AE
:10B7A00000E010E02E010894411C511C2AC0D60173
:10B7B00011968C90119799247801E3E0F594E79421
:10B7C000EA95E1F7E60CF71C77E0A72EB12CA02252
:10B7D000B122883130F00E94D945AC01C701B501D2
:10B7E00007C00E94C6459A838983C701B501A2019B
:10B7F00094010E94065B080D191DE2E0F0E0CE0EF8
:10B80000DF1ED6018C91882391F621E030E002C042
:10B8100020E030E0C9010F900F90CF91DF911F9190
:10B820000F91FF90EF90DF90CF90BF90AF909F90DF
:10B830008F907F906F905F904F900895E0918F066A
:10B84000F091900609950895E0913806F091390637
:10B8500009950895E0919306F0919406099508954D
:10B86000E0919506F09196060995089580E090E0A4
:10B8700008950895E0911A06F0911B060995089520
:10B88000009731F0E0911A06F0911B060995089592
:10B89000E0911C06F0911D060995089580E090E066
:10B8A00008950F931F93DF93CF93CDB7DEB7E09743
:10B8B0000FB6F894DEBF0FBECDBF0E94E4448C01EA
:10B8C0000E949244602FAE014F5F5F4F0E948464DC
:10B8D000882309F445C088A99801281B3109C901AA
:10B8E0000E946E440097E1F12E81222371F18A8536
:10B8F0009B853BEA8D3C930721F03FEF8F3F9307F9
:10B9000079F5223041F088E090E007C0019722915C
:10B910002F3F41F00BC082E090E0FE01E80FF91FDD
:10B920003C96F4CF181619068CF30FC089E1BE01BE
:10B93000645F7F4F0E94CF4589E10E94D94561EC49
:10B9400074E20E94973B009759F088E1BE016A5E5D
:10B950007F4F0E94CF45E0917806F09179060995D6
:10B96000E0960FB6F894DEBF0FBECDBFCF91DF914A
:10B970001F910F910895AF92BF92CF92DF92EF92F5
:10B98000FF920F931F93DF93CF93CDB7DEB7E0976E
:10B990000FB6F894DEBF0FBECDBF6C018B01FE0168
:10B9A000319680E3DF011D928A95E9F781E0898372
:10B9B0008CE00E94C6458C831D821F8280910011FD
:10B9C00089878F5F8093001183E0E82EE8868DECF5
:10B9D0009BEA9B878A8789E10E94D94562E575E0E9
:10B9E0000E94973B009731F082E08E838FEF8C8727
:10B9F0008D8709C089E10E94D945BC01CE010C9612
:10BA00000E948E3BEE828DEC9BEA9D8B8C8BCE014F
:10BA1000469661EC74E20E948E3B0E9492449FA77E
:10BA20008EA70E94E44488AB7E010894E11CF11CBF
:10BA3000C7010E947B63A82E90E00E94FA44009701
:10BA400041F10E949A44BC01C7014A2D0E949963AA
:10BA5000A0901006B09011060E949A447C010E94AA
:10BA6000EE44BC01C701F5010995C114D10489F068
:10BA7000009721F08130910561F404C0C80160E0B5
:10BA800070E003C0C80164E070E041E050E0F601FE
:10BA90000995E0960FB6F894DEBF0FBECDBFCF91EB
:10BAA000DF911F910F91FF90EF90DF90CF90BF90AB
:10BAB000AF9008950E94BB5E80930011E0911A063A
:10BAC000F0911B0609950895EF92FF92CF93DF93B3
:10BAD000E82EE7017E01F92EE70104C060E070E086
:10BAE0000E94FC3D899199910097C1F7DF91CF9118
:10BAF000FF90EF900895EF92FF92CF93DF93E82E9F
:10BB0000E7017E01F92EE70102C00E94413D8991C3
:10BB100099910097D1F7DF91CF91FF90EF90089521
:10BB2000CF93DF93EC017B836A830E944D4E998310
:10BB30008883DF91CF910895FC01808191812281DA
:10BB40003381820F931F918380830895CF93DF9376
:10BB5000EC010E944D4E99838883DF91CF91089527
:10BB6000CF93DF93EC010E944D4E28813981821BD7
:10BB7000930B019621E030E04A815B814817590719
:10BB800010F020E030E0C901DF91CF910895EF92ED
:10BB9000FF92CF93DF93FC01C281D3818081918199
:10BBA000C80FD91F0E944D4EC81BD90BCE01DF9183
:10BBB000CF91FF90EF900895CF93DF93EAE3F7E200
:10BBC000CCEFD6E2AEE2B7E211921192199219923D
:10BBD000199219921D9287E2E235F807A9F7DF91D1
:10BBE000CF9108950F931F93CF93DF93FC01DC0156
:10BBF000A25DB84D8C91882339F100919400109189
:10BC00009500EF01CC0FDD1FCC0FDD1FC450D94DC7
:10BC1000DF01AA0FBB1FA65CB84D8D919C911197B7
:10BC20009801281B390B40E050E0688179818A81B6
:10BC30009B81260F371F481F591F288339834A834A
:10BC40005B8311961C930E93EE0FFF1FEE0FFF1FE9
:10BC5000E450F94D6081718182819381DF91CF91B0
:10BC60001F910F91089560E070E0CB010895FC01F1
:10BC7000EE0FFF1FEE0FFF1FE450F94D408351837D
:10BC8000628373830895EF92FF920F931F93CF9374
:10BC9000DF932EE237E2CCEFD6E2EAE3F7E2D90116
:10BCA0008D919D018823C9F0409194005091950099
:10BCB000808191817A01E81AF90A00E010E0888118
:10BCC0009981AA81BB818E0D9F1DA01FB11F888302
:10BCD0009983AA83BB835183408324963296B7E22B
:10BCE0002A333B07E1F6DF91CF911F910F91FF902F
:10BCF000EF9008950E94F86208950F931F93FC013E
:10BD0000CB0140910111509102113383228315839D
:10BD1000048371836083F0930211E0930111411554
:10BD2000510511F40E94126380E090E01F910F9181
:10BD3000089580910111909102110097C1F0109225
:10BD4000021110920111DC0114966D917C911597EE
:10BD50001296ED91FC9113970995E0910111F091E4
:10BD60000211309721F0808191810E941263089521
:10BD70000E94E17708950E94DC77089589E996E0B2
:10BD80000E94353E81EA96E00E94353E0895EF928A
:10BD9000FF92CF93DF930E94A1440097C9F081EAFC
:10BDA00096E00E94553EE82EE7017E01F92EE7015C
:10BDB000209731F10E94E444998388830E94DF44F4
:10BDC0009B838A83C70104960E940D448CAB18C0E4
:10BDD00089E996E00E94553EEC017E01F92EE701CB
:10BDE000209771F0C70102960E94244499838883AA
:10BDF000B7016E547F4FC7018E579F4F0E949145E8
:10BE0000CE01DF91CF91FF90EF900895BC016E5469
:10BE10007F4F8E579F4F0E9491450895CF93DF9398
:10BE2000EC0189E996E0BE010E94A03E009719F05E
:10BE300089E996E009C081EA96E0BE010E94A03E31
:10BE4000009729F081EA96E0BE010E947B3EDF91D7
:10BE5000CF910895EF92FF92CF93DF93EC0189E9A0
:10BE600096E0BE010E94A03E009779F0688179813A
:10BE7000CE0102960E945E45BE016E547F4FCE01F8
:10BE80008E579F4F0E94A6451BC081EA96E0BE01D7
:10BE90000E94A03E0097A1F00E94354568817981FB
:10BEA0008A819B810E945E458CA990E00E94FA44A1
:10BEB0000E949A444CA92496BE0150E00E940C7A3C
:10BEC000DF91CF91FF90EF900895EF92FF92CF9383
:10BED000DF93EC0189E996E0BE010E94A03E009745
:10BEE00011F022960DC081EA96E0BE010E94A03EAC
:10BEF000009721F00A80DB81C02D02C0C0E0D0E0B5
:10BF0000CE01DF91CF91FF90EF900895FC018081E9
:10BF10009181089570E06F5B7F4F660F771F680F08
:10BF2000791FCB010895E62FF0E0EF5BFF4FEE0F96
:10BF3000FF1FE80FF91F808191810895089589E519
:10BF400097E10E94AB40009721F089E597E10E94BC
:10BF500096400895E0916617F0916717309711F0B9
:10BF60000995089580E00895EF92FF920F931F9333
:10BF7000CF93DF93EC018A0188819981009731F09A
:10BF800023E08C30920709F006C12BC080E00BC083
:10BF9000E82FF0E0EE0FFF1FEE0FFF1FE95BF84EFA
:10BFA000118210828F5F843098F3809361178091A3
:10BFB000880E9091890E90935817809357170E947E
:10BFC0003A3D8093522789E597E160E470E00E9452
:10BFD00080400E9413668CE093E09983888381E01F
:10BFE000DDC0623009F4B9C0633030F4662309F46F
:10BFF00089C0613081F79CC0673819F0683859F7FB
:10C0000041C01092621747E4E42E47E1F42E18C0B5
:10C01000F701828193818017910749F48081918192
:10C020000E945A67F701118210821382128284E003
:10C0300090E0E80EF91E809162178F5F809362177F
:10C0400080916217843020F3E2E6FCE2848D958DC6
:10C050008017910719F4158E148E118EB0969CE2FC
:10C06000E23EF90799F7E8EFFCE2818592858017B7
:10C07000910711F4158214823D962DE2EA37F207FA
:10C08000A1F7A9CF87E14935580709F0A4CFCA0124
:10C090000E94AB40009709F49ECF109262172DC00A
:10C0A000F0E035E0EE0FFF1F3A95E1F7EE59F34D62
:10C0B000818D8823E9F089E597E10E94964080917F
:10C0C000621790E025E0880F991F2A95E1F78E59B5
:10C0D000934D9093612C8093602C82E00E948E6738
:10C0E0008091532790915427009711F00E94AA5FE6
:10C0F000809162178F5F80936217E0916217E4303E
:10C1000078F269CF4115510509F465CF5093612C40
:10C110004093602C83E00E948E678091532790911A
:10C120005427009711F00E94AA5F0E949F5F53CF8F
:10C130004115510509F44FCF50935D2C40935C2C71
:10C1400085E00E948E678091532790915427009735
:10C1500009F441CF0E94AA5F3ECF8091532790916E
:10C160005427009709F437CF80916427863031F443
:10C1700080917C2781FF02C00E949F5F81E00E9426
:10C180008E678091532790915427009709F423CF0D
:10C190000E94DD6120CF1982188283E0DF91CF9168
:10C1A0001F910F91FF90EF900895909367178093E0
:10C1B000661708952091880E3091890E60E0E7E4BB
:10C1C000F7E113C0408151814817590761F442815A
:10C1D00053814217530739F4609365171182108217
:10C1E0000E945A67089534966F5F643058F36093E5
:10C1F0006517089540E0E7E4F7E116C0542F5F5F4C
:10C20000208131812115310569F4409364179183B0
:10C2100080832091880E3091890E338322830E947F
:10C22000746708953496452F443040F34093641763
:10C230000895FC018091880E9091890E958F848FCE
:10C24000778F668F0895FC018091880E9091890EFA
:10C2500092878187748763870895CF93DF93EA017C
:10C260000E94D666FC01009741F08091880E909163
:10C27000890E92878187D487C387CF01DF91CF91C1
:10C2800008950F931F93DF93CF9300D000D0CDB7C5
:10C29000DEB78C01AB018FEF89838A838B838C831C
:10C2A000CE010196B8010E942D61FC01009711F0AA
:10C2B00015830483CF010F900F900F900F90CF91B3
:10C2C000DF911F910F91089586EB96E062E040E0C8
:10C2D00050E00E94ED3D109254271092532708958C
:10C2E000AC0186EB96E061E00E94CA3D0895AC0186
:10C2F00086EB96E060E00E94CA3D08950F931F937D
:10C30000CF93DF93EA010E944C668C01009761F0A5
:10C310008091880E9091890EF801958F848FD78F28
:10C32000C68FC8010E947761C801DF91CF911F912C
:10C330000F910895CF93DF93A091602CB091612C61
:10C34000109719F0ED016C9605C0C0915C2CD0914E
:10C350005D2C299680915B2C86FF22C0109263177A
:10C3600040E0E7E4F7E116C02081318114968D9119
:10C370009C9115972817390759F48281938100976A
:10C3800039F040936317998388831B821A8206C011
:10C3900034964F5F443040F3409363170E949F5F91
:10C3A00088819981009731F04A815B8160915227A1
:10C3B0000E94ED3DDF91CF9108950F931F93CF938E
:10C3C000DF9380916427863009F074C080915327F1
:10C3D0009091542725E08030920709F06BC0C4E9A2
:10C3E000D2E0D0935427C093532702E000935D27F7
:10C3F00014E910935E271092802710927F270E94E5
:10C400000B66809590959093802780937F2710925C
:10C410006627109265270E94FA6580959095909303
:10C420006627809365270E94AA5FD0935427C09304
:10C43000532700935D2710935E2790915E2C809187
:10C440005F2CE92FF82FDF01A459BD4F8CE692E055
:10C450000D9001920197E1F783E797E26CE672E0B5
:10C460000E949E658091572780937327809158275B
:10C4700080937427809159278093752780915A273C
:10C48000809376271092802710927F270E940B6658
:10C49000809590959093802780937F2710926627B0
:10C4A000109265270E94FA65809590959093662773
:10C4B000809365270E94AA5FDF91CF911F910F9112
:10C4C0000895282F392FF90120E030E080E0A8E11D
:10C4D00012C0419198E0542F5827B52FB17050FDEC
:10C4E0008A278695B13009F48068915011F04695FD
:10C4F000F2CF2F5F3F4F2617370759F708951F9246
:10C500000F920FB60F920BB60F9211242F933F93F9
:10C510004F935F936F937F938F939F93AF93BF934B
:10C52000EF93FF93809194009091950090933F2713
:10C5300080933E2781E08093302780917100807D39
:10C54000809371000E94995E809130278823E9F1E1
:10C55000809194009091950020913E2730913F2743
:10C5600082179307A0F48091042790910527A0914A
:10C570000627B09107278C57914EAF4FBF4F80933E
:10C58000042790930527A0930627B093072780914F
:10C59000940090919500821B930BA0E0B0E0209155
:10C5A0000427309105274091062750910727820FD5
:10C5B000931FA41FB51F8093042790930527A09372
:10C5C0000627B093072710923027FF91EF91BF9174
:10C5D000AF919F918F917F916F915F914F913F911B
:10C5E0002F910F900BBE0F900FBE0F901F901895BC
:10C5F0009FB7F894E1E7F0E08081807D808388B385
:10C600008F6288BB10929000E1E9F0E010821092F6
:10C610009200109295001092940080818560808332
:10C620009FBF08952FB7F894909399008093980036
:10C6300088B38F6288BBE1E7F0E08081826080830D
:10C640002FBF0895EF92FF92CF93DF93FC01DB01A0
:10C6500085E0EB0119928A95E9F7858190E0837076
:10C660009070009711F082E08C93878190E0837046
:10C670009070009721F082E012968C93129785813A
:10C6800090E083709070009799F0878190E08370BC
:10C690009070009769F023893489818592852817E5
:10C6A000390731F481E0848312961C92129701C0FD
:10C6B0001482858183708250823030F4C82FD0E09C
:10C6C000C054D94F888101C080E011968C93119796
:10C6D000E781E370E250E23028F4F0E0E054F94FF3
:10C6E000808101C080E013968C931397DF91CF91E6
:10C6F000FF90EF900895DF93CF9300D000D00F927A
:10C70000CDB7DEB7BE016F5F7F4F0E942263898184
:10C710009A81890F8D5F9B81890F9C81890F9D81F3
:10C72000890F0F900F900F900F900F90CF91DF9186
:10C730000895AF92BF92CF92DF92EF92FF920F9344
:10C740001F93DF93CF9300D000D000D0CDB7DEB7DA
:10C750008C017B01BE016F5F7F4F4E830E9422637D
:10C76000C9809A81A92EBB24DB808C81682F70E060
:10C7700095012C0D311D2D5F3F4F2D0D311D260FC5
:10C78000371F5D81250F311D4E8150E04217530741
:10C790000CF4A8C0D80111964C91119750E041704B
:10C7A0005070E3E0440F551FEA95E1F712962C9183
:10C7B000129730E02170307054E0220F331F5A95E9
:10C7C000E1F7242B3C913770232B13963C91139760
:10C7D000E32FF0E0E170F07045E0EE0FFF1F4A95A7
:10C7E000E1F72E2B14963C911497E32FF0E0E170C3
:10C7F000F07036E0EE0FFF1F3A95E1F72E2BF701B0
:10C80000208315964C91159750E043705070440F5B
:10C81000551F440F551F16962C91169730E0237024
:10C82000307054E0220F331F5A95E1F7242B1796EE
:10C830003C9117973295330F330F307C322B318375
:10C8400018962C9118972283FC2DF23069F41996D2
:10C850002C91D70113962C931397F80122851496E7
:10C860002C93149745E001C043E0E92FF0E03B969C
:10C87000E00FF11F542F0AC09701250F311DC29000
:10C88000D901CC925F5F0894A108B108A114B1044A
:10C8900099F7940FBD2DB23089F4F701E90FF11D1E
:10C8A000D80153962C91539720839F5FF701E90F8E
:10C8B000F11D54962C91549720839F5FE82FF0E050
:10C8C0007596E00FF11F292F08C0D701A20FB11DE7
:10C8D00032913C932F5F6150704061157105A9F74B
:10C8E000890F01C080E026960FB6F894DEBF0FBE18
:10C8F000CDBFCF91DF911F910F91FF90EF90DF900F
:10C90000CF90BF90AF900895BF92CF92DF92EF92F9
:10C91000FF920F931F93CF93DF937C01D62EEA01F2
:10C92000633008F4ADC0FC018081B82EB294B69497
:10C93000B694B3E0BB22F1E0BF22F7019181292F29
:10C94000269526952370C92EC294C694C694A3E05A
:10C95000CA22382F37703883382F3695369536955A
:10C9600031703983382F329531703A8382958695AC
:10C9700081708B83BC822D83892F829583708E83F7
:10C98000CF828281888787010D5F1F4F222361F14B
:10C99000F801918180E0F7013381830F911D9A871F
:10C9A000898787010B5F1F4F223081F4CA010B96E4
:10C9B00062E575E00E948E3BF80181818B87F7016B
:10C9C00085818C878701095F1F4F16C02330A1F432
:10C9D000F7013D96DA011B9682918D93E017F107DE
:10C9E000D9F7085F1F4F08C0CA010B9662E575E0D2
:10C9F0000E948E3B1A861986CC2089F1BB2059F4FF
:10CA0000F801918180E02081820F911D9C8B8B8B9E
:10CA10000E5F1F4F04C089859A859C8B8B8BFC2DE4
:10CA2000F23071F4CE01459662E575E00E948E3BCE
:10CA3000F80181818D8B80818E8B0E5F1F4F17C017
:10CA4000FC2DF330A1F4085F1F4FD801FE0175964D
:10CA500080E09E9191938F5F8830D9F708C0CE0116
:10CA6000459662E575E00E948E3B1C8A1B8A802FEA
:10CA70008E199D2D981B9FA71EA70DA7D81608F4E9
:10CA800080E0DF91CF911F910F91FF90EF90DF90A9
:10CA9000CF90BF9008959C0141505040460F571FC2
:10CAA000DB0110C0FC91E0E011968C911197BF0161
:10CAB000680F711D260F371F2617370710F42F5FD9
:10CAC0003F4F1296A417B50768F3A417B50749F4AA
:10CAD0009C9180E0280F391F2817390710F42F5F29
:10CAE0003F4FC9010895CF93DF9390915E27C92FDF
:10CAF000D0E0649730915D2720E0C20FD31F9E01E4
:10CB0000280F311DC90167E677E248E050E00E9436
:10CB10004B656FE677E2AE010E944B65009719F016
:10CB2000382F292F02C02FEF3FEFC901DF91CF919E
:10CB3000089590937717809376170895FC014381A9
:10CB4000460F40935A27872F99272281280F209339
:10CB50005927A181A093582750815093572730E03F
:10CB60002817390748F48A2F8F5F80935827882326
:10CB700019F45F5F50935727842F90E070708617E9
:10CB8000970798F4809159278F5F809359278823BE
:10CB900061F4809158278F5F80935827882329F468
:10CBA000809157278F5F809357270895BC0180910C
:10CBB000602C9091612C08960E949E65E091602CFB
:10CBC000F091612C80915727808780915827818729
:10CBD00080915927828780915A27838708959C01E5
:10CBE000AB0180E090E0B9010E944B65382F292FFE
:10CBF000C901089580E090E06BE577E244E150E000
:10CC00000E944B65009719F0382F292F02C02FEF93
:10CC10003FEFC901089586E00E947365089581E1A0
:10CC20000E947365089580E009C0E82FF0E0EE0FE0
:10CC3000FF1FEE51F34D118210828F5F8430A8F3F5
:10CC400080E00BC0E82FF0E095E0EE0FFF1F9A9513
:10CC5000E1F7EE59F34D118E8F5F843098F380E049
:10CC600094E0909379178093781740E08DE090E0FE
:10CC70000EC0242F30E0289FF001299FF00D389F2F
:10CC8000F00D1124E850F34D158214824F5F4A30A5
:10CC900080F3409374170895209178173091791795
:10CCA0002F5F3F4F4DE72030340710F020E030E198
:10CCB000522F432FA0E013C0EA2FF0E0B5E0EE0FB3
:10CCC000FF1FBA95E1F7EE59F34DB18DBB2331F05B
:10CCD0000480F581E02DE417F50711F3AF5FA43070
:10CCE00059F730937917209378171092741720E032
:10CCF000E0E0F0E01EC0A22FB0E035E0AA0FBB1FBD
:10CD00003A95E1F7AE59B34D59963C915997332373
:10CD100021F420937417FD0110C0373049F4309787
:10CD200031F05A964C915A97328D341708F4FD0120
:10CD30002F5F243000F3209374173097A9F122E07D
:10CD4000218F20916E17248720916F1725872091BE
:10CD50007017268720917117278728ED34E0338BD1
:10CD6000228B358B248B21E030E0318B208B138E8E
:10CD700021E0228F23E0208F168A20E1278B20914B
:10CD80007817309179173227232732273583248368
:10CD900077836683DC012D913D914D915C911397D2
:10CDA0002083318342835383CF0108950F931F93D0
:10CDB000CF93DF9320917817309179174DE050E0B1
:10CDC0002F5F3F4FADE720303A0710F020E030E111
:10CDD000B22FA32F10E012C0C12FD0E0C49FF001EA
:10CDE000C59FF00DD49FF00D1124E850F34D048041
:10CDF000F581E02DEA17FB0719F31F5F1A3061F781
:10CE0000309379172093781710E02DE030E01AC0A6
:10CE1000012F0F5FC12FD0E0C29FF001C39FF00D23
:10CE2000D29FF00D1124E850F34DDF011496448198
:10CE300055814115510529F410937417309749F421
:10CE400033C0102F1A3020F310937417E0E0F0E095
:10CE50002BC020917817309179173227232732275A
:10CE600011963C932E9377836683009729F4108262
:10CE700011821282138209C0DC012D913D914D91E6
:10CE80005C9120833183428353838DE090E0C89F7F
:10CE9000D001C99FB00DD89FB00D1124A850B34D3B
:10CEA00080E418968C931897CF01DF91CF911F9152
:10CEB0000F91089540E013C0E42FF0E0542F5F5F1E
:10CEC000EE0FFF1FEE51F34D2081318128173907F6
:10CED00029F440937417118210820895452F44302D
:10CEE00058F340937417089540E013C0E42FF0E026
:10CEF000542F5F5FEE0FFF1FEE51F34D2081318104
:10CF00002115310529F44093741791838083089586
:10CF1000452F443058F3409374170895EF92FF92D1
:10CF20000F931F93CF93DF93C091602CD091612C0E
:10CF3000843009F4F7C103E817E210935F2C0093E3
:10CF40005E2C1093562700935527833071F4898DFA
:10CF500090E08F7090708330910509F074C08889DB
:10CF60009989009709F02FC78DC0823009F08EC0D3
:10CF7000809171178F5F80937117882399F4809146
:10CF800070178F5F80937017882361F480916F17FB
:10CF90008F5F80936F17882329F480916E178F5FBE
:10CFA00080936E1710925427109253271092F72CEB
:10CFB0001092F62C898D873011F0853041F48A8DDE
:10CFC0008F5F8A8F843109F0FEC6198EFCC68823D4
:10CFD00009F4F9C6288939892115310509F44EC0AB
:10CFE0009A8D292F21502A8F992309F0ECC69B8D09
:10CFF000983031F0282F2150223048F4953039F400
:10D00000198E80E880935B2C0E949A6195C59530BB
:10D0100048F423E030E0092E02C0220F331F0A94A7
:10D02000E2F701C020E32A8F9F5F9B8F90E08F7013
:10D03000907083309105E1F0843091054CF481309B
:10D04000910509F461C38230910509F0BCC60DC099
:10D050008630910509F40CC58830910509F408C59E
:10D060008430910509F0AFC603C510927C274FC3E9
:10D0700084E080935B2C0E949A6190C58F7083300E
:10D0800009F0A1C688E080935B2C4BC5853019F56B
:10D09000E0915C2CF0915D2C84819581009709F4DE
:10D0A00092C61092612C1092602C0C50104010937C
:10D0B0005F2C00935E2C10935627009355271092F7
:10D0C000F72C1092F62C109254271092532788E0D8
:10D0D00080935B2C25C10852104080915B278534DA
:10D0E00009F071C690915D2780E020915E277C0158
:10D0F000E20EF11C80915327909154278E159F05C5
:10D1000008F461C6F0925427E0925327809161277A
:10D1100090E08F739070009709F055C68091622758
:10D12000882309F050C68091F22C9091F32CC09185
:10D13000C606D091C7068C179D0759F44091F42C70
:10D140005091F52C2091C8063091C906421753071B
:10D15000A1F020916B2730916C272817390709F02F
:10D1600032C620916D2730916E278091F42C9091DA
:10D17000F52C2817390709F026C60E94FA652FEF0B
:10D180008F3F920709F01FC680916427863009F40B
:10D1900031C18131E9F1813009F015C680916F27E5
:10D1A000883009F010C610926F27809171279091F6
:10D1B00072274FEF873F940710F0099601C0089639
:10D1C00090937227809371278091672790916827A9
:10D1D000A0916927B0916A2780936B2790936C2761
:10D1E000A0936D27B0936E278091F22C9091F32C31
:10D1F000A091F42CB091F52C809367279093682729
:10D20000A0936927B0936A2780E4F8018087B8C5A6
:10D21000C7014C97909354278093532787E797E251
:10D2200090935F2C80935E2C809175279091762748
:10D23000009739F00E940F66FFEF8F3F9F0709F0BC
:10D24000C2C520917127309172272115310509F44B
:10D25000BAC588EF9CE290935D2C80935C2C609122
:10D26000C8067091C9064091C2065091C30600914C
:10D27000C4061091C50639C084819581009781F15B
:10D280002817390769F586819781009739F0A091B1
:10D290006F27B0917027A817B90711F58081918188
:10D2A0008C179D0729F4A281B381A617B70739F11E
:10D2B0008417950729F4A281B381A017B107F9F06B
:10D2C000A0916727B0916827A817B90749F4A091E2
:10D2D0006927B0916A2782819381A817B90779F0ED
:10D2E0003D96F0935D2CE0935C2CE0915C2CF091EA
:10D2F0005D2C8DE2EA37F80708F4BECF64C51092C2
:10D30000612C1092602C82E080935B2C87E797E27F
:10D3100090935627809355271092F72C1092F62C55
:10D320000E949A618091F62C9091F72C009709F455
:10D330004AC59C01245E3F4F3093542720935327C6
:10D3400030935D2720935E27E0915C2CF0915D2C5B
:10D3500020852093632721E120936427089698274E
:10D3600089279827909374278093732710927627A4
:10D3700010927527848195819093702780936F27F1
:10D380008681978190937227809371278091F22CE8
:10D390009091F32CA091F42CB091F52C80936727F9
:10D3A00090936827A0936927B0936A278081918121
:10D3B000A281B38180936B2790936C27A0936D27F4
:10D3C000B0936E2783E897E290935F2C80935E2C56
:10D3D0000E940F668095909590937627809375278D
:10D3E000009709F0CDC48FEF9FEF9093762780933D
:10D3F0007527C6C40E940B66EFEF8F3F9E0709F0AA
:10D40000E2C48091712790917227009709F4DBC4E0
:10D4100020916F27309170272115310509F4D3C46D
:10D42000C2E6DCE2498D4423E9F06C817D818617F8
:10D430009707C1F46E817F812617370799F4E09131
:10D440006727F091682768817981E617F70751F41B
:10D45000E0916927F0916A276A817B81E617F707D7
:10D4600009F46DC1A096FCE2C23EDF07D9F6209117
:10D470007C272F732230B9F490937317809372171F
:10D4800040E00DC0E42FF0E0EE0FFF1FEE51F34D32
:10D49000208131814F5F8217930709F46EC04430B9
:10D4A00088F34093741780917C2782FD8CC484E1BB
:10D4B000F80181A388E290E090935427809353274A
:10D4C00080E580A38091762790917A27938F309181
:10D4D000752790917927928F368F2091742790919C
:10D4E0007827918F258F909173279093741740918F
:10D4F0007727408F948F8F5F878F882361F4832FE6
:10D500008F5F868F882339F4822F8F5F858F8823E2
:10D5100011F49F5F948F80916F2790917027909363
:10D520007317809372172091712730917227F80139
:10D53000358B248B978B868B8091672790916827FA
:10D54000A0916927B0916A2780936B2790936C27ED
:10D55000A0936D27B0936E278091F22C9091F32CBD
:10D56000A091F42CB091F52C8093672790936827B5
:10D57000A0936927B0936A27E8C31092741780E0DC
:10D58000C0E0D0E022C0E82FF0E075E0EE0FFF1F12
:10D590007A95E1F7EE59F34D918D992321F480931B
:10D5A0007417EF0116C0973079F4209721F0228D7F
:10D5B0009A8D921748F4C82FD0E065E0CC0FDD1F9C
:10D5C0006A95E1F7CE59D34D8F5F8430E0F28093B6
:10D5D0007417209709F4F7C3D093612CC093602C83
:10D5E00083E08A8F888F1E8A84E08F8B1B8E8091C8
:10D5F0007127909172279D838C8380916F279091E2
:10D6000070279F838E838091672790916827A091D0
:10D610006927B0916A2788839983AA83BB8381E0B5
:10D62000898F80916E178C8780916F178D8780917D
:10D6300070178E87809171178F8781E090E0998BAA
:10D64000888B809176278B87809175278A87809138
:10D650007427898780917327888781E090E00E94F2
:10D66000D66580917B27282F30E0207F30702135D0
:10D6700031050CF449C082958F7090E00597880FB2
:10D68000991F880F991F5091751740E034C0F90118
:10D69000E55AF84D50A5552329F44093741710927C
:10D6A000751732C0513011F44F5F25C05230E1F48C
:10D6B00061A56430C9F4409374175093751732A56F
:10D6C00020E083A590E0822B932B90937317809397
:10D6D0007217F4E0893D9F0710F088ED94E09B8B72
:10D6E0008A8B9D8B8C8B10C0255A384DF90121A552
:10D6F000222331F0420F242F30E0281739073CF263
:10D70000409374175093751780E180937C27809124
:10D710007C27826080937C2782E08093832784E04B
:10D72000809384278093852788ED809386278CE2D9
:10D7300090E0909354278093532780E6B3C2D09310
:10D74000612CC093602C10925B2C80917C2790E020
:10D7500082FF03C0198E80E24EC220917B27229562
:10D760002F70220F220F20937417B701621B7109CB
:10D770009B0124513040309354272093532750E08D
:10D780004F7050704230510539F4AC014F735070F6
:10D790004231510551F42AC04130510531F4AC01F8
:10D7A0004F7350704230510509F12115310531F4A4
:10D7B0009C012370307021153105C1F03091732721
:10D7C0002885321709F064C23091742729853217F1
:10D7D00009F05EC2309175272A85321709F058C2C8
:10D7E000309176272B85321709F052C284FF4AC048
:10D7F000688979896115710509F444C0CE010C96D8
:10D800000E949E6530917727809157273817D1F570
:10D8100020917827809158272817A1F59091792792
:10D8200080915927981771F580917A2740915A274E
:10D83000841741F53C872D879E878F878B8D8823A2
:10D84000D1F42E89888D9A8D891B922F9695969565
:10D850009695891B280F2E8B87FD81959F89392FDF
:10D8600036953695931B980F9F8B822F86958695BC
:10D870008695890F888F81E080935B2C888D8A8FB5
:10D88000198A188A298D30E0C9018F709070843010
:10D89000910509F4B5C18530910564F48230910594
:10D8A000C9F1833091050CF0B9C08130910509F0C0
:10D8B0008AC211C08630910509F4E2C18630910513
:10D8C0000CF4BEC18730910509F4E2C1883091059E
:10D8D00009F079C28AC180915B2C80FF14C083E07B
:10D8E000898F80E480935B2C198A188A8091532752
:10D8F00090915427009709F410C122E420935B2CE7
:10D900000E94D6650AC180917C278F73823009F00E
:10D910005AC2FACE80915B2C80FF75C080917C2723
:10D920008F73823109F06FC080917B27282F30E000
:10D93000207F3070213531050CF449C082958F70FD
:10D9400090E00597880F991F880F991F50917517C0
:10D9500040E034C0F901E55AF84D50A5552329F4AB
:10D96000409374171092751732C0513011F44F5F05
:10D9700025C05230E1F461A56430C9F440937417B6
:10D980005093751732A520E083A590E0822B932B4E
:10D99000909373178093721774E0893D970710F086
:10D9A00088ED94E09B8B8A8B9D8B8C8B10C0255AC5
:10D9B000384DF90121A5222331F0420F242F30E008
:10D9C000281739073CF2409374175093751783E07A
:10D9D000898F8091732788878091742789878091A8
:10D9E00075278A87809176278B8781E090E00E9457
:10D9F000D66582E480935B2C198A188A109254278A
:10DA0000109253278AC080E280935B2C0E949A6117
:10DA1000E091602CF091612C118E45CD80917C2796
:10DA200080FF2AC024FD28C088899989009709F0C1
:10DA3000CAC1809153279091542701960E94D665C0
:10DA400020915B2C822F806180935B2C80915327E7
:10DA500090915427009719F0226120935B2C0E942B
:10DA60009A6181E090E0998B888B88E0898F1B8E8A
:10DA700081E180937C270FC185FF1CC050918127D5
:10DA800040E08091822790E0842B952B40915E2C82
:10DA900050915F2C480F591F50935F2C40935E2C80
:10DAA0004091532750915427481B590B50935427AA
:10DAB000409353278091532790915427009749F022
:10DAC00024FD07C020915B2C226020935B2C0E94D8
:10DAD000D66590917D2780E020917E27820F911D51
:10DAE00090937317809372172C893D8928173907F3
:10DAF00010F0009721F430937317209372178091E0
:10DB00007217909173179B8B8A8B80915B2C90E09E
:10DB100083709070009709F456C11092F72C109200
:10DB2000F62C0E949A6180915B2C85FF07C01092B1
:10DB3000F72C1092F62C198E84E19BCF84FF0AC03B
:10DB40001092F72C1092F62C81E090E0998B888B44
:10DB500084E08CCF2091F62C3091F72C21153105E3
:10DB6000E1F080FF02C0198A188A88899989009794
:10DB700081F48A899B898217930720F49093F72C6C
:10DB80008093F62C8091F62C9091F72C998B888BB2
:10DB900004C09093F72C8093F62C1B8E8091552710
:10DBA0009091562790935F2C80935E2C8091F62C59
:10DBB0009091F72C009759F088899989009739F04E
:10DBC0008896909354278093532788E10BC08091C7
:10DBD0005B2C81FFF8C088E290E0909354278093FB
:10DBE000532780E180937C275CC080915B2C80FF71
:10DBF000EAC0198E80E180935B2C0E949A61E3C099
:10DC00008091532790915427009711F00E94D66578
:10DC100090917C2780915B2C90FF0BC080FF06C009
:10DC200087E0898F1A8E198A188A19C086E0898F31
:10DC300016C080FF1EC085E0898F198A188AC3C06C
:10DC40008091532790915427009711F00E94D66538
:10DC500080917C2780FF0DC087E0898F1A8E81E03C
:10DC600090E00E94D66580E180935B2C0E949A61CF
:10DC70000FC08091532790915427009749F4A3C077
:10DC800080915B2C80FF9FC087E0898F1A8E9BC09C
:10DC900080E1F80181A388E290E09093542780937B
:10DCA000532780E580937B27888580937727898514
:10DCB000809378278A85809379278B8580937A272C
:10DCC0008C85809373278D85809374278E858093B0
:10DCD00075278F858093762786E0809364278C81D3
:10DCE0009D819093702780936F278E819F81909361
:10DCF0007227809371278091F22C9091F32CA09140
:10DD0000F42CB091F52C8093672790936827A0930B
:10DD10006927B0936A2788819981AA81BB81809302
:10DD20006B2790936C27A0936D27B0936E27898DF6
:10DD300084FF05C010927E2710927D2706C084E0E4
:10DD400080937D2788ED80937E2780E480936327EE
:10DD5000809153279091542790935D2780935E275D
:10DD600010928227109281271092802710927F278D
:10DD70000E940B66809590959093802780937F27D3
:10DD800085E480935B2710925C27109262271092A3
:10DD90006127809176179091771701969093771766
:10DDA0008093761790935F27809360271092662761
:10DDB000109265270E94FA6580959095909366274A
:10DDC0008093652704C01092542710925327109215
:10DDD0005B2CDF91CF911F910F91FF90EF900895F1
:10DDE000382F292FC9010895382F292F40E050E0FE
:10DDF00076276727762780E090E0CB017727662794
:10DE0000262B372B482B592BB901CA010895AC0199
:10DE1000E0915527F0915627222733272E1B3F0BE1
:10DE2000255A334D621773070CF49B011216130623
:10DE300064F42093F62C3093F72C4E175F0729F0EB
:10DE4000CF01BA01A9010E940C7A08950F93DF93C4
:10DE5000CF93CDB7DEB760970FB6F894DEBF0FBE95
:10DE6000CDBF002309F459C029833A834B835C83D7
:10DE70006D837E838F839887E0E2E01B29813A815E
:10DE80004B815C811E16BCF019861A861B861C8687
:10DE90008E2F992787FD9095909581959F4F04C06F
:10DEA000220F331F441F551F8A95D2F72D873E87B7
:10DEB0004F87588B2AC0CA01B901002E04C0660FD3
:10DEC000771F881F991F0A94D2F769877A878B87F3
:10DED0009C87DA01C90104C0B695A79597958795E7
:10DEE000EA95D2F72D813E814F81588504C0220FDB
:10DEF000331F441F551F0A95D2F7822B932BA42B57
:10DF0000B52B8D879E87AF87B88B29853A854B8542
:10DF10005C856D857E858F85988960960FB6F894AF
:10DF2000DEBF0FBECDBFCF91DF910F910895A0E16D
:10DF3000B0E0EDE9FFE60C945F7729833A834B83E9
:10DF40005C836D837E838F839887A986BA86CB8610
:10DF5000DC86ED86FE860F87188B2D813E814F81F2
:10DF600058858D859E85AF85B889281739074A075A
:10DF70005B07C8F082179307A407B50790F02981C3
:10DF80003A814B815C8189859A85AB85BC85281750
:10DF900039074A075B0738F082179307A407B507CC
:10DFA00020F482E003C080E001C081E06096EAE0F6
:10DFB0000C947B772F923F924F925F926F927F9259
:10DFC0008F929F92AF92BF92CF92DF92EF92FF9289
:10DFD0000F931F93DF93CF93CDB7DEB763970FB641
:10DFE000F894DEBF0FBECDBF6C017F876E87FC014A
:10DFF00017821682838181FD04C06FC34C855D85C5
:10E0000004C01E010894211C311CF6019381EE8589
:10E01000FF8593FD859193FF8191FF87EE8788238C
:10E0200009F457C3853241F493FD859193FF8191A3
:10E03000FF87EE87853259F490E0B6014A8B5B8BFF
:10E040000E946E7A4A895B895D874C87D7CF10E042
:10E05000FF2400E00032B0F48B3269F08C3228F4F7
:10E06000803251F0833271F40BC08D3239F080333D
:10E0700049F401602CC00260046029C0086027C018
:10E08000006125C007FD2EC0282F20532A3098F4A8
:10E0900006FF08C0812F880F182F110F110F180FBE
:10E0A000120F15C08F2D880FF82EFF0CFF0CF80EE5
:10E0B000F20E00620CC08E3221F406FD0AC3006429
:10E0C00006C08C3611F4006802C0883659F4EE851B
:10E0D000FF8593FD859193FF8191FF87EE878823CC
:10E0E00009F0B8CF982F9554933018F40061805EF2
:10E0F00006C0982F9556933008F09BC10F7E06FFFF
:10E1000016E06FE3E62EE022853619F4F0E4EF2AFC
:10E1100007C0863619F420E8E22A02C01111115016
:10E12000E7FE06C01C3340F4912E939427E00BC009
:10E13000183030F4212F06C027E03CE3932E03C0B3
:10E1400027E017E09924CA0104969D878C87FA017D
:10E150006081718182819381A101092D0E941C79C6
:10E160005C016980262D30E0398B288B60FE03C06E
:10E17000388933FF06C0E1FC06C0E2FE06C000E2BB
:10E1800005C00DE203C00BE201C000E08889998957
:10E190008C7090700097C1F1002311F084E001C0F1
:10E1A00083E08F1558F4F81AE3FC09C080E290E090
:10E1B000B6010E946E7AFA94C9F701C0FF240023C9
:10E1C00029F0802F90E0B6010E946E7A888983FD45
:10E1D00003C002E31FE00EC00EE21FE00BC0A1145B
:10E1E000B10409F0805290E0B6010E946E7A0F5F90
:10E1F0001F4F05C0AE2CBB2490E1A922BB24F8011F
:10E200008491882361F762C2E7FE0EC09A0CF889F8
:10E21000F4FF04C08A81813309F49A94191454F5E7
:10E22000292D293050F52DC0E6FC2BC0812F90E020
:10E230008A159B054CF03CEFA3163FEFB30624F084
:10E2400080E8E82A01C01150112349F0E2E0F0E033
:10E25000EC0FFD1FE10FF11D80818033A1F3E7FE7C
:10E2600010C0912E9394812F90E0A816B90644F423
:10E270001A1907C09924939404C098E0992E01C0FC
:10E2800010E0E7FE07C01A141B043CF495012F5F51
:10E290003F4F05C025E030E002C021E030E0002320
:10E2A00011F02F5F3F4F112329F0812F90E001964D
:10E2B000280F391F8F2D90E02817390714F4F21A10
:10E2C00001C0FF244E2C5524C20189709070009724
:10E2D00049F406C080E290E0B6010E946E7AFA949A
:10E2E000FF20C1F7002329F0802F90E0B6010E94A3
:10E2F0006E7A43FC09C006C080E390E0B6010E943C
:10E300006E7AFA94FF20C1F7E7FE46C03501B7FEEA
:10E3100002C06624772425010894411C511C46182C
:10E320005708420C531CF501E919F1094F01812FDF
:10E3300090E000271127081B190BFFEF6F16FFEF66
:10E340007F0629F48EE290E0B6010E946E7AA61450
:10E35000B70434F0861497041CF4F201808101C0E4
:10E3600080E30894610871080894411C511C6016F0
:10E3700071062CF090E0B6010E946E7ADECF6A142E
:10E380007B0441F49A81963320F4953319F4F8898B
:10E39000F4FF81E390E049C08A81813311F02FEED0
:10E3A000622290E0B6010E946E7A112389F08EE21B
:10E3B00090E0B6010E946E7A02E0F101E00FF11DDB
:10E3C0000F5F808190E0B6010E946E7A1150A9F72C
:10E3D00044FE03C085E490E002C085E690E0B6010B
:10E3E0000E946E7AB7FC05C0A114B10441F464FE2A
:10E3F00006C0B094A194B108B3948DE201C08BE241
:10E4000090E0B6010E946E7A80E305C08F5FE6EF70
:10E41000FFEFAE0EBF1EFAE0AF16B104BCF790E0FE
:10E42000B6010E946E7AC501C096B6010E946E7A4E
:10E430004DC1833631F0833789F0833509F059C0F7
:10E4400022C09A012E5F3F4F3D872C87FA018081C1
:10E450008983310181E0A82EB12C13C09A012E5F6F
:10E460003F4F3D872C87FA016080718006FF03C013
:10E47000612F70E002C06FEF7FEFC3010E94347A1A
:10E480005C010F7714C09A012E5F3F4F3D872C87A8
:10E49000FA016080718006FF03C0612F70E002C046
:10E4A0006FEF7FEFC3010E94FC795C01006803FD00
:10E4B0001CC006C080E290E0B6010E946E7AFA9419
:10E4C0008F2D90E0A816B906A8F30FC0F30107FD41
:10E4D000859107FF81913F0190E0B6010E946E7A1D
:10E4E000F110FA940894A108B108A114B10471F7CD
:10E4F000EDC0843611F0893661F507FF0BC09A0133
:10E500002C5F3F4F3D872C87FA01608171818281AA
:10E5100093810CC09A012E5F3F4F3D872C87FA01F3
:10E5200060817181882777FD8095982F0F7697FFFE
:10E5300008C090958095709561957F4F8F4F9F4F44
:10E540000068A1012AE030E00E94807B982E92189A
:10E5500041C0853721F40F7E2AE030E020C0097FDA
:10E560008F36A9F0803720F4883509F0B2C00BC08F
:10E57000803721F0883709F0ACC001C0006104FF8A
:10E5800009C0046007C004FF08C0066006C028E098
:10E5900030E005C020E130E002C020E132E007FFBA
:10E5A0000AC0CA0104969D878C87FA016081718137
:10E5B0008281938109C0CA0102969D878C87FA01E6
:10E5C0006081718180E090E0A1010E94807B982EA3
:10E5D00092180F7706FF09C00E7F911630F404FFE2
:10E5E00006C002FD04C00F7E02C0E92C01C0E12E6E
:10E5F000802F90E004FF0CC0FE01E90DF11D208189
:10E60000203311F4097E09C0E39402FF06C004C060
:10E6100086789070009709F0E394A02EBB2403FD48
:10E6200014C000FF0FC0EF1428F4192D1F0D1E1980
:10E63000EF2C08C0192D06C080E290E0B6010E94C0
:10E640006E7AE394EF14C0F304C0EF1410F4FE18D4
:10E6500001C0FF24A4FE0FC080E390E0B6010E9439
:10E660006E7AA2FE1FC0A1FE03C088E590E010C034
:10E6700088E790E00DC0C50186789070009791F012
:10E68000A1FC02C080E201C08BE207FD8DE290E0B8
:10E69000B6010E946E7A06C080E390E0B6010E9447
:10E6A0006E7A11509116C0F39A94F101E90DF11DA3
:10E6B000808190E0B6010E946E7A9920A9F706C089
:10E6C00080E290E0B6010E946E7AFA94FF20C1F7D2
:10E6D00095CCF6012681378102C02FEF3FEFC901AB
:10E6E00063960FB6F894DEBF0FBECDBFCF91DF911A
:10E6F0001F910F91FF90EF90DF90CF90BF90AF9060
:10E700009F908F907F906F905F904F903F902F9051
:10E7100008955058BB27AA270ED044C135D130F0F8
:10E720003AD120F031F49F3F11F41EF42AC10EF4C7
:10E73000E095E7FB20C1E92F46D180F3BA176207C5
:10E7400073078407950718F071F49EF55EC10EF407
:10E75000E0950B2EBA2FA02D0B01B90190010C01F1
:10E76000CA01A0011124FF27591B99F0593F50F409
:10E77000503E68F11A16F040A22F232F342F442761
:10E78000585FF3CF469537952795A795F040539559
:10E79000C9F77EF41F16BA0B620B730B840BBAF029
:10E7A0009150A1F0FF0FBB1F661F771F881FC2F794
:10E7B0000EC0BA0F621F731F841F48F487957795A8
:10E7C0006795B795F7959E3F08F0B3CF9395880F5F
:10E7D00008F09927EE0F979587950895A8D008F42B
:10E7E00081E008950CD0DEC0D6D040F0CDD030F01E
:10E7F00021F45F3F19F0BFC0511108C1C2C0E3D07E
:10E8000098F39923C9F35523B1F3951B550BBB27F7
:10E81000AA2762177307840738F09F5F5F4F220FA4
:10E82000331F441FAA1FA9F333D00E2E3AF0E0E89D
:10E8300030D091505040E695001CCAF729D0FE2FE9
:10E8400027D0660F771F881FBB1F2617370748077B
:10E85000AB07B0E809F0BB0B802DBF01FF27935831
:10E860005F4F2AF09E3F510568F085C0CFC05F3FE3
:10E87000ECF3983EDCF3869577956795B795F79519
:10E880009F5FC9F7880F911D9695879597F9089511
:10E89000E1E0660F771F881FBB1F621773078407AD
:10E8A000BA0720F0621B730B840BBA0BEE1F88F7BC
:10E8B000E0950895E89409C097FB3EF49095809503
:10E8C000709561957F4F8F4F9F4F9923A9F0F92F36
:10E8D00096E9BB279395F695879577956795B795B4
:10E8E000F111F8CFFAF4BB0F11F460FF1BC06F5F9A
:10E8F0007F4F8F4F9F4F16C0882311F096E911C0AC
:10E90000772321F09EE8872F762F05C0662371F0CC
:10E9100096E8862F70E060E02AF09A95660F771FE0
:10E92000881FDAF7880F9695879597F90895990FBC
:10E930000008550FAA0BE0E8FEEF16161706E807C9
:10E94000F907C0F012161306E407F50798F0621BEA
:10E95000730B840B950B39F40A2661F0232B242BBF
:10E96000252B21F408950A2609F4A140A6958FEFDE
:10E97000811D811D089597F99F6780E870E060E030
:10E9800008959FEF80EC089500240A941616170648
:10E9900018060906089500240A9412161306140690
:10E9A00005060895092E0394000C11F4882352F0F3
:10E9B000BB0F40F4BF2B11F460FF04C06F5F7F4FAB
:10E9C0008F4F9F4F089557FD9058440F551F59F092
:10E9D0005F3F71F04795880F97FB991F61F09F3F4C
:10E9E00079F087950895121613061406551FF2CF75
:10E9F0004695F1DF08C0161617061806991FF1CFC5
:10EA000086957105610508940895E894BB276627EB
:10EA10007727CB0197F908950BD0C4CFB5DF28F045
:10EA2000BADF18F0952309F0A6CFABCF1124EECFB3
:10EA3000CADFA0F3959FD1F3950F50E0551F629F59
:10EA4000F001729FBB27F00DB11D639FAA27F00D47
:10EA5000B11DAA1F649F6627B00DA11D661F829F6E
:10EA60002227B00DA11D621F739FB00DA11D621F53
:10EA7000839FA00D611D221F749F3327A00D611D70
:10EA8000231F849F600D211D822F762F6A2F112452
:10EA90009F5750408AF0E1F088234AF0EE0FFF1FA5
:10EAA000BB1F661F771F881F91505040A9F79E3FDC
:10EAB000510570F060CFAACF5F3FECF3983EDCF3D6
:10EAC000869577956795B795F795E7959F5FC1F719
:10EAD000FE2B880F911D9695879597F90895FA0159
:10EAE000EE0FFF1F30962105310599F16115710573
:10EAF00061F48038BFE39B0749F168949038810541
:10EB000061F08038BFEF9B0741F0992342F5FF3F4A
:10EB1000E1053105210511F1E8940894E795D90143
:10EB2000AA2329F4AB2FBE2FF85FD0F310C0FF5FEC
:10EB300070F4A695E0F7F73950F019F0FF3A38F481
:10EB40009F779F930CD00F9007FC905808953EF04C
:10EB500018CF60E070E080E89FE308954FE79F776B
:10EB60005F934F933F932F939ED02F913F914F915F
:10EB70005F9152DF05C019F40EF0FDCE46CF01CFF4
:10EB80002ADFC8F39638C0F707F80F92E8942BE312
:10EB90003AEA48EB5FE74EDF0F920F920F924DB7C4
:10EBA0005EB70F92C0D0E0E2F1E016D04F915F91D6
:10EBB000EF91FF91E595EE1FFF1F49F0FE57E068CA
:10EBC0004427EE0F441FFA95E1F74195550B32D0DB
:10EBD0000F9007FE26C00895DF93CF931F930F93E6
:10EBE000FF92EF92DF927B018C01689405C0DA2ED0
:10EBF000EF011EDFFE01E894A59125913591459125
:10EC00005591AEF3EF0197DDFE019701A801DA946B
:10EC100079F7DF90EF90FF900F911F91CF91DF91E7
:10EC200008959B01AC0160E070E080E89FE3DACDDD
:10EC3000A2CEACC0D0DEE8F39923D9F3940F511DD6
:10EC4000BBF39150504094F059F0882332F0660F96
:10EC5000771F881F91505040C1F79E3F510544F7E0
:10EC6000880F911D9695879597F908955F3FACF0B1
:10EC7000983E9CF0BB27869577956795B79508F4E5
:10EC8000B1609395C1F7BB0F58F711F460FFE8CF5F
:10EC90006F5F7F4F8F4F9F4FE3CFB8CE0EF076C0A0
:10ECA00070CE689468CE97DEC8F39923D1F3C6F38B
:10ECB000DF93CF931F930F93FF92C92FDD278823F4
:10ECC0002AF02197660F771F881FDAF720E030E0DF
:10ECD00040E85FEB9FE3883920F0803E30F02196DA
:10ECE0008F7718DDE8E4F1E003C014DDE5E7F1E03B
:10ECF00073DF8B01BE01EC01FB2E6F577109759517
:10ED0000771F880B990BD8DD28E132E741E35FE3F9
:10ED10008FDEAF2D9801AE01FF900F911F91CF9123
:10ED2000DF9109DD3FCEFA01DC01AA0FBB1F9B0179
:10ED3000AC01BF5728F422273327442750781FC03F
:10ED4000B75188F4AB2F0024469537952795011CC1
:10ED5000A395D2F3002069F0220F331F441FB3950F
:10ED6000DAF30DD0D6CC61307105A0E88A07B94638
:10ED700030F49B01AC01662777278827907830967E
:10ED800021F0208331834283538308959F3F31F0E4
:10ED9000915020F4879577956795B795880F911DC9
:10EDA0009695879597F90895629FD001739FF0011A
:10EDB000829FE00DF11D649FE00DF11D929FF00D0B
:10EDC000839FF00D749FF00D659FF00D9927729F42
:10EDD000B00DE11DF91F639FB00DE11DF91FBD01CD
:10EDE000CF0111240895AA1BBB1B51E107C0AA1F24
:10EDF000BB1FA617B70710F0A61BB70B881F991FDC
:10EE00005A95A9F780959095BC01CD01089597FB7F
:10EE1000092E07260AD077FD04D0E5DF06D00020B2
:10EE20001AF4709561957F4F0895F6F79095819546
:10EE30009F4F0895A1E21A2EAA1BBB1BFD010DC016
:10EE4000AA1FBB1FEE1FFF1FA217B307E407F5079A
:10EE500020F0A21BB30BE40BF50B661F771F881F76
:10EE6000991F1A9469F760957095809590959B010C
:10EE7000AC01BD01CF01089597FB092E05260ED0E8
:10EE800057FD04D0D7DF0AD0001C38F450954095C8
:10EE9000309521953F4F4F4F5F4F0895F6F790956E
:10EEA0008095709561957F4F8F4F9F4F08952F925A
:10EEB0003F924F925F926F927F928F929F92AF920A
:10EEC000BF92CF92DF92EF92FF920F931F93CF9357
:10EED000DF93CDB7DEB7CA1BDB0B0FB6F894DEBFEE
:10EEE0000FBECDBF09942A88398848885F846E8414
:10EEF0007D848C849B84AA84B984C884DF80EE805E
:10EF0000FD800C811B81AA81B981CE0FD11D0FB666
:10EF1000F894DEBF0FBECDBFED010895AF92BF9252
:10EF2000CF92DF92EF92FF920F931F93CF93DF93D5
:10EF3000EC01688179818A819B8161157105810568
:10EF4000910521F464E279ED8BE597E02DE133EF53
:10EF500041E050E00E943C7779018A0127EA31E4E0
:10EF600040E050E00E94D4765B016C01C801B7011B
:10EF70002CEE34EF4FEF5FEF0E94D4766A0D7B1DCD
:10EF80008C1D9D1D97FF04C06150704080409048CB
:10EF9000688379838A839B837F77CB01DF91CF91CD
:10EFA0001F910F91FF90EF90DF90CF90BF90AF90A7
:10EFB00008950E948E7708958AEC96E00E948E77DD
:10EFC0000895A0E0B0E08093CA069093CB06A0938A
:10EFD000CC06B093CD0608952F923F924F925F9248
:10EFE0006F927F929F92AF92BF92CF92DF92EF92F9
:10EFF000FF920F931F93CF93DF933B01EA016115BB
:10F00000710519F0FB0180839183209739F09E01EF
:10F01000225030402332310508F0D5C0C82ED92EF9
:10F02000F60111916F017F01812F90E00E94F47928
:10F030000097B1F71D3231F4F60111917F01992447
:10F04000939406C01B3219F4F60111917F019924A3
:10F05000209719F0C031D105D1F4103389F4F701AC
:10F060008081883711F0883559F4F701118182E0E9
:10F0700090E0E80EF91E92E0992AC0E1D0E007C0C6
:10F08000209729F41033B1F0CAE0D0E02BC0CA3089
:10F09000D10541F1C031D10521F0C830D105A9F425
:10F0A00009C02FEFA22E2FEFB22E2FEFC22E2FE08E
:10F0B000D22E20C0C8E0D0E09FEFA92E9FEFB92E3E
:10F0C0009FEFC92E9FE1D92E15C09E01442737FD21
:10F0D0004095542F6FEF7FEFCB010E941A775901B3
:10F0E0006A0108C089E9A82E89E9B82E89E9C82EE5
:10F0F00089E1D82E60E020E030E0A9011E0144241F
:10F1000037FC4094542C012F00530A3060F0812FBB
:10F1100081548A3110F4075006C0812F81568A31FC
:10F1200050F5012F0755802F90E08C179D071CF597
:10F130006F3FE9F0A216B306C406D506A8F0CA01CF
:10F14000B901A20191010E94D4769B01AC01802FEC
:10F1500090E0A0E0B0E0280F391F4A1F5B1F28177E
:10F1600039074A075B0710F46FEF01C061E0F70150
:10F1700011917F01C8CF6114710481F0662339F0C9
:10F180000894E108F108F301F182E08207C091FEE2
:10F1900005C0C7010297F3019183808390FE07C0E9
:10F1A00050954095309521953F4F4F4F5F4F67FFEA
:10F1B0000DC082E290E09093812D8093802D2FEFFF
:10F1C0003FEFA90103C020E030E0A901B901CA0165
:10F1D000DF91CF911F910F91FF90EF90DF90CF9033
:10F1E000BF90AF909F907F906F905F904F903F90B7
:10F1F0002F900895662777270C94197CFC018827A7
:10F200009927E89421912032E9F3293010F02E302B
:10F21000C8F32B3241F02D3239F4689404C00E94B7
:10F22000667A820F911D219120532A30C0F31EF47B
:10F23000909581959F4F0895283008F027E0332757
:10F24000DA01990F311D87FD916000966105710506
:10F2500039F432602E5F3D9330E32A95E1F708954B
:10F260009F3F30F080387105610509F03C5F3C5FDD
:10F270003D93913008F08068911DDF93CF931F93E9
:10F280000F93FF92EF92192F987F9695E92F9695FD
:10F290009695E90FFF27E057F04F99273327EE2483
:10F2A000FF24A701E70105900894079428F4360F7E
:10F2B000E71EF81E491F511D660F771F881F991FF3
:10F2C0000694A1F70590079428F4E70EF81E491F4D
:10F2D000561FC11D770F881F991F661F0694A1F73F
:10F2E0000590079428F4F80E491F561FC71FD11D1B
:10F2F000880F991F661F771F0694A1F70590079442
:10F3000020F4490F561FC71FD81F990F661F771F7C
:10F31000881F0694A9F784911095177041F0D6952F
:10F32000C79557954795F794E7941A95C1F7E6E383
:10F33000FFE0689415901591359165919591059030
:10F340007FE27395E118F10A430B560BC90BD00904
:10F35000C0F7E10CF11E431F561FC91FD01D7EF4DC
:10F36000703311F48A95E6CFE894015030F0080F1D
:10F370000AF40027021708F4202F2395022F7A336E
:10F3800028F079E37D932A95E9F710C07D932A95BB
:10F3900089F6069497956795379517951794E11810
:10F3A000F10A430B560BC90BD00998F023957E91B7
:10F3B00073957A3308F070E37C932013B8F77E914D
:10F3C00070617D9330F0839571E37D9370E32A95AE
:10F3D000E1F71124EF90FF900F911F91CF91DF91F2
:10F3E000992787FD909508959111B1C3803219F046
:10F3F00089508550D0F70895FC0105906150704008
:10F400000110D8F7809590958E0F9F1F08954AE7B9
:10F4100057E10E943F7A0895FB01DC0102C0019090
:10F420000D9241505040D8F70895DC0101C06D9312
:10F4300041505040E0F70895FB01DC018D910190AF
:10F4400080190110D9F3990B0895FB01DC0141509B
:10F45000504048F001900D920020C9F701C01D9264
:10F4600041505040E0F70895FC0161507040019018
:10F470000110D8F7809590958E0F9F1F0895FA017F
:10F48000A191B081009719F41097E1F0CD01DC0152
:10F49000CD010D90002011F4C00113C0FB0121919A
:10F4A000222319F02015D9F7F3CFFB012191201564
:10F4B00019F41E92119606C02223C1F70D90002068
:10F4C000A1F7D001FA01A193B08308957AE0979F44
:10F4D000902D879F802D910D112408950F931F93D8
:10F4E000CF93DF938C01EB018B8181FF1BC082FFE7
:10F4F0000DC02E813F818C819D812817390764F4CE
:10F50000E881F9810193F983E88306C0E885F985EC
:10F51000802F0995009731F48E819F8101969F83FA
:10F520008E8302C00FEF1FEFC801DF91CF911F91B3
:10F530000F910895DF93CF93CDB7DEB7FE013596D7
:10F540006191719180917C2D90917D2DAF010E94F0
:10F55000DA6FCF91DF910895DF93CF93CDB7DEB708
:10F56000FE0135966191719180917C2D90917D2D58
:10F57000DC0113962C911397286013962C93AF01FE
:10F580000E94DA6FE0917C2DF0917D2D2381277F01
:10F590002383CF91DF91089560917C2D70917D2D13
:10F5A0000E946E7A0895EF92FF920F931F93CF936C
:10F5B000DF938C01E0917C2DF0917D2D838181FF83
:10F5C0001FC0C0E0D0E00AC0DB011896ED91FC91AD
:10F5D00019970995009711F0CFEFDFEFF8018191AE
:10F5E0008F0160917C2D70917D2D882369F7DB015F
:10F5F0001896ED91FC9119978AE00995009711F002
:10F60000CFEFDFEFCE01DF91CF911F910F91FF90F0
:10F61000EF9008950F931F93DF93CF93CDB7DEB78D
:10F620002E970FB6F894DEBF0FBECDBF0D891E8991
:10F630008F89988D26E02C831A83098397FF02C057
:10F6400080E090E801979E838D839E01255E3F4F69
:10F65000CE010196698D7A8DA9010E94DA6F4D81E4
:10F660005E8157FD0AC02F813885421753070CF47D
:10F670009A01020F131FF80110822E960FB6F8940C
:10F68000DEBF0FBECDBFCF91DF911F910F910895C7
:10F690000F931F93DF93CF93CDB7DEB72E970FB69F
:10F6A000F894DEBF0FBECDBF8C01CB01BA0146E09E
:10F6B0004C831A83098397FF02C080E090E801978A
:10F6C0009E838D83CE010196A9010E94DA6F4D8140
:10F6D0005E8157FD0AC02F813885421753070CF40D
:10F6E0009A01020F131FF80110822E960FB6F8949C
:10F6F000DEBF0FBECDBFCF91DF911F910F91089557
:10F70000FA01AA27283051F1203181F1E8946F9352
:10F710006E7F6E5F7F4F8F4F9F4FAF4FB1E03ED0F8
:10F72000B4E03CD0670F781F891F9A1FA11D680F96
:10F73000791F8A1F911DA11D6A0F711D811D911DC9
:10F74000A11D20D009F468943F912AE0269F11243E
:10F750003019305D3193DEF6CF010895462F4770A2
:10F76000405D4193B3E00FD0C9F7F6CF462F4F70FD
:10F77000405D4A3318F0495D31FD4052419302D05B
:10F78000A9F7EACFB4E0A695979587957795679501
:10F79000BA95C9F700976105710508959B01AC0101
:10F7A0000A2E06945795479537952795BA95C9F728
:10F7B000620F731F841F951FA01D0895DC01CB01EC
:10F7C000FC01F999FECF06C0F2BDE1BDF89A319671
:10F7D00000B40D9241505040B8F70895F999FECF0A
:10F7E00092BD81BDF89A992780B50895A8E1B0E04F
:10F7F00042E050E00C94E07BDC01CB0103C02D9192
:10F800000E94077C41505040D0F70895262FF99967
:10F81000FECF1FBA92BD81BD20BD0FB6F894FA9AF3
:10F82000F99A0FBE019608950E94067C272F0C942A
:10F83000077C6F927F928F929F92AF92BF92CF92EE
:10F84000DF92EF92FF920F931F93DF93CF930F926C
:10F85000CDB7DEB75B016115710521F0DB018C933B
:10F8600011969C93482F592F6A01F601E1906F0180
:10F870008F018E2D90E00E94F4790097B1F7FE2D54
:10F88000FD3229F4D601ED908D0121E007C0BE2D97
:10F89000BB3219F4F601E1908F0120E06801089471
:10F8A000C108D108C60160E370E143E050E029835C
:10F8B0000E94AA7D2981009711F572E0E72EF12CB4
:10F8C000E00EF11EC70163E370E145E050E00E94E5
:10F8D000AA7D2981009729F467E0E62EF12CE00E3D
:10F8E000F11EA114B10421F0D5011196FC92EE9203
:10F8F00020FF0FC130E020E090E88FEF12C1C60179
:10F9000068E370E143E050E029830E94AA7D2981E9
:10F91000009731F060E070E0CB01662477240AC0E4
:10F92000A114B10409F4F9C00E5F1F4FF501118352
:10F930000083F3C03E2D30533A30A0F52260E22F11
:10F94000F0E0AF014870507022FF07C0411551052B
:10F9500071F50894611C711C2AC04115510519F0FC
:10F960000894610871086B017C0152E0CC0CDD1C2D
:10F97000EE1CFF1C5A95D1F76C0D7D1D8E1D9F1D31
:10F98000660F771F881F991F630F711D811D911DC1
:10F990006839F9E97F07F9E98F07F9E19F0738F03E
:10F9A000246005C03E3F39F423FD3FC02860D801E4
:10F9B000ED908D01BFCF353311F03531B1F5F80140
:10F9C00031913D3211F4206102C03B3241F4D80143
:10F9D00011963C911197319642E050E002C041E00F
:10F9E00050E030533A3020F08F01041B150B1DC03E
:10F9F00040E050E0BCE040385B075CF4DA01AA0F5D
:10FA0000BB1FAA0FBB1F4A0F5B1F440F551F430F9D
:10FA1000511D319130538F013A3060F324FF03C000
:10FA2000509541955F4F640E751EC22EDD2421FF57
:10FA300008C0A114B10429F001501040F501118350
:10FA400000830E945A747B018C01F3E0CF22DD24F5
:10FA500033E0C316D10421F417FB109517F9109564
:10FA6000C801B70120E030E0A9010E94EE738823AD
:10FA700009F44AC077FE09C04FE4C42E40E1D42EF9
:10FA8000709461947108739404C037E6C32E30E11A
:10FA9000D32E26E0822E912C90E2A92EB12C0FC0FD
:10FAA000F6012591359145915491C801B7010E9405
:10FAB0000C75E62EF72E082F192F6A187B086A148A
:10FAC0007B0474F7B594A794089481089108811475
:10FAD000910429F08CEF9FEFC80ED91EF0CFB7012B
:10FAE000C801282F220F292F221F2F3F39F020E095
:10FAF00030E0A9010E94EE73882331F482E290E0A5
:10FB00009093812D8093802D3E2D2F2D902F812F2E
:10FB100008C030E020E090E803C030E020E090EC46
:10FB20008FE7F901AC016F2F722F852F942F0F9063
:10FB3000CF91DF911F910F91FF90EF90DF90CF90C9
:10FB4000BF90AF909F908F907F906F90089599276E
:10FB500088270895FB01DC014150504088F08D91C9
:10FB600081341CF08B350CF4805E659161341CF09F
:10FB70006B350CF4605E861B611171F3990B08956F
:08FB8000881BFCCFF894FFCFB5
:10FB8800263A202573205B414444523D252D642E9E
:10FB9800252D64205345513D252D642054544C3D5A
:10FBA800252D7520525353493D252D75204C51491B
:10FBB8003D252D75204452503D252D642E2530328B
:10FBC800645D0A00523D252D75204C3D252D75207C
:10FBD800533D252D64200054696D656F757420416F
:10FBE8004444523D252D642E252D64205345513D16
:10FBF800252D6420525353493D252D75204C5149DC
:10FC08003D252D750A002845787450777229000023
:10FC180045554936343D00253032582D00253032BF
:10FC2800580A00534E3D00413A202564202564209F
:10FC38002564200A00433A20256420256420256491
:10FC4800200A007374617475733D307825303278FA
:10FC58000A20006669726D776172653D53312D35F2
:10FC68002E332D323031342D30382D313700656543
:10FC780070726F6D006F6E006F666600666F7263FC
:10FC8800655F69646C650064656570004F6E00614E
:10FC980031007265736574006E6F6E6500613200C5
:10FCA800765F696E0031003200330034006175748C
:10FCB8006F00666C75736800414444523D252D649D
:10FCC8002E252D64205345513D252D642052535334
:10FCD800493D252D75204C51493D252D750A00704B
:10FCE8007772733D25730A007472696D00747874B5
:10FCF8003D25730A00746573740043683D252D64BF
:10FD08002054785077723D252D640A004572726F31
:10FD180072205458204C656E6774683D25640A004B
:10FD28005458543D2573200049443D00253032780D
:10FD3800002050533D25640020543D252D362E3299
:10FD480066002054313D252D362E32660020545F42
:10FD58004D43553D252D352E31660020565F4D43C8
:10FD6800553D252D342E3266002050303D30782503
:10FD78002D6C58002050305F543D252D372E3366AA
:10FD8800002050313D3078252D6C58002050315FCF
:10FD9800543D252D372E3366002055503D307825AB
:10FDA8002D6C58002052483D252D342E31660020F8
:10FDB800565F494E3D252D352E32660020565F414F
:10FDC800313D252D352E32660020565F41323D25C6
:10FDD8002D352E32660020503D252D6C64002050B4
:10FDE800413D252D372E326600263A2025730A001C
:10FDF800545820706B74206C656E203D2025640A71
:10FE08000025303258006C656E3D25640A000100FB
:10FE1800ED478A3C22FFCC3B22FFCC3B1A20090D40
:10FE2800009D046162636465666768696A6B6C6DEE
:10FE38006E6F70261400003C000A00636D64207029
:10FE4800726F63657373000000BB046E33000000BB
:10FE580000737464696E2070726F63657373000059
:10FE680000D104120F0000000062726F61646361C8
:10FE780073742070726F63657373000000E9044146
:10FE88003400000000536C6565702070726F636504
:10FE98007373000000050502100000000050657231
:10FEA800696F6469632070726F6365737300000023
:10FEB8001D05B11600000000C704DF04FB042E0571
:10FEC80013050000790800001D00400004074407DE
:10FED80010000000BD3BB13B181000000000457643
:10FEE800656E742074696D65720000005E05C83F18
:10FEF800000000004374696D65722070726F63655D
:10FF08007373000000740506410000000002030638
:10FF1800070A0B0E0F020306070A0B0E0F284329C8
:10FF28002032303132204865726A756C660055742B
:10FF38007665636B6C696E67202020202020004363
:10FF48006F6E74696B6920322E3500000000020064
:10FF5800000000414F00000000C600C500C400C1F9
:10FF680000C200000000CE00CD00CC00C900CA00CD
:10FF780000000052463233302064726976657200A0
:10FF88000000F305F853000000006952E751475498
:10FF980091550A539A51085002508951EB5000016B
:10FFA80001010101010101010101010101010052E9
:10FFB800696D65002F060C57D35661646174612E14
:10FFC8006E756D20776179206F757420746865721D
:10FFD800653A2025640A004E584D58575A865BBE2C
:10FFE800590080C0E0F0F8FCFEFF6E756C6C6D6126
:08FFF80063006A06395C1E5C1F
:020000021000EC
:10000000245C2A5C305C365C736963736C6F776D5B
:1000100061630080065A5DBB5C515C3A5C405C4E9B
:100020005CBA00080003110B1135000200DB16DD7D
:10003000165443502F495020737461636B000000C5
:10004000A906B45F000000000208FFFFFFFF0000E8
:06005000000001000000A9
:00000001FF
